:020000040800F2
:1000000000800120891B0408837201088F72010897
:10001000957201089B720108A5720108000000009A
:10002000000000000000000000000000AB720108AA
:10003000B772010800000000C3720108CF72010806
:10004000CD1B0408CD1B0408CD1B0408A3740108B4
:10005000CD1B0408CD1B0408D9720108F7720108F2
:10006000157301083373010851730108CD1B04088F
:10007000CD1B0408CD1B0408CD1B0408CD1B0408B0
:10008000CD1B0408CD1B0408CD1B04080000000094
:100090000000000000000000000000006F73010875
:1000A000CD1B0408CD1B0408CD1B0408CD1B040880
:1000B000CD1B0408CD1B0408CD1B0408CD1B040870
:1000C000CD1B0408CD1B0408CD1B04087576010860
:1000D0008976010801760108157601080000000004
:1000E000F5730108CD1B0408CD1B040800000000B7
:1000F000000000000000000000000000CD1B04080C
:1001000000000000CD1B0408616701089D7601080E
:1001100000000000000000000000000000000000DF
:10012000CD1B0408CD1B0408CD1B0408CD1B0408FF
:10013000CD1B0408000000000000000000000000CB
:10014000000000000000000000000000CD1B0408BB
:10015000CD1B0408CD1B0408CD1B0408297601081B
:10016000CD1B0408CD1B04080000000000000000A7
:10017000000000000000000000000000000000007F
:1001800000000000CD1B040800000000000000007B
:04019000CD1B040877
:08019400B40A000001000000A4
:1001A00081F0004102E000BF83F0004330B54FEA28
:1001B00041044FEA430594EA050F08BF90EA020F95
:1001C0001FBF54EA000C55EA020C7FEA645C7FEA28
:1001D000655C00F0E2804FEA5454D4EB5555B8BF4B
:1001E0006D420CDD2C4480EA020281EA030382EABC
:1001F000000083EA010180EA020281EA0303362D4E
:1002000088BF30BD11F0004F4FEA01314FF4801C20
:100210004CEA113102D0404261EB410113F0004F32
:100220004FEA03334CEA133302D0524263EB4303E9
:1002300094EA050F00F0A780A4F10104D5F1200E87
:100240000DDB02FA0EFC22FA05F2801841F10001E2
:1002500003FA0EF2801843FA05F359410EE0A5F1B6
:1002600020050EF1200E012A03FA0EFC28BF4CF0E7
:10027000020C43FA05F3C01851EBE37101F000459D
:1002800007D54FF0000EDCF1000C7EEB00006EEBAA
:100290000101B1F5801F1BD3B1F5001F0CD3490834
:1002A0005FEA30004FEA3C0C04F101044FEA44528B
:1002B00012F5800F80F09A80BCF1004F08BF5FEA12
:1002C000500C50F1000041EB045141EA050130BDF2
:1002D0005FEA4C0C404141EB010111F4801FA4F195
:1002E0000104E9D191F0000F04BF01460020B1FAEA
:1002F00081F308BF2033A3F10B03B3F120020CDA22
:100300000C3208DD02F1140CC2F10C0201FA0CF0FF
:1003100021FA02F10CE002F11402D8BFC2F1200C64
:1003200001FA02F120FA0CFCDCBF41EA0C0190401A
:10033000E41AA2BF01EB0451294330BD6FEA040463
:100340001F3C1CDA0C340EDC04F11404C4F120024E
:1003500020FA04F001FA02F340EA030021FA04F360
:1003600045EA030130BDC4F10C04C4F1200220FAB7
:1003700002F001FA04F340EA0300294630BD21FAF5
:1003800004F0294630BD94F0000F83F4801306BFBB
:1003900081F480110134013D4EE77FEA645C18BFAF
:1003A0007FEA655C29D094EA050F08BF90EA020F46
:1003B00005D054EA000C04BF1946104630BD91EA3E
:1003C000030F1EBF0021002030BD5FEA545C05D141
:1003D0004000494128BF41F0004130BD14F5800480
:1003E0003CBF01F5801130BD01F0004545F0FE41F4
:1003F00041F470014FF0000030BD7FEA645C1ABF29
:10040000194610467FEA655C1CBF0B46024650EA5F
:10041000013406BF52EA033591EA030F41F400218B
:1004200030BD00BF90F0000F04BF0021704730B511
:100430004FF4806404F132044FF000054FF00001E6
:1004400050E700BF90F0000F04BF0021704730B5A7
:100450004FF4806404F1320410F0004548BF40427C
:100460004FF000013EE700BF42004FEAE2014FEAD1
:1004700031014FEA02701FBF12F07F4393F07F4FAC
:1004800081F06051704792F0000F14BF93F07F4FDE
:10049000704730B54FF4607401F0004521F0004121
:1004A00020E700BF50EA010208BF704730B54FF0A7
:1004B00000050AE050EA010208BF704730B511F0AC
:1004C000004502D5404261EB41014FF4806404F1E4
:1004D00032045FEA915C3FF4DCAE4FF003025FEA66
:1004E000DC0C18BF03325FEADC0C18BF033202EBEE
:1004F000DC02C2F1200300FA03FC20FA02F001FA48
:1005000003FE40EA0E0021FA02F11444C1E600BFE6
:1005100070B54FF0FF0C4CF4E06C1CEA11541DBF99
:100520001CEA135594EA0C0F95EA0C0F00F0DEF864
:100530002C4481EA030621EA4C5123EA4C5350EA49
:10054000013518BF52EA033541F4801143F480139A
:1005500038D0A0FB02CE4FF00005E1FB02E506F02B
:100560000042E0FB03E54FF00006E1FB03569CF080
:10057000000F18BF4EF0010EA4F1FF04B6F5007F86
:1005800064F5407404D25FEA4E0E6D4146EB0606F8
:1005900042EAC62141EA55514FEAC52040EA5E5081
:1005A0004FEACE2EB4F1FD0C88BFBCF5E06F1ED82B
:1005B000BEF1004F08BF5FEA500E50F1000041EB62
:1005C000045170BD06F0004646EA010140EA02000F
:1005D00081EA0301B4EB5C04C2BFD4EB0C0541EA31
:1005E000045170BD41F480114FF0000E013C00F346
:1005F000AB8014F1360FDEBF002001F0004170BD6A
:10060000C4F10004203C35DA0C341BDC04F1140482
:10061000C4F1200500FA05F320FA04F001FA05F20E
:1006200040EA020001F0004221F0004110EBD370DB
:1006300021FA04F642EB06015EEA430E08BF20EA07
:10064000D37070BDC4F10C04C4F1200500FA04F3AA
:1006500020FA05F001FA04F240EA020001F000413C
:1006600010EBD37041F100015EEA430E08BF20EAAF
:10067000D37070BDC4F1200500FA05F24EEA020EF7
:1006800020FA04F301FA05F243EA020321FA04F026
:1006900001F0004121FA04F220EA020000EBD370DD
:1006A0005EEA430E08BF20EAD37070BD94F0000FDD
:1006B0000FD101F00046400041EB010111F4801F11
:1006C00008BF013CF7D041EA060195F0000F18BFC2
:1006D000704703F00046520043EB030313F4801FFE
:1006E00008BF013DF7D043EA0603704794EA0C0FB8
:1006F0000CEA135518BF95EA0C0F0CD050EA4106CE
:1007000018BF52EA4306D1D181EA030101F000414A
:100710004FF0000070BD50EA410606BF1046194672
:1007200052EA430619D094EA0C0F02D150EA01367E
:1007300013D195EA0C0F05D152EA03361CBF1046BF
:1007400019460AD181EA030101F0004141F0FE415E
:1007500041F470014FF0000070BD41F0FE4141F4E2
:10076000780170BD70B54FF0FF0C4CF4E06C1CEAE2
:1007700011541DBF1CEA135594EA0C0F95EA0C0F97
:1007800000F0A7F8A4EB050481EA030E52EA033552
:100790004FEA013100F088804FEA03334FF0805573
:1007A00045EA131343EA12634FEA022245EA1115A0
:1007B00045EA10654FEA00260EF000419D4208BF51
:1007C000964244F1FD0404F5407402D25B084FEAFE
:1007D0003202B61A65EB03055B084FEA32024FF4AA
:1007E00080104FF4002CB6EB020E75EB030E22BF07
:1007F000B61A754640EA0C005B084FEA3202B6EBC7
:10080000020E75EB030E22BFB61A754640EA5C0075
:100810005B084FEA3202B6EB020E75EB030E22BF05
:10082000B61A754640EA9C005B084FEA3202B6EB06
:10083000020E75EB030E22BFB61A754640EADC00C5
:1008400055EA060E18D04FEA051545EA16754FEA27
:1008500006164FEAC30343EA52734FEAC2025FEA45
:100860001C1CC0D111F4801F0BD141EA00014FF0D4
:1008700000004FF0004CB6E711F4801F04BF0143A5
:100880000020B4F1FD0C88BFBCF5E06F3FF6AFAEC1
:10089000B5EB030C04BFB6EB020C5FEA500C50F151
:1008A000000041EB045170BD0EF0004E4EEA1131D4
:1008B00014EB5C04C2BFD4EB0C0541EA045170BDDB
:1008C00041F480114FF0000E013C90E645EA060E1F
:1008D0008DE60CEA135594EA0C0F08BF95EA0C0F4D
:1008E0003FF43BAF94EA0C0F0AD150EA01347FF495
:1008F00034AF95EA0C0F7FF425AF104619462CE76C
:1009000095EA0C0F06D152EA03353FF4FDAE1046CE
:10091000194622E750EA410618BF52EA43067FF41F
:10092000C5AE50EA41047FF40DAF52EA43057FF4AF
:10093000EBAE12E74FF0FF3C06E000BF4FF0010CBA
:1009400002E000BF4FF0010C4DF804CD4FEA410C1E
:100950007FEA6C5C4FEA430C18BF7FEA6C5C1BD0EB
:1009600001B050EA410C0CBF52EA430C91EA030F6C
:1009700002BF90EA020F0020704710F1000F91EAC9
:10098000030F58BF994208BF90422CBFD8176FEA97
:10099000E37040F0010070474FEA410C7FEA6C5C65
:1009A00002D150EA013C07D14FEA430C7FEA6C5C6C
:1009B000D6D152EA033CD3D05DF8040B704700BF98
:1009C0008446104662468C461946634600E000BFE6
:1009D00001B5FFF7B7FF002848BF10F1000F01BDB8
:1009E0004DF808EDFFF7F4FF0CBF012000205DF883
:1009F00008FB00BF4DF808EDFFF7EAFF34BF012008
:100A000000205DF808FB00BF4DF808EDFFF7E0FFA0
:100A100094BF012000205DF808FB00BF4DF808EDF1
:100A2000FFF7CEFF94BF012000205DF808FB00BF58
:100A30004DF808EDFFF7C4FF34BF012000205DF83A
:100A400008FB00BF4FEA410C7FEA6C5C02D150EA20
:100A5000013C0AD14FEA430C7FEA6C5C02D152EAB6
:100A6000033C02D14FF0000070474FF00100704787
:100A70004FEA410212F5001215D211D56FF47873C6
:100A8000B3EB625212D94FEAC12343F0004343EA69
:100A9000505311F0004F23FA02F018BF4042704744
:100AA0004FF00000704750EA013005D111F00040CE
:100AB00008BF6FF0004070474FF00000704700BF64
:100AC0004A0011D212F5001211D20DD56FF47873CD
:100AD000B3EB62520ED44FEAC12343F0004343EA22
:100AE000505323FA02F070474FF00000704750EA6D
:100AF000013002D14FF0FF3070474FF000007047D7
:100B00004FEA4102B2F1E04324BFB3F5001CDCF12F
:100B1000FE5C0DD901F0004C4FEAC0024CEA507067
:100B2000B2F1004F40EB830008BF20F00100704796
:100B300011F0804F21D113F13872BCBF01F0004099
:100B4000704741F480114FEA5252C2F11802C2F1CB
:100B5000200C10FA0CF320FA02F018BF40F001004C
:100B60004FEAC1234FEAD32303FA0CFC40EA0C00FE
:100B700023FA02F34FEA4303CCE77FEA625307D13B
:100B800050EA01331EBF4FF0FE4040F44000704772
:100B900001F0004040F0FE4040F40000704700BF0C
:100BA00053B94AB9002908BF00281CBF4FF0FF31D4
:100BB0004FF0FF3000F0B6B9ADF1080C6DE904CE8E
:100BC00000F042F8DDF804E0DDE9022304B07047EC
:100BD00038B50022002304460D46FFF70BFF28B965
:100BE00020462946BDE8384000F00AB8204605F105
:100BF000004100F005F8404261EB410138BD00BF03
:100C0000D0B500220E4B06460F46FFF781FCFFF7DA
:100C100057FF0446FFF706FC00220A4BFFF778FC5B
:100C200002460B4630463946FFF7BEFAFFF748FF4B
:100C30002346002242EA000210461946D0BD00BFFA
:100C40000000F03D0000F0412DE9F0478C460D46D4
:100C50000446089E002B51D18A4217466DD9B2FA3C
:100C600082FEBEF1000F0BD0CEF1200C01FA0EF582
:100C700020FA0CFC02FA0EF74CEA050C00FA0EF40E
:100C80004FEA174A250CBCFBFAF81FFA87F90AFB52
:100C900018CC45EA0C4508FB09F3AB420AD9ED191B
:100CA00008F1FF3280F02381AB4240F22081A8F1AD
:100CB00002083D44ED1AA4B2B5FBFAF00AFB105548
:100CC00044EA054400FB09F9A14509D9E41900F1FA
:100CD000FF3380F00A81A14540F2078102383C448D
:100CE000A4EB090440EA08400021002E61D024FA58
:100CF0000EF4002334607360BDE8F0878B4207D99F
:100D0000002E54D0002186E821000846BDE8F08777
:100D1000B3FA83F1002940F08E80AB4202D38242C5
:100D200000F2FA80841A65EB03050120AC46002E20
:100D30003FD086E81010BDE8F08712B90127B7FB55
:100D4000F2F7B7FA87FEBEF1000F34D1EB1B3A0C75
:100D50001FFA87FC0121B3FBF2F8250C02FB1833C4
:100D600045EA03450CFB08F3AB4207D9ED1908F13E
:100D7000FF3002D2AB4200F2D1808046ED1AA3B21E
:100D8000B5FBF2F002FB105543EA05440CFB00FCF6
:100D9000A44507D9E41900F1FF3302D2A44500F2BB
:100DA000B8801846A4EB0C0440EA08409DE73146A1
:100DB0003046BDE8F087CEF1200405FA0EF307FABD
:100DC0000EF720FA04F83A0C25FA04F448EA03086E
:100DD000B4FBF2F14FEA184502FB11441FFA87FCFD
:100DE00045EA044501FB0CF3AB4200FA0EF409D9C5
:100DF000ED1901F1FF3080F08A80AB4240F287802C
:100E000002393D44EB1A1FFA88F5B3FBF2F002FBFE
:100E1000103345EA034500FB0CF3AB4207D9ED194B
:100E200000F1FF386FD2AB426DD902383D44EB1A66
:100E300040EA01418FE7C1F1200722FA07F88B4011
:100E400005FA01F448EA030320FA07FE4FEA134CBF
:100E5000FD404EEA040EB5FBFCF94FEA1E440CFBC4
:100E600019551FFA83F844EA054509FB08F4AC421A
:100E700002FA01F200FA01FA08D9ED1809F1FF307F
:100E800043D2AC4241D9A9F102091D442D1B1FFADE
:100E90008EFEB5FBFCF00CFB10554EEA054400FB42
:100EA00008F8A04507D9E41800F1FF3529D2A0457C
:100EB00027D902381C4440EA0940A4EB0804A0FBEF
:100EC00002894C45C6464D4615D312D056B1BAEBF1
:100ED0000E0364EB050404FA07F7CB401F43CC4034
:100EE000376074600021BDE8F0871846F8E6904648
:100EF000E0E6C245EAD2B8EB020E69EB0305013821
:100F0000E4E72846D7E7404691E78146BEE7014639
:100F100078E702383C4445E7084608E7A8F10208AC
:100F20003D442BE7704700BF10F8012B11F8013B3F
:100F3000012A28BF9A42F7D0D01A7047034613F807
:100F4000012B002AFBD1181A0138704702440346CE
:100F5000934200D1704703F8011BF9E780B483B0D6
:100F600000AF786008497B689BB243F08003DA43A6
:100F7000054BDB6803F080031343CB600C37BD46A1
:100F80005DF8047B704700BF0028004080B487B044
:100F900000AF78600023FB7500233B610023FB60FA
:100FA000134B1B6C03F004033B61114B9A687B6885
:100FB0001A407B68D90B3B690B401343FB600C4B19
:100FC000DA687B681B0913403B61FB68002B06D085
:100FD0003B699BB2002B02D00123FB7501E000238B
:100FE000FB75FB7D18461C37BD465DF8047B7047DA
:100FF0000028004080B485B000AF78600023FB601B
:101000007B681B09FB600849FB689BB243F08003C7
:10101000DA43054BDB6803F080031343CB601437DE
:10102000BD465DF8047B70470028004080B485B061
:1010300000AF786039600023FB817B681B68FB810F
:10104000FB8903F44153FB813B681A883B685B884A
:1010500013439AB23B689B8813439AB23B68DB8880
:1010600013439AB23B681B8913439AB23B685B896E
:1010700013439AB23B689B8913439AB23B68DB895E
:1010800013439AB2FB891343FB81FA897B681A6088
:101090007B68DA694FF2FF7313407A68D3613B686B
:1010A0001B8A1A467B681A611437BD465DF8047BBB
:1010B000704780B483B000AF78600B46FB70FB785C
:1010C000002B06D07B681B6843F040027B681A60E7
:1010D00006E07B681A684FF6BF7313407A681360A6
:1010E0000C37BD465DF8047B704780B483B000AF19
:1010F00078600B467B807B681A684FF2FF73134061
:101100007A6813607B681A687B881A437B681A6068
:101110000C37BD465DF8047B704780B483B000AFE8
:1011200078607B68DB689BB218460C37BD465DF87B
:10113000047B704780B483B000AF78600B467B803F
:101140007A887B68DA600C37BD465DF8047B7047AF
:1011500080B485B000AF78600B46FB701346BB705F
:101160000023FB810023BB81FB781B09DBB2FB81E1
:10117000FB89012202FA03F3BB81BB78002B06D066
:101180007B685A68BB891A437B685A6007E07B68B2
:101190005B68BA89D24392B21A407B685A601437AE
:1011A000BD465DF8047B704780B485B000AF7860C1
:1011B0000B467B800023FB737B689A687B88134017
:1011C000002B02D00123FB7301E00023FB73FB7BA8
:1011D00018461437BD465DF8047B704780B485B06F
:1011E00000AF78600B46FB700023FB730023BB81CC
:1011F00000237B8100233B81FB7803F00F03012256
:1012000002FA03F3BB81FB781B09DBB27B817B898C
:10121000012202FA03F37B817B685B689AB27B89C7
:1012200013403B817B689A68BB891340002B05D033
:101230003B89002B02D00123FB7301E00023FB73E9
:10124000FB7B18461437BD465DF8047B70470000F1
:1012500090B484B000AF03460A46FB711346BB71DD
:101260000023FB60BB7903F003039B000F2202FA0B
:1012700003F3FB601649BB799B08DBB21846144A9E
:10128000BB799B08DBB2023352F82320FB68DB43B7
:101290001A40831C41F823200D48BB799B08DBB220
:1012A0001C460B4ABB799B08DBB2023352F8232061
:1012B000F979BB7903F003039B0001FA03F31A43A6
:1012C000A31C40F823201037BD4690BC704700BFD8
:1012D0000038014080B485B000AF786039600023E9
:1012E000FB817B681B68FB817B681C4A93420FD0A3
:1012F0007B68B3F1804F0BD07B68194A934207D0CB
:101300007B68184A934203D07B68174A934208D1FE
:10131000FB8923F07003FB813B685A88FB891343E8
:10132000FB81FA897B681A603B685A687B68DA62DD
:101330003B681B881A467B689A627B68074A93421F
:1013400004D13B689B7A1A467B681A637B6801224A
:101350005A611437BD465DF8047B704700000140B8
:101360000004004000080040000C004080B483B03E
:1013700000AF78607B684FF0FF325A607B680022D4
:101380001A807B6800221A817B6800225A807B6861
:1013900000229A720C37BD465DF8047B704780B41A
:1013A00083B000AF78600B467B8013463B807A8821
:1013B0007B689A623A887B685A610C37BD465DF853
:1013C000047B704780B483B000AF786039607B687D
:1013D0003A68DA620C37BD465DF8047B704780B42A
:1013E00083B000AF78600B46FB70FB78002B06D013
:1013F0007B681B6843F080027B681A6006E07B68AC
:101400001A684FF67F7313407A6813600C37BD4635
:101410005DF8047B704780B483B000AF78600B4602
:10142000FB70FB78002B06D07B681B6843F0010241
:101430007B681A6006E07B681A684FF6FE731340FB
:101440007A6813600C37BD465DF8047B7047000076
:1014500080B485B000AF7860396000237B810023C1
:10146000FB810023BB817B681A6A4FF6FE73134031
:101470007A6813627B681B6AFB817B685B68BB814F
:101480007B689B697B817B8923F070037B817B89EF
:1014900023F003037B813B681A887B8913437B819C
:1014A000FB8923F00203FB813B689A89FB89134384
:1014B000FB813B685A88FB891343FB817B681C4A8C
:1014C000934223D1FB8923F00803FB813B68DA892F
:1014D000FB891343FB81FB8923F00403FB813B68F9
:1014E0009A88FB891343FB81BB8923F48073BB81FA
:1014F000BB8923F40073BB813B681A8ABB89134301
:10150000BB813B685A8ABB891343BB81BA897B681C
:101510005A607A897B689A613B689A687B685A63EB
:10152000FA897B681A621437BD465DF8047B704700
:101530000000014080B485B000AF786039600023BE
:101540007B810023FB810023BB817B681A6A4FF6F5
:10155000EF7313407A6813627B681B6AFB817B68B8
:101560005B68BB817B689B697B817B8923F4E0435B
:101570007B817B8923F440737B813B681B881B0242
:101580009AB27B8913437B81FB8923F02003FB8183
:101590003B689B891B019AB2FB891343FB813B6823
:1015A0005B881B019AB2FB891343FB817B68204A4D
:1015B00093422BD1FB8923F08003FB813B68DB89BD
:1015C0001B019AB2FB891343FB81FB8923F0400383
:1015D000FB813B689B881B019AB2FB891343FB810B
:1015E000BB8923F48063BB81BB8923F40063BB8187
:1015F0003B681B8A9B009AB2BB891343BB813B6843
:101600005B8A9B009AB2BB891343BB81BA897B6812
:101610005A607A897B689A613B689A687B689A63AA
:10162000FA897B681A621437BD465DF8047B7047FF
:101630000000014080B485B000AF786039600023BD
:101640007B810023FB810023BB817B681A6A4FF6F4
:10165000FF6313407A6813627B681B6AFB817B68B7
:101660005B68BB817B68DB697B817B8923F07003CE
:101670007B817B8923F003037B813B681A887B890C
:1016800013437B81FB8923F40073FB813B689B89B7
:101690001B029AB2FB891343FB813B685B881B02E8
:1016A0009AB2FB891343FB817B68204A93422BD17A
:1016B000FB8923F40063FB813B68DB891B029AB240
:1016C000FB891343FB81FB8923F48063FB813B6827
:1016D0009B881B029AB2FB891343FB81BB8923F4CD
:1016E0008053BB81BB8923F40053BB813B681B8AB9
:1016F0001B019AB2BB891343BB813B685B8A1B0108
:101700009AB2BB891343BB81BA897B685A607A89D4
:101710007B68DA613B689A687B68DA63FA897B6880
:101720001A621437BD465DF8047B70470000014023
:1017300080B485B000AF786039600023BB8100239E
:101740007B810023FB817B681A6A4EF6FF7313408E
:101750007A6813627B681B6A7B817B685B68FB81AC
:101760007B68DB69BB81BB8923F4E043BB81BB8918
:1017700023F44073BB813B681B881B029AB2BB8970
:101780001343BB817B8923F400537B813B689B8996
:101790001B039AB27B8913437B813B685B881B03E5
:1017A0009AB27B8913437B817B68104A93420AD1AA
:1017B000FB8923F48043FB813B681B8A9B019AB21F
:1017C000FB891343FB81FA897B685A60BA897B687D
:1017D000DA613B689A687B681A647A897B681A6266
:1017E0001437BD465DF8047B704700BF0000014020
:1017F00080B483B000AF78607B6800221A807B6879
:1018000000225A807B6800229A807B6800229A60BE
:101810007B6800229A817B680022DA817B68002243
:101820001A827B6800225A820C37BD465DF8047B21
:10183000704780B483B000AF786039607B683A68E5
:101840005A630C37BD465DF8047B704780B483B0A3
:1018500000AF786039607B683A689A630C37BD46A0
:101860005DF8047B704780B483B000AF7860396066
:101870007B683A68DA630C37BD465DF8047B7047D5
:1018800080B483B000AF786039607B683A681A64CE
:101890000C37BD465DF8047B704780B485B000AF5F
:1018A00078600B467B800023FB817B689B69FB8112
:1018B000FB8923F00803FB81FA897B881343FB81B2
:1018C000FA897B689A611437BD465DF8047B7047DE
:1018D00080B485B000AF78600B467B800023FB812D
:1018E0007B689B69FB81FB8923F40063FB817B8818
:1018F0001B029AB2FB891343FB81FA897B689A61C8
:101900001437BD465DF8047B704780B485B000AFE6
:1019100078600B467B800023FB817B68DB69FB8161
:10192000FB8923F00803FB81FA897B881343FB8141
:10193000FA897B68DA611437BD465DF8047B70472D
:1019400080B485B000AF78600B467B800023FB81BC
:101950007B68DB69FB81FB8923F40063FB817B8867
:101960001B029AB2FB891343FB81FA897B68DA6117
:101970001437BD465DF8047B704780B483B000AF78
:1019800078600B46FB70FB78002B06D07B685B6CA5
:1019900043F400427B685A6405E07B685B6CC3F3E8
:1019A0000E027B685A640C37BD465DF8047B7047B5
:1019B00080B483B000AF78600B467B8013467B70A9
:1019C0007B78002B06D07B68DA687B881A437B68BB
:1019D000DA6007E07B68DB687A88D24392B21A400B
:1019E0007B68DA600C37BD465DF8047B704780B4D5
:1019F00085B000AF78600B467B800023FB7300232B
:101A0000BB8100237B817B681B699AB27B88134072
:101A1000BB817B68DB689AB27B8813407B81BB8982
:101A2000002B05D07B89002B02D00123FB7301E042
:101A30000023FB73FB7B18461437BD465DF8047B1F
:101A4000704780B483B000AF78600B467B807B88A2
:101A5000DB439BB21A467B681A610C37BD465DF8C2
:101A6000047B704780B58AB000AF7860396000238E
:101A70007B6200233B620023FB610023BB617B6828
:101A80001B697B627B6A23F440537B623B68DB8883
:101A90001A467B6A13437B627B6A9BB21A467B6859
:101AA0001A617B68DB687B627B6A23F4B05323F0A6
:101AB0000C037B623B689A883B681B8913439AB28C
:101AC0003B685B8913439BB21A467B6A13437B6274
:101AD0007B6A9BB21A467B68DA607B685B697B62D3
:101AE0007B6A23F440737B623B689B891A467B6A5E
:101AF00013437B627B6A9BB21A467B685A6107F18B
:101B00000803184600F0D8FC7B68304A934203D0A3
:101B10007B682F4A934202D17B693B6201E03B69BB
:101B20003B627B68DB6803F40043002B0CD03A6A0D
:101B300013469B0013449A001A443B681B685B00E1
:101B4000B2FBF3F3FB610BE03A6A13469B001344CC
:101B50009A001A443B681B689B00B2FBF3F3FB61DD
:101B6000FB691C4AA2FB03235B091B017B627B6AA6
:101B70001B09642202FB03F3FA69D31ABB617B6879
:101B8000DB6803F40043002B0CD0BB69DB0032336D
:101B9000104AA2FB03235B0903F007037A6A13438D
:101BA0007B620BE0BB691B0132330A4AA2FB0323B1
:101BB0005B0903F00F037A6A13437B627B6A9BB273
:101BC0001A467B689A602837BD4680BD00100140E8
:101BD000001401401F85EB5180B485B000AF7860E0
:101BE00039600023FB607B681B69FB60FB6823F4A2
:101BF0007063FB603B681A883B685B8813439AB24A
:101C00003B689B8813439AB23B68DB8813439BB2C3
:101C10001A46FB681343FB60FB689BB21A467B685D
:101C20001A611437BD465DF8047B704780B483B0F9
:101C300000AF78607B6800221A807B6800225A809F
:101C40007B6800229A807B680022DA800C37BD46D0
:101C50005DF8047B704780B483B000AF78600B46BA
:101C6000FB70FB78002B06D07B68DB6843F40052E6
:101C70007B68DA6006E07B68DA684DF6FF73134034
:101C80007A68D3600C37BD465DF8047B704780B43A
:101C900083B000AF78600B467B807B88C3F308027B
:101CA0007B685A600C37BD465DF8047B704780B492
:101CB00083B000AF78607B685B689BB2C3F30803B6
:101CC0009BB218460C37BD465DF8047B704780B464
:101CD00087B000AF78600B467B8013467B70002393
:101CE0003B610023FB600023BB6000237B617B68BA
:101CF0007B617B88DBB25B09DBB23B617B8803F0F5
:101D00001F03FB600122FB6802FA03F3BB603B691F
:101D1000012B03D17B690C337B6109E03B69022B0A
:101D200003D17B6910337B6102E07B6914337B61F3
:101D30007B78002B06D07B697A691168BA680A4300
:101D40001A6006E07B697A691168BA68D2430A4072
:101D50001A601C37BD465DF8047B704780B485B0BF
:101D600000AF78600B467B800023FB737B681A68AA
:101D70007B881340002B02D00123FB7301E000237A
:101D8000FB73FB7B18461437BD465DF8047B704738
:101D900080B487B000AF78600B467B800023FB6087
:101DA00000237B610023BB600023FB747B88DBB2D4
:101DB0005B09DBB2BB607B8803F01F037B61012200
:101DC0007B6902FA03F37B61BB68012B05D17B6859
:101DD000DB687A6913407B610DE0BB68022B05D19B
:101DE0007B681B697A6913407B6104E07B685B69EF
:101DF0007A6913407B617B881B0A9BB2FB600122DE
:101E0000FB6802FA03F3FB607B681B68FA68134007
:101E1000FB607B69002B05D0FB68002B02D00123FF
:101E2000FB7401E00023FB74FB7C18461C37BD46A5
:101E30005DF8047B704780B485B000AF78600B46D6
:101E40007B800023FB810023BB817B881B0AFB81F5
:101E5000FB89012202FA03F3BB81BB89DB439BB2FE
:101E60001A467B681A601437BD465DF8047B7047DC
:101E700080B500AF154A154BD3F8883043F4700392
:101E8000C2F88830124A124B1B6843F001031360FA
:101E90000F4B00229A600E4A0D4B1B6823F084738F
:101EA00023F4803313600A4B0A4A5A60084A084BED
:101EB0001B6823F480231360054B0022DA6000F0D6
:101EC00085F8024B4FF000629A6080BD00ED00E0A3
:101ED000003802401030002480B487B000AF0023E7
:101EE0003B6100237B610223FB600023BB60022374
:101EF0007B60314B9B6803F00C033B613B69042B17
:101F000007D0082B09D0002B3DD12C4B2C4A1A604E
:101F10003CE02A4B2B4A1A6038E0274B5B689B0D4C
:101F200003F00103BB60244B5B6803F03F037B605D
:101F3000BB68002B0CD0234A7B68B2FBF3F31E4A2C
:101F400052689209C2F3080202FB03F37B610BE0C3
:101F50001B4A7B68B2FBF3F3174A52689209C2F33B
:101F6000080202FB03F37B61134B5B681B0C03F05D
:101F7000030301335B00FB607A69FB68B2FBF3F398
:101F80000E4A136002E00D4B0D4A1A600A4B9B6823
:101F90001B0903F00F030C4AD35CDBB23B61074B18
:101FA0001A683B6922FA03F3044A13601C37BD46E2
:101FB0005DF8047B704700BF003802402801002014
:101FC0000024F40000127A002C01002080B483B0B9
:101FD00000AF00237B6000233B60334A324B1B6819
:101FE00043F480331360304B1B6803F400333B60D1
:101FF0007B6801337B603B68002B03D17B68B3F5C2
:10200000A04FF0D1284B1B6803F40033002B02D003
:1020100001233B6001E000233B603B68012B3ED184
:10202000214A214B1B6C43F0805313641F4A1F4B02
:102030001B6843F4404313601B4A1B4B9B6893602F
:10204000194A194B9B689360174A174B9B6843F4D6
:1020500080539360144B164A5A60134A124B1B6804
:1020600043F080731360104B1B6803F00073002B68
:10207000F9D0104B40F202621A600B4A0A4B9B687F
:1020800023F003039360084A074B9B6843F0020365
:102090009360054B9B6803F00C03082BF9D10C37B8
:1020A000BD465DF8047B7047003802400070004078
:1020B00008544107003C024080B483B000AF786010
:1020C0007B6841F288321A607B6800229A807B68C4
:1020D0004BF6FF72DA807B6800221A817B6800224F
:1020E0005A817B684FF480429A810C37BD465DF877
:1020F000047B704780B483B000AF78600B46FB7000
:10210000FB78002B06D07B681B6843F001027B68DC
:102110001A6006E07B681A684FF6FE7313407A680F
:1021200013600C37BD465DF8047B704780B483B004
:1021300000AF78600B46FB70FB78002B06D07B6805
:102140001B6843F480727B681A6006E07B681A683B
:102150004FF6FF6313407A6813600C37BD465DF895
:10216000047B704780B483B000AF78600B46FB708F
:10217000FB78002B06D07B681B6843F400727B68F9
:102180001A6006E07B681A684FF6FF5313407A68BE
:1021900013600C37BD465DF8047B704780B483B094
:1021A00000AF78600B46FB701346BB70BB78002B0A
:1021B00004D0FB7843F00103FB7003E0FB7823F0CD
:1021C0000103FB70FA787B681A610C37BD465DF835
:1021D000047B704780B483B000AF78600B46FB701F
:1021E000FB78002B06D07B681B6843F480627B6819
:1021F0001A6006E07B681A684FF6FF3313407A686E
:1022000013600C37BD465DF8047B704780B483B023
:1022100000AF78600B46FB70FA787B681A610C3768
:10222000BD465DF8047B704780B483B000AF786032
:102230007B681B69DBB218460C37BD465DF8047B32
:10224000704780B487B000AF7860396000233B618D
:102250000023FB600023BB600023FB757B685B6988
:10226000FB607B689B69BB60BB681B04BB60FA6852
:10227000BB68134323F07F433B613A693B681A40D4
:102280003B689A4202D10123FB7501E00023FB75F4
:10229000FB7D18461C37BD465DF8047B704780B453
:1022A00087B000AF786039600023FB7500233B6185
:1022B0000023FB607B68FB603B681B0F3B613B6856
:1022C00023F07F433B603B69002B03D0FB68143352
:1022D000FB6005E03B681B0C3B60FB681833FB6050
:1022E000FB681A683B681340002B02D00123FB7582
:1022F00001E00023FB75FB7D18461C37BD465DF8E9
:10230000047B704780B483B000AF0346FB80044A6F
:10231000FB8813600C37BD465DF8047B704700BF37
:102320000030004080B483B000AF0346FB71044A24
:10233000FB7953600C37BD465DF8047B704700BFE6
:102340000030004080B483B000AF0346FB80044AF5
:10235000FB8893600C37BD465DF8047B704700BF77
:102360000030004080B400AF034B4AF6AA221A6046
:10237000BD465DF8047B70470030004080B400AF7C
:10238000034B4CF6CC421A60BD465DF8047B7047A7
:102390000030004080B483B000AF0346FB71044AB4
:1023A000FB7913600C37BD465DF8047B704700BFB6
:1023B000800E474280B485B000AFF860B9607A60A3
:1023C0003B600A497B689A01BB681A433B685B081B
:1023D000013B1B041A43FB681A43BB691B061343EA
:1023E0004B601437BD465DF8047B704700380240EF
:1023F00080B483B000AF0346FB71044AFB791360DD
:102400000C37BD465DF8047B704700BF6000474253
:1024100080B485B000AF78600023FB60094B9B68F7
:10242000FB60FB6823F00303FB60FA687B681343DF
:10243000FB60044AFB6893601437BD465DF8047B7B
:10244000704700BF0038024080B485B000AF7860AC
:102450000023FB60094B9B68FB60FB6823F4E0539F
:10246000FB60FA687B681343FB60044AFB68936077
:102470001437BD465DF8047B704700BF003802404A
:1024800080B485B000AF78600023FB60094B9B6887
:10249000FB60FB6823F46043FB607B68DB00FA6849
:1024A0001343FB60034AFB6893601437BD465DF835
:1024B000047B70470038024080B489B000AF786078
:1024C0000023BB6100237B610023FB6102233B618E
:1024D0000023FB600223BB60464B9B6803F00C03A8
:1024E000BB61BB69042B07D0082B09D0002B3DD161
:1024F0007B68414A1A603CE07B68404A1A6038E0D9
:102500003C4B5B689B0D03F00103FB60394B5B6840
:1025100003F03F03BB60FB68002B0CD0374ABB685D
:10252000B2FBF3F3334A52689209C2F3080202FB8A
:1025300003F3FB610BE0304ABB68B2FBF3F32D4AB7
:1025400052689209C2F3080202FB03F3FB61294BB4
:102550005B681B0C03F0030301335B003B61FA690A
:102560003B69B2FBF3F27B681A6002E07B68224AA7
:102570001A60204B9B6803F0F003BB61BB691B0929
:10258000BB611F4ABB6913441B78DBB27B617B686C
:102590001A687B69DA407B685A60164B9B6803F4C3
:1025A000E053BB61BB699B0ABB61154ABB6913441D
:1025B0001B78DBB27B617B685A687B69DA407B6899
:1025C0009A600C4B9B6803F46043BB61BB695B0B77
:1025D000BB610B4ABB6913441B78DBB27B617B6830
:1025E0005A687B69DA407B68DA602437BD465DF85B
:1025F000047B7047003802400024F40000127A0087
:102600001801002080B483B000AF78600B46FB70E7
:10261000FB78002B06D00949084B1A6B7B681343E3
:102620000B6306E00549054B1A6B7B68DB431340DF
:102630000B630C37BD465DF8047B704700380240E1
:1026400080B483B000AF78600B46FB70FB78002B42
:1026500006D00949084B1A6C7B6813430B6406E0EB
:102660000549054B1A6C7B68DB4313400B640C3740
:10267000BD465DF8047B70470038024080B483B0EB
:1026800000AF78600B46FB70FB78002B06D0094941
:10269000084B5A6C7B6813434B6406E00549054BB5
:1026A0005A6C7B68DB4313404B640C37BD465DF8C6
:1026B000047B70470038024080B483B000AF78607C
:1026C0000B46FB70FB78002B06D00949084B1A6AB1
:1026D0007B6813430B6206E00549054B1A6A7B6869
:1026E000DB4313400B620C37BD465DF8047B70473B
:1026F0000038024080B487B000AF0346FB7100236E
:10270000FB6000237B610023FB74FB795B09DBB278
:10271000FB60FB68012B03D1124B1B687B6109E056
:10272000FB68022B03D10F4B1B6F7B6102E00D4B4B
:102730005B6F7B61FB7903F01F03FB607A69FB68C9
:1027400022FA03F303F00103002B02D00123FB74F0
:1027500001E00023FB74FB7C18461C37BD465DF886
:10276000047B70470038024080B58EB000AF3B1D3F
:10277000184618F007FE034683F00103DBB2002B76
:1027800001D0002311E0D7F816303A1D10469847C3
:102790003B1D18461AF01AFB034687F837303B1DDD
:1027A000184618F075FE97F8373018463837BD468A
:1027B00080BD80B500AF19F0DBFD80BD80B58EB067
:1027C00000AF18F0C3FD0346002B13D03B1D184685
:1027D00018F0D8FD034683F00103DBB2002B08D1CB
:1027E0003B1D184619F0CAFD3B1D184618F050FE57
:1027F00000E000BF3837BD4680BD000090B599B0FD
:1028000000AF78600B46FB7078683AF0C2FC034674
:1028100083F00103DBB2002B01D000231CE238F06F
:1028200059FFF862FB6A002B01D1002314E207F183
:10283000080300227968184632F04EF90023FB6540
:102840000023BB654FF0FF337B654FF0FF333B65E3
:102850004FF0FF33FB644FF0FF33BB6400237B6416
:1028600000233B6461E007F10803184604F0D1FB44
:10287000034687F82B3097F82B302F2B18D1FB6DA0
:102880000133FB65FB6C002B01DA7B6CFB64BB6DD9
:10289000012B0DD1FB6D022B0AD17B6D002B07DACA
:1028A0007B6C7B654FF0FF33FB644FF0FF33BB6401
:1028B00097F82B303A2B0AD1BB6D0133BB657B6D8A
:1028C000002B04DBFB6C002B01DA7B6C3B653B6D62
:1028D000002B19DB7A6C3B6D9A4215DDFB6C002BEB
:1028E00012DA97F82B302F2B0ED997F82B30392B83
:1028F0000AD83A6C13469B0013445B001A4697F8BB
:102900002B30303B13443B6497F82B303F2B04D1E2
:10291000FB6C002B01DB7B6CBB6407F108031846E2
:1029200032F0ECF97B6C01337B6407F10803184645
:1029300004F085FB0346002B95D107F108031846E8
:1029400004F090FBFB6C002B01DA7B6CFB64FB6CEE
:10295000002B01DA7B6CFB643B6D002B01DB3B6DD4
:1029600000E0FB6C7B627B6D002B0CDD7B6D013B23
:102970001A460021786836F0D7FE03461A46B84951
:10298000F86A36F0FFF8B74838F04CFD03461A46AF
:10299000B549F86A36F0F6F87B6D013319467B6D60
:1029A00001337A6AD31A1A46786836F0BDFE0346B8
:1029B0001A46AE49F86A36F0E5F8FB6C6FF0004253
:1029C0001946786836F0B0FE3862386A39F06DFE24
:1029D0000346002B03D1A649386A36F05DFD3A6AFA
:1029E000A449F86A36F0CEF8F96CBB6C002B03DB17
:1029F000BA6CFB6CD31A01E06FF000431A4678689A
:102A000036F092FE3862386A39F04FFE0346002BEA
:102A100003D19749386A36F03FFD3A6A9649F86A19
:102A200036F0B0F8BB6C002B08DBBB6C6FF00042DB
:102A30001946786836F078FE034602E004F0D2FAD0
:102A400003461A468D49F86A36F09CF83B6C002B19
:102A500003DD3B6CB3F5803F04DB02203BF094FACE
:102A6000034603E0386C38F0A9FD03461A46844952
:102A7000F86A36F087F8BB6C002B09DBBB6C0133BE
:102A80006FF000421946786836F04EFE034602E0C9
:102A900004F0A8FA0346FB63FB78002B00F0D68015
:102AA000F86B3AF03AFD034683F00103DBB2002BEA
:102AB00000F0CC80FB6BFB6107F108030022F96B8F
:102AC000184632F009F838F005FEF86304F07EFA93
:102AD000B86304F07BFA7863002387F8333088E02A
:102AE00007F10803184604F094FA034687F83230D9
:102AF00097F83230262B25D1B86B39F0D6FD034636
:102B0000002B05D1786B39F0D0FD0346002B67D040
:102B1000B86B39F09EFDB863796BB86B38F080FE06
:102B2000B96BF86B35F036FA796BB86B38F09EFA02
:102B300004F04CFAB86304F049FA7863002387F88C
:102B400033304EE097F8333083F00103DBB2002BD3
:102B500007D097F832303D2B03D1012387F833306B
:102B60003FE097F83230252B28D107F108031846AB
:102B700032F0C4F807F10803184604F04AFA034695
:102B800087F8323007F10803184632F0B7F897F8A3
:102B9000323018462FF03FFB03461B015CB207F1B1
:102BA0000803184604F035FA034618462FF033FBA5
:102BB00003465BB223435BB287F8323097F8333079
:102BC000002B06D097F832301946786B04F012FAD1
:102BD00007E097F832301946B86B04F00BFA00E0C2
:102BE00000BF07F10803184632F088F87B6C013308
:102BF0007B6407F10803184604F021FA0346002B12
:102C00007FF46EAF07F10803184604F02BFAF86959
:102C100038F000FAB86B39F048FD0346002B05D1B7
:102C2000786B39F042FD0346002B0BD0B86B39F0BE
:102C300010FDB863796BB86B38F0F2FDB96BF86BC7
:102C400035F0A8F9796BB86B38F010FAFA6B0D49CA
:102C5000F86A35F097FFFB6A18466437BD4690BDA9
:102C6000407B04084C7B0408507B0408587B040814
:102C7000607B0408647B04086C7B0408787B040890
:102C8000807B0408887B040880B584B000AF78603E
:102C9000786837F01DFEF860F8683AF032FB0346BA
:102CA00083F00103DBB2002B08D0F96809482FF04C
:102CB00081FBF86838F0AEF9002307E0F86838F0D7
:102CC000A9F9796800201AF091F9034618461037DF
:102CD000BD4680BD907B040880B594B000AFF8601D
:102CE000B9601346FB71002387F84F30F8683AF05B
:102CF00050FA0346002B07D00021F868FFF77EFD4D
:102D0000F860012387F84F30F8683AF053FB034628
:102D100083F00103DBB2002B05D0F96838482FF0AF
:102D200049FB002367E0B8683AF0E7FB034683F00D
:102D30000103DBB2002B0ED0B8683AF0E2FA03468A
:102D400083F00103DBB2002B05D0B9682D482FF0CA
:102D500031FB00234FE0FB7903F00303022B23D167
:102D600007F11003184618F00DFB0346002B1BD08B
:102D700000222549F86835F015FE0346184637F05D
:102D80008FF9B864D7F81920BB6C9A4207DABB6C8C
:102D9000C7F8193007F11003184618F069FB07F15E
:102DA0001003184618F074FBFB79BA68F9681846E6
:102DB00015F0E0F9786497F84F30002B02D0F868EE
:102DC00038F028F9FB7903F00303002B12D107F147
:102DD0001003184618F024FB0346002B0AD007F115
:102DE0001003796C184615F0CBFB07F11003184659
:102DF00018F04EFB7B6C18465037BD4680BD00BFB7
:102E0000B87B0408907B0408E87B040880B584B094
:102E100000AF7860396078683AF0CCFA0346002B4E
:102E200003D138F057FC034600E07B68FB600222C8
:102E30003968F868FFF750FFB860FA687B689A4213
:102E400002D0F86838F0E6F8BB6818461037BD467F
:102E500080BD000080B598B002AFF860B9607A60BC
:102E60003B60F8683AF0A6FA034683F00103DBB250
:102E7000002B05D0404A40F2E91140482FF052FBA8
:102E8000B8683AF086F9034683F00103DBB2002B01
:102E900005D03B4A4FF4F57138482FF043FB07F15A
:102EA0001003184618F0BCFA034683F00103DBB2A6
:102EB000002B5DD10021386E36F006F9F864F86C0D
:102EC0003AF0FEF90346002B1FD0786836F03CFE3E
:102ED000B864386836F038FE786404F077F87865BE
:102EE0007B6D002B05D107F11003184618F0D0FABE
:102EF0003EE0BA6C7B6CB968786D36F0B7FB0121A7
:102F0000386E36F0E1F8386517E0F86C38F082F882
:102F1000BB687B657B68FB643B683B65F86C3AF09B
:102F2000CFF9034683F00103DBB2002B05D0154A2D
:102F300040F2012111482FF0F5FAF86C36F004FE4A
:102F400003469BB207F1100000933B6D7A6DF96860
:102F500015F08AF97A6DBB689A4204D03A6DF96C23
:102F6000786D38F091F807F11003184618F090FAD0
:102F70005837BD4680BD00BFF87B04080C7C0408B0
:102F8000287C04083C7C040880B584B000AFF8605D
:102F90000B467A607B81FB6818463BF05FFA03467C
:102FA000FB60FB687A680D49184635F073FDFB68D5
:102FB00079890222184600F04FF80346184638F087
:102FC00029F8F86807F10C020123044924F0E4FE13
:102FD000FB6818461037BD4680BD00BF507C040812
:102FE00080B590B000AF786007F10C03184618F078
:102FF00017FA034683F00103DBB2002B0BD107F174
:103000000C037968184615F07FFB07F10C0318468E
:1030100018F03EFA00E000BF4037BD4680BD80B5E5
:1030200092B000AFF860B9607A6007F114031846F7
:1030300018F0F6F9034683F00103DBB2002B07D149
:1030400007F114007B68BA68F96819F0FDFF00E029
:1030500000BF4837BD4680BD80B592B000AFF86074
:10306000B9601346FB71F8683BF0F8F9F86007F1B6
:103070001403184618F0D4F9034683F00103DBB2B9
:10308000002B01D0FB680DE0BB689AB2FB7907F119
:103090001400F96819F0FEFF07F11403184618F040
:1030A000F7F9FB6818464837BD4680BD80B590B03B
:1030B00000AF786007F10C03184618F0B1F9034629
:1030C00083F00103DBB2002B0BD107F10C0379680D
:1030D000184615F01FF807F10C03184618F0D8F938
:1030E00000E000BF4037BD4680BD80B592B002AF62
:1030F0007860396007F10C03184618F091F903461F
:1031000083F00103DBB2002B01D000230EE007F1B6
:103110000C000023009300233A68796815F0A4F8A6
:1031200007F10C03184618F0B3F90023184640378E
:10313000BD4680BD80B590B000AF7860396007F1C2
:103140000C03184618F06CF9034683F00103DBB258
:10315000002B18D138683AF0D0F9034683F0010308
:10316000DBB2002B03D039687868FFF7BEFF07F1A8
:103170000C037968184615F0C7FA07F10C031846D6
:1031800018F086F900E000BF4037BD4680BD000062
:1031900080B584B000AF7860786837F099FBF8604C
:1031A000F8683AF0AEF8034683F00103DBB2002B77
:1031B00008D0F96809482FF0FDF8F86837F02AFFC1
:1031C000002307E0F86837F025FF7968012019F03F
:1031D0000DFF034618461037BD4680BD907B04089E
:1031E00080B592B000AF7860396007F108031846E7
:1031F00018F016F9034683F00103DBB2002B01D06F
:1032000000234AE078683AF0D5F80346002B0DD049
:10321000244838F007F97864234A796C786834F0E8
:10322000B4FF0346796C184637F020FF386837F052
:103230004FFB3864386C3AF060F9034683F00103C1
:10324000DBB2002B11D0386C3AF05BF8034683F008
:103250000103DBB2002B08D0396C14482FF0AAF818
:10326000386C37F0D7FE002317E0386C37F0D2FE09
:10327000012239687868FFF72FFDF863FB6B002B9C
:1032800005D007F10803F96B184615F03DFA07F170
:103290000803184618F0FCF8FB6B18464837BD4683
:1032A00080BD00BF4C7B0408507B0408907B040861
:1032B00080B582B000AF786039603968786815F001
:1032C000E9FA002318460837BD4680BD80B582B0B4
:1032D00000AF7860396038683AF00FF9034683F040
:1032E0000103DBB2002B03D039687868FFF7E0FFF9
:1032F000786815F035FB0837BD4680BD80B584B0D1
:1033000000AFF860B9607A607A68B968F86815F05B
:1033100059FA1037BD4680BD80B590B000AF7860D7
:1033200007F10C030321184617F0D2FF07F10C0335
:10333000184618F09DF807F10C03184618F0A8F885
:10334000786815F05BFB054B02221A7078683BF039
:1033500085F8034618464037BD4680BD8457012096
:1033600090B585B000AF03463960FB710023BB60A8
:1033700007F108031946386839F016FAF860FB6857
:10338000002B23D1386831F059FB0346BB60BB6882
:1033900003F580742FF09EFF03469C4204D9204918
:1033A00001202FF04BF811E0BB6807330733DB082F
:1033B000DB00ADEB030D6B460733DB08DB00FB6086
:1033C000BB681A46F968386831F06CFBFB68002B63
:1033D00005D13A68134901202FF030F81DE0BB6891
:1033E000002B04D1104901202FF028F815E0B9680E
:1033F0000E4BA3FB01235A0813465B001344CA1A61
:10340000002A04D00A4901202FF018F805E0BA6814
:10341000FB79F968184600F00DF81437BD4690BDE9
:10342000587C0408807C0408AC7C0408ABAAAAAAD7
:10343000CC7C040880B58AB000AF0346B9607A60DE
:10344000FB73FB7B18462AF039F9034683F001032E
:10345000DBB2002B05D0584901202EF0EFFF0023EE
:10346000A6E00023FB8400233B624BE0FA7B534839
:103470003B6A590013469B0013445B0013440B4402
:103480000344B3F803309BB203F47F63B3F5007FCA
:1034900035DBFA7B49483B6A590013469B001344CD
:1034A0005B0013440B440344B3F803309BB203F4B2
:1034B0007F63B3F5087F22DCFA7B40483B6A590002
:1034C00013469B0013445B0013440B440344B3F8BE
:1034D00003309BB203F47043B3F5805F0FD1FA7BE6
:1034E00036483B6A590013469B0013445B00134463
:1034F0000B440344DA781B791B021343FB843B6AB9
:1035000001333B623B6A032BB0D9FB8C184625F094
:1035100095FE0346FB77FB8C002B02D0FB7F002B34
:1035200005D1274901202EF089FF002340E007F153
:103530001403184620F015FE224B7B61FB7BFB76C3
:1035400007F11402FB7F1146184612F0F7FBFB7FD0
:103550000121184612F002FEFB7F0021184612F0EE
:103560003FFE16F067F900233B620BE0BA683B6A46
:1035700013441978F87F0C23082220F0E3FC3B6AFF
:1035800001333B623A6A7B689A42EFD3F87F0023AB
:103590000022002120F0D6FC16F053F9FB7F1846DC
:1035A00012F05AFEFB7F0021184612F0D7FD0123CE
:1035B00018462837BD4680BDF87C0408D878040832
:1035C0000C7D040800D4300080B483B000AF786074
:1035D000054A7B6843F0BF6343F40033D3600C3784
:1035E000BD465DF8047B704700ED00E080B485B017
:1035F00000AF78600023FB730023BB730F237B7342
:103600007B68DB78002B39D0274BDB68DB431B0A58
:10361000DBB203F00703FB73FB7BC3F10403BB7353
:103620007A7BFB7B42FA03F37B737B685B781A46F9
:10363000BB7B02FA03F3FB737B689A787B7B1340B6
:10364000DAB2FB7B1343FB73FB7B1B01FB73174A53
:103650007B681B781344FA7B83F80023134A7B684A
:103660001B785B09DBB218467B681B7803F01F03ED
:10367000012101FA03F342F820300FE00B497B6887
:103680001B785B09DBB218467B681B7803F01F03CD
:1036900001229A4000F1200341F823201437BD464F
:1036A0005DF8047B704700BF00ED00E000E100E042
:1036B00080B483B000AF78607B68042B06D1094AE0
:1036C000084B1B6843F00403136005E0054A054BF3
:1036D0001B6823F0040313600C37BD465DF8047BC0
:1036E000704700BF10E000E080B485B000AF7860A4
:1036F00039600023FB600023FB727B685B68FB6022
:10370000FB6823F0407323F48073FB603B681B79F4
:103710001A023B681B681343FA681343FB607B681B
:10372000FA685A607B689B68FB60FA68174B134025
:10373000FB603B681A693B68DB681A433B689B681F
:103740001A433B685B795B001343FA681343FB60E1
:103750007B68FA689A607B68DB6AFB60FB6823F42D
:103760007003FB603B681B7D013BDAB2FB7A1343BD
:10377000FB72FB7A1B05FA681343FB607B68FA68EF
:10378000DA621437BD465DF8047B7047FDF7FFC071
:1037900080B483B000AF78607B6800221A607B68D9
:1037A00000221A717B6800225A717B6800229A609D
:1037B0007B680022DA607B6800221A617B68012244
:1037C0001A750C37BD465DF8047B704780B485B030
:1037D00000AF78600023FB600E4B5B68FB60FA680B
:1037E0000D4B1340FB607B681A687B685B681A436B
:1037F0007B689B681A437B68DB681343FA68134352
:10380000FB60044AFB6853601437BD465DF8047BD7
:10381000704700BF00230140E030FCFF80B483B05C
:1038200000AF78607B6800221A607B6800225A60D3
:103830007B6800229A607B680022DA600C37BD4604
:103840005DF8047B704780B483B000AF78600B46AE
:10385000FB70FB78002B06D07B689B6843F001026D
:103860007B689A6005E07B689B6823F001027B68B7
:103870009A600C37BD465DF8047B704780B483B016
:1038800000AF0346FB71FB79002B06D0084A084BBA
:103890005B6843F40003536005E0054A044B5B6832
:1038A00023F4000353600C37BD465DF8047B70477A
:1038B0000023014080B485B000AF7860084611460F
:1038C0001A460346FB700B46BB7013467B70002301
:1038D000FB600023BB60FB78092B23D97B68DB6886
:1038E000FB60FB78A3F10A0213465B001344072236
:1038F00002FA03F3BB60BB68DB43FA681340FB606A
:103900007978FB78A3F10A0213465B00134401FAAD
:1039100003F3BB60FA68BB681343FB607B68FA681B
:10392000DA601EE07B681B69FB60FA7813465B0077
:103930001344072202FA03F3BB60BB68DB43FA6857
:103940001340FB607978FA7813465B00134401FA60
:1039500003F3BB60FA68BB681343FB607B68FA68DB
:103960001A61BB78062B21D87B685B6BFB60BB7848
:103970005A1E13469B0013441F2202FA03F3BB6036
:10398000BB68DB43FA681340FB60F978BB785A1ECA
:1039900013469B00134401FA03F3BB60FA68BB684B
:1039A0001343FB607B68FA685A6347E0BB780C2BD3
:1039B00021D87B681B6BFB60BB78DA1F13469B002A
:1039C00013441F2202FA03F3BB60BB68DB43FA68AF
:1039D0001340FB60F978BB78DA1F13469B00134451
:1039E00001FA03F3BB60FA68BB681343FB607B68B2
:1039F000FA681A6322E07B68DB6AFB60BB78A3F19C
:103A00000D0213469B0013441F2202FA03F3BB600E
:103A1000BB68DB43FA681340FB60F978BB78A3F11D
:103A20000D0213469B00134401FA03F3BB60FA68CE
:103A3000BB681343FB607B68FA68DA621437BD46E3
:103A40005DF8047B704780B483B000AF78607B681A
:103A50009B6843F080427B689A600C37BD465DF8F6
:103A6000047B704780B483B000AF78607B68DB6C08
:103A70009BB218460C37BD465DF8047B704780B496
:103A800085B000AF78600B46FB700023FB737B684A
:103A90001A68FB781340002B02D00123FB7301E06E
:103AA0000023FB73FB7B18461437BD465DF8047B8F
:103AB0007047000080B485B000AF78600023FB60E1
:103AC000344BFB607B689B79002B4FD03149314BE5
:103AD0001A687B681B68DB4313400B602D492D4B34
:103AE0005A687B681B68DB4313404B607B681B791B
:103AF0001A46FB681344FB60FB68FA6811687A6831
:103B000012680A431A602349224B9A687B681B6833
:103B1000DB4313408B601F491E4BDA687B681B68D0
:103B2000DB431340CB607B685B79102B0ED11949C6
:103B3000184B9A687B681B6813438B601549154BBB
:103B4000DA687B681B681343CB601DE0114BFB6098
:103B50007B685B791A46FB681344FB60FB68FA6874
:103B600011687A6812680A431A600DE07B681B7955
:103B70001A46FB681344FB60FB68FA6811687A68B0
:103B80001268D2430A401A601437BD465DF8047BC0
:103B9000704700BF003C014080B483B000AF786044
:103BA0007B6800221A607B6800221A717B680C22F5
:103BB0005A717B6800229A710C37BD465DF8047B10
:103BC0007047000080B485B000AF78600023FB73BD
:103BD000084B5A697B681340002B02D00123FB730A
:103BE00001E00023FB73FB7B18461437BD465DF8EC
:103BF000047B7047003C014080B483B000AF786024
:103C0000034A7B6853610C37BD465DF8047B7047FF
:103C1000003C014080B483B000AF7860044B7A6808
:103C2000D2B21A700C37BD465DF8047B704700BFF6
:103C3000003C024080B400AF064B1B69002B05DA44
:103C4000044B054A5A60034B044A5A60BD465DF86E
:103C5000047B7047003C024023016745AB89EFCDF0
:103C600080B400AF044A044B1B6943F00043136166
:103C7000BD465DF8047B7047003C024080B584B0CF
:103C800000AF78600B46FB700023FB600923FB72DA
:103C9000FB78002B02D10023FB6010E0FB78012BA6
:103CA00003D14FF48073FB6009E0FB78022B03D152
:103CB0004FF40073FB6002E04FF44073FB6000F0D0
:103CC000BDF80346FB72FB7A092B2FD11A4A1A4B17
:103CD0001B6923F4407313611749174B1A69FB687A
:103CE00013430B61144A144B1B6923F0F80313614F
:103CF0001149114B1A697B68134343F002030B61AE
:103D00000D4A0D4B1B6943F48033136100F096F8A4
:103D10000346FB72084A084B1B6923F00203136138
:103D2000054A054B1B6923F0F8031361FB7A18461B
:103D30001037BD4680BD00BF003C024080B584B056
:103D400000AF786039600923FB7300F077F8034611
:103D5000FB73FB7B092B1ED1114A114B1B6923F40A
:103D6000407313610E4A0E4B1B6943F400731361D9
:103D70000B4A0B4B1B6943F0010313617B683A68E4
:103D80001A6000F05BF80346FB73054A044B1B699D
:103D900023F001031361FB7B18461037BD4680BD3D
:103DA000003C024080B483B000AF7860034A7B6877
:103DB000D3600C37BD465DF8047B7047003C024081
:103DC00080B483B000AF0923FB711B4BDB6803F4A5
:103DD0008033B3F5803F02D10123FB7125E0164B00
:103DE000DB6803F01003002B02D00623FB711CE0FC
:103DF000114BDB6803F48073002B02D00223FB71AC
:103E000013E00D4BDB6803F0EF03002B02D0072318
:103E1000FB710AE0084BDB6803F00203002B02D0C1
:103E20000823FB7101E00923FB71FB7918460C376D
:103E3000BD465DF8047B7047003C024080B582B00F
:103E400000AF0923FB71FFF7BBFF0346FB7103E0E3
:103E5000FFF7B6FF0346FB71FB79DBB2012BF7D00E
:103E6000FB79DBB218460837BD4680BD80B487B009
:103E700000AF7860396000237B6100233B61002341
:103E8000FB6000237B6176E001227B6902FA03F389
:103E90003B613B681A683B691340FB60FA683B6909
:103EA0009A4265D17B681A687B695B00032101FA3D
:103EB00003F3DB431A407B681A607B681A683B682F
:103EC0001B7919467B695B0001FA03F31A437B688F
:103ED0001A603B681B79012B03D03B681B79022BCE
:103EE0002ED17B689A687B695B00032101FA03F39A
:103EF000DB431A407B689A607B689A683B685B7911
:103F000019467B695B0001FA03F31A437B689A60E8
:103F10007B685A687B699BB2194601238B40DB435F
:103F20001A407B685A607B685B683A6892791146F0
:103F30007A6992B201FA02F292B21A437B685A602D
:103F40007B68DA687B699BB25B00032101FA03F3AB
:103F5000DB431A407B68DA607B68DA683B68DB79B0
:103F600019467B695B0001FA03F31A437B68DA6048
:103F70007B6901337B617B690F2B85D91C37BD467B
:103F80005DF8047B704780B485B000AF78600B4665
:103F90007B800023FB737B681A697B881340002BAE
:103FA00002D00123FB7301E00023FB73FB7B184667
:103FB0001437BD465DF8047B704780B483B000AF12
:103FC00078600B467B807A887B689A610C37BD46A7
:103FD0005DF8047B704780B483B000AF78600B4617
:103FE0007B807B881B041A467B689A610C37BD4630
:103FF0005DF8047B704780B485B000AF78600B46F5
:104000007B8013467B700023FB600023BB607A78C3
:104010007B8803F007039B0002FA03F3FB607B88B5
:10402000DB089BB218467B88DB089BB21A467B688C
:10403000083253F822207B8803F007039B000F21EE
:1040400001FA03F3DB4302EA03017B6800F1080293
:1040500043F822107B88DB089BB21A467B68083243
:1040600053F82220FB681343BB607B88DB089BB2BC
:104070001A467B680832B96843F822101437BD46E7
:104080005DF8047B7047000080B58AB000AF7860AF
:1040900039600023FB8400237B840423BB84564BBC
:1040A000FB617B685B68FB84FB8C23F03F03FB8434
:1040B00007F10C031846FEF7FFF97B69FB61FB690A
:1040C0004E4AA2FB03239B0C7B84FA8C7B8C13430C
:1040D000FB84FA8C7B685A607B681A684FF6FE7323
:1040E00013407A6813600023FB843B681B68444AD2
:1040F000934215D83B681B685B00FA69B2FBF3F387
:10410000BB84BB8C032B01D80423BB84FA8CBB8CEF
:104110001343FB847B8C01331A467B681A6241E0AF
:104120003B68DB884BF6FF72934209D13B681A6803
:1041300013465B001344FA69B2FBF3F3BB840EE051
:104140003B681A6813469B0013449A001344FA69AB
:10415000B2FBF3F3BB84BB8C43F48043BB84BB8CC6
:10416000C3F30B03002B03D1BB8C43F00103BB84CF
:10417000BA8CFB8C13439BB26FEA43436FEA534301
:10418000FB847B8C4FF4967202FB03F31D4A82FB87
:1041900003129211DB17D31A9BB201339BB21A465A
:1041A0007B681A62FA8C7B68DA617B681B6843F073
:1041B00001027B681A607B681B68FB84FB8C23F41C
:1041C000816323F00203FB843B689A883B685B8928
:1041D00013439AB2FB8C1343FB84FA8C7B681A60FE
:1041E0003B689A893B681B8913439BB21A467B68DC
:1041F0009A602837BD4680BD00127A0083DE1B43DB
:10420000A0860100D34D621080B586B000AF294B67
:104210005B6800222849184634F0C4FB78617B694A
:10422000002B44D03B1D7969184630F083FE30E006
:104230003B1D184605F0FFF8386100221F49386918
:1042400034F0B0FB0346184635F044FF0346FB73D9
:10425000FB7B002B15D000220021386905F01CF9EA
:10426000B860B8681EF0D4FA034683F00103DBB2ED
:10427000002B03D0124901202EF0E0F8B86836F088
:10428000C9FE386936F0C6FE3B1D7969184630F024
:10429000D4FE3B1D184605F0E2F80346002BC7D1BB
:1042A0003B1D184605F0ECF8786936F0B3FE183778
:1042B000BD4680BD58510120387D0408887E040821
:1042C000407D040880B588B000AF786039607B68B5
:1042D000002B05DC454901202EF0B0F8002381E0D9
:1042E0000023FB770023BB77386839F063F8034677
:1042F000002B29D000223E49386834F053FB034696
:10430000184635F0E7FE0346FB7700223949386846
:1043100034F048FB0346184635F0C2FE78617B69ED
:10432000002B0BD07B69082B08D07B69102B05D0A4
:10433000314901202EF082F8002353E07B69102BD5
:1043400011D10123BB770FE0386839F0D6F8034666
:1043500083F00103DBB2002B06D03A682749012025
:104360002EF06CF800E000BFBB7F002B01D00223D1
:1043700000E001237B827B8A7968184630F0E2F8FE
:10438000F8600023BB61FB7F002B05D07B8A796836
:10439000184630F0D7F8B8611949002028F0B6FE69
:1043A000B860BB68002B08D0FB68002B05D0FB7FF2
:1043B000002B09D0BB69002B06D1BA69F968B8682F
:1043C00036F062FE00230DE0FA680E49B86834F05A
:1043D000D9FBBB69002B04D0BA690B49B86834F02B
:1043E000D1FBBB6818462037BD4680BD607D040800
:1043F000807D040814A80408907D0408A87D0408A2
:10440000E07D0408EC7D0408F47D04080000000051
:10441000F0B595B004AF7861C7E902230B46FB7491
:104420000022A149786934F0BDFA0346184635F0F8
:1044300051FE034687F8353097F83530002B04D00D
:104440009A4901202DF0FAFF25E1FB7C184629F05E
:1044500035F9034683F00103DBB2002B04D0944905
:1044600001202DF0EBFF16E1BB683B60FB6823F0F9
:1044700000437B604FF0FF328E4BD7E90001FCF721
:10448000E1FA0346002B13D14FF0FF32894BD7E9F5
:104490000001FCF7CDFA0346002B09D180A3D3E934
:1044A0000023D7E90201FCF7A5FA0346002B04D04C
:1044B000814901202DF0C2FFEDE015F06DFEC7E946
:1044C0000E01002387F83730B86D38F073FF0346CC
:1044D000002B53D000227949B86D34F063FA0346BB
:1044E000184635F0E9FDC7E90A01BC6AFB6A23F00A
:1044F000004501231E464FF0FF326E4B20462946F1
:10450000FCF7A0FA0346002B0BD14FF0FF32694BAA
:1045100020462946FCF78CFA0346002B01D10023E4
:104520001E46F3B283F00103DBB2002B19D04FF02B
:1045300000024FF00003D7E90A01FCF779FA0346BD
:10454000002B0ED04FF000025D4BD7E90A01FBF7BC
:10455000DFFF03460C461846214615F0C9FDC7E9A2
:104560000E0100225749B86D34F01CFA0346184674
:1045700035F0B0FD034687F837300DE0B86D38F000
:10458000BCFF034683F00103DBB2002B04D0BA6DFD
:104590004D4901202DF052FF0023FB7607F11B034C
:1045A0001A460021786904F077FF78620022012121
:1045B000786904F071FF3862FB7E002B09D097F810
:1045C0005C30002B01D0052300E0062387F836304D
:1045D00008E097F85C30002B01D0032300E00423AF
:1045E00087F83630D7E902234FF000003449FCF752
:1045F000B9F803460C461846214615F079FD97F8A0
:104600003730002B06D03B6A002B01D03B6A02E01A
:104610007B6A00E0002397F83620039202937B6ABE
:104620000193FB7C009302460B46D7E90E011EF076
:1046300043F8034683F00103DBB2002B02D023488A
:104640002DF0DAFE396A786A36F010FD012036F076
:10465000CAFF03461A461449786934F093FAD7E939
:10466000020136F0D7FF03461A461949786934F03B
:1046700089FA184B5B6803221749184634F092F9FF
:10468000F861FB69002B06D07969F86934F06EFE99
:10469000F86936F0BFFC4437BD46F0BDAFF300808B
:1046A000FCA9F1D24D62503F887E0408FC7D0408CD
:1046B000187E0408FFFFEF7F247E0408447E040870
:1046C00000408F404C7E0408A87D0408547E0408F6
:1046D000707E040858510120387D040880B586B0EA
:1046E00002AFF860C7E900230B46FB72F97A012399
:1046F0000193BB690093D7E90023F868FFF788FEB0
:104700001037BD4680BD80B586B002AFF860C7E9FE
:1047100000230B46FB72FB7A184615F041FE4FF062
:1047200000024FF00003FCF765F90346002B09D1A6
:10473000F97A00230193BB690093D7E90023F86855
:10474000FFF766FE1037BD4680BD000080B584B01F
:1047500000AF786000221849786834F023F90346E6
:10476000184635F0B7FC0346FB73FB7B83F001036F
:10477000DBB2002B04D0114901202DF05FFE17E0C1
:1047800000220021786804F087FEB860B8681EF047
:104790003FF8034683F00103DBB2002B03D0084946
:1047A00001202DF04BFEB86836F034FC04F0B0FE6A
:1047B0001037BD4680BD00BF887E0408787E04089F
:1047C000407D040880B582B000AF78607B681B68CC
:1047D000002B01D1002305E07B681B68184636F0EA
:1047E00077F8034618460837BD4680BD80B483B0CD
:1047F00000AF78607B681B68002B14BF0123002387
:10480000DBB218460C37BD465DF8047B704780B5B7
:1048100082B000AF78607B681B68184636F0FAFB00
:104820000837BD4680BD90B484B000AFC7E9000131
:104830004FF000034FF00044C7E902343B46D3E990
:10484000001207F10803D3E90034A24206BF9942DF
:1048500001230023DBB218461037BD4690BC7047D9
:1048600090B583B000AFC7E90001D7E900013DF082
:1048700067FC03460C46184621460C37BD4690BDE2
:10488000B0B582B000AFC7E900014FF000024FF0B1
:104890000003D7E90001FCF7ADF80346002B04D074
:1048A0003C687B6883F0004501E0D7E9004523467A
:1048B0002C46184621460837BD46B0BD90B583B09A
:1048C00000AFC7E90001D7E900013DF081F90346D7
:1048D0000C46184621460C37BD4690BDB0B58CB08D
:1048E00000AFC7E90401C7E90223D7E90423C7E9F8
:1048F00008233B693B607B6923F000437B604FF0FA
:10490000FF325C4BD7E90001FCF79CF80346002B13
:1049100012D14FF0FF32574BD7E90001FCF788F86E
:104920000346002B08D1D7E90223D7E90201FCF79F
:1049300089F80346002B03D04FF000044E4D91E060
:104940004FF000024FF00003D7E90801FCF752F8DE
:104950000346002B05D03B693B617B6983F0004334
:104960007B614FF000024FF00003D7E90201FCF732
:1049700041F80346002B05D0BB68BB60FB6883F0A1
:104980000043FB604FF000024FF00003D7E9020143
:10499000FCF726F80346002B4CD14FF0FF32354B85
:1049A000D7E90201FCF730F80346002B42D04FF064
:1049B000FF32304BD7E90401FCF726F80346002B01
:1049C0002ED137E04FF000024FF08043D7E90401C9
:1049D000FBF7C8FE02460B46C7E90623D7E90223C8
:1049E000C7E90A2309E0D7E90A0102460B46FBF7AB
:1049F000DDFB02460B46C7E90A23D7E90A23D7E9BC
:104A00000601FCF70BF80346002BECD1D7E90A238B
:104A1000D7E90401FBF7C8FB02460B46C7E90423AC
:104A2000D7E90223D7E90401FBF7F8FF0346002B7F
:104A3000C8D105E04FF000024FF00003C7E904239E
:104A40004FF000024FF00003D7E90801FBF7D2FF57
:104A50000346002B04D03C697B6983F0004501E0EC
:104A6000D7E9044523462C46184621463037BD4633
:104A7000B0BD00BFFFFFEF7F0000F87F0000000027
:104A8000B0B584B000AFC7E900013C687B6823F093
:104A900000454FF0FF32364B20462946FBF7D2FF48
:104AA0000346002B10D14FF0FF32314B20462946F0
:104AB000FBF7BEFF0346002B06D1D7E90001FFF745
:104AC000B2FE0346002B05D0D7E9000136F0A2FD67
:104AD00003463FE04FF000024FF00003D7E900012A
:104AE000FBF788FF0346002B03D01DA4D4E9003454
:104AF00002E01DA4D4E900341A462346D7E9000198
:104B0000FBF754FB03460C46C7E90034D7E9000124
:104B1000FCF75EF803460C46C7E90234D7E90234D5
:104B2000234312D14FF000024FF00003D7E90001F8
:104B3000FBF760FF0346002B07D04FF000004FF05B
:104B4000004136F067FD034604E0D7E9020136F084
:104B500079FD034618461037BD46B0BDAFF300805F
:104B60002083E4FFFFFFDFBF2083E4FFFFFFDF3F81
:104B7000FFFFEF7F90B583B000AFC7E900014FF0B2
:104B800000024FF00003D7E90001FBF747FF03469F
:104B9000002B11D0D7E900013DF092FB4FF000024D
:104BA000094BFBF7B5FC03460C46184621463DF081
:104BB0000FFB03460C4602E04FF00003034C18467F
:104BC00021460C37BD4690BD0000E03F0000F87F55
:104BD00090B585B000AFC7E90201C7E90023D7E966
:104BE0000023D7E90201FBF705FF0346002B03D0A2
:104BF000D7E90034C7E90234D7E90823D7E902012D
:104C0000FBF716FF0346002B03D0D7E90834C7E9AA
:104C10000234D7E90234184621461437BD4690BD08
:104C200090B589B000AF78600B46FB70FB78002B25
:104C300003D04FF000032D4C02E04FF000032C4C4A
:104C4000C7E9063407F10C037968184630F072F9A9
:104C500037E007F10C031846FFF7B4FD034618468A
:104C600035F02AFAC7E90401FB78002B08D0D7E910
:104C70000623D7E90401FBF7DBFE0346002B17D11F
:104C8000FB7883F00103DBB2002B08D0D7E90623C1
:104C9000D7E90401FBF7AEFE0346002B08D1D7E9A4
:104CA0000423D7E90401FBF7CDFE0346002B03D014
:104CB000D7E90434C7E9063407F10C03184630F08D
:104CC0008CF907F10C031846FFF790FD0346002B03
:104CD000BFD107F10C031846FFF799FDD7E9063459
:104CE000184621462437BD4690BD00BF0000F0FFA6
:104CF0000000F07F80B483B000AF78607B68002252
:104D00005A7100229A717B684FF0FF321A734FF08C
:104D1000FF325A734FF0FF329A734FF0FF32DA735B
:104D20007B6800221A7400225A7400229A740022AE
:104D3000DA747B684FF0FF321A754FF0FF325A7504
:104D40007A68937D43F0030393757A68937D43F00B
:104D50000C0393757A68937D6FF3051393757B68E5
:104D60000022DA7500221A767B6800225A76002229
:104D70009A767B680022DA77002262F07F0283F85D
:104D800020207B68002283F82120002262F07F022D
:104D900083F822207B684FF0FF32DA76002242F05F
:104DA0007F021A777B684FF0FF325A77002242F079
:104DB0007F029A770C37BD465DF8047B704780B45C
:104DC00083B000AF78607B681B69002B01D10023A2
:104DD00005E07B681A697B681B6813441B781846DA
:104DE0000C37BD465DF8047B704780B483B000AFDC
:104DF00078607B681A687B685B689A4234BF0123DD
:104E00000023DBB218460C37BD465DF8047B7047C3
:104E100080B483B000AF78607B689A687B681B6859
:104E2000134418460C37BD465DF8047B704780B5C7
:104E300082B000AF78607B68DB68184636F0EAF82D
:104E40000837BD4680BD80B500AF19F012FF0023C2
:104E5000184680BD80B400AFBD465DF8047B704746
:104E600080B500AF044B5B6800220449184633F05C
:104E700099FD0346184680BD58510120907E0408D4
:104E800080B483B000AF78607B68012B11D07B6861
:104E9000022B0ED07B68042B0BD07B68082B08D02C
:104EA0007B68102B05D07B68182B02D07B68202BE9
:104EB00001D1012300E0002303F00103DBB2184617
:104EC0000C37BD465DF8047B7047000080B594B098
:104ED00000AFF860B9607A603B60FB68002B0ADDC8
:104EE000BB68002B07DDFB68B3F5004F03DABB6836
:104EF000B3F5004F05DB8A4901202DF09FFA00230E
:104F00000AE17868FFF7BCFF034683F00103DBB2D8
:104F1000002B05D0834901202DF090FA0023FBE0FF
:104F20008149002028F0F2F8F864FB6C002B01D1D5
:104F30000023F1E007F110031846FFF7DBFE002322
:104F40003B7500237B750023BB75FB6C3B61FB68E5
:104F50009BB2A7F81730BB689BB2A7F819307B68E3
:104F6000DBB2FB76386838F025FA0346002B00F0F8
:104F7000C88000226D49386833F014FD0346184696
:104F800035F0A8F80346002B07D0B7F815309BB2D0
:104F900043F001039BB2A7F815300022644938683A
:104FA00033F000FD0346184635F094F80346002B15
:104FB00007D0B7F815309BB243F004039BB2A7F8B3
:104FC000153000225B49386833F0ECFC0346184684
:104FD00035F080F80346002B1ED0FB7E012B0FD14D
:104FE000B7F815309BB243F002039BB2A7F8153017
:104FF000B7F819309BB203F00703002B06D10BE082
:105000004D4901202DF01AFA002385E04B4901207B
:105010002DF014FA00237FE000224949386833F06C
:10502000C1FCB864BB6C002B6BD04649B86C35F042
:105030006DFD0346002B61D14349B86C35F066FD28
:10504000034683F00103DBB2002B08D0B7F815301C
:105050009BB243F040039BB2A7F815304EE03B49AA
:10506000B86C35F053FD034683F00103DBB2002B2F
:1050700008D0B7F815309BB243F080039BB2A7F875
:1050800015303BE03249B86C35F040FD034683F003
:105090000103DBB2002B08D0B7F815309BB243F008
:1050A000C0039BB2A7F8153028E02A49B86C35F048
:1050B0002DFD034683F00103DBB2002B08D0B7F8C7
:1050C00015309BB243F480739BB2A7F8153015E0FE
:1050D0002149B86C35F01AFD034683F00103DBB2B9
:1050E000002B08D0B7F815309BB243F4A0739BB2E5
:1050F000A7F8153002E019482DF07EF9B86C35F0AC
:1051000089FF07F1100318461AF08EF907F1100312
:10511000184618F0A5FCFB6C18465037BD4680BDFC
:10512000947E0408A47E0408B07E0408BC7E0408B3
:10513000C47E0408C87E0408D87E0408087F0408DA
:10514000447F0408507F0408547F0408587F0408F3
:105150005C7F0408607F0408647F0408687F04089B
:1051600080B596B000AFF860B9607A603B60FB68CC
:10517000002B0ADDBB68002B07DDFB68B3F5004F91
:1051800003DABB68B3F5004F05DB4B4901202DF076
:1051900055F900238CE07868FFF772FE034683F030
:1051A0000103DBB2002B05D0444901202DF046F964
:1051B00000237DE000237B6500233B65386838F0E1
:1051C000F9F80346002B0FD0786D35F023FF00224D
:1051D0003B49386833F0E6FB786500223949386886
:1051E00033F0E0FB386503E0386839F037F978656B
:1051F000786D38F086F8034683F00103DBB2002BAC
:105200000AD07A6D304901202DF018F9396D786D8A
:1052100035F02CFF00234BE0386D38F06EF9034673
:1052200083F00103DBB2002B13D0386D38F069F83E
:10523000034683F00103DBB2002B0AD03A6D22490A
:1052400001202DF0FBF8396D786D35F00FFF00234C
:105250002EE01E49002027F059FFF864FB6C002B5C
:1052600001D1002324E007F114031846FFF742FDA3
:1052700001233B76FB6C7B61FB689BB2A7F81B307C
:10528000BB689BB2A7F81D307B68DBB2FB7707F1E8
:1052900014033A6D796D184615F0CEFE07F114032C
:1052A000184618F0DDFB396D786D35F0DFFEFB6CCC
:1052B00018465837BD4680BD947E0408A47E040875
:1052C0008C7F0408987F0408A47F0408B07E04083B
:1052D00080B592B000AF7860786837F05AFF034627
:1052E00083F00103DBB2002B05D06C4903202DF0C5
:1052F000A5F80023CDE000237B6400233B6400235A
:10530000FB630023BB6300237B6307F108030022D8
:10531000796818462FF0E0FB2EE007F108031846E5
:10532000FFF74DFD034687F8333097F833300A2BEB
:105330000DD17B6C002B04D13B6C002B01D10123E0
:105340007B6300237B643B6C01333B640FE03A6C6E
:10535000BB6B9A4202DB3B6C0133BB637B6C01335A
:105360007B647A6CFB6B9A4201DD7B6CFB6307F11B
:10537000080318462FF0C2FC07F108031846FFF790
:1053800034FD0346002BC8D107F108031846FFF788
:105390004EFD36F09FF9F862FB6A002B01D1002325
:1053A00077E0F86B36F00AF903461A463C49F86A8A
:1053B00033F0E8FBB86B36F001F903461A46394979
:1053C000F86A33F0DFFBFB6BBA6B02FB03F30733C6
:1053D000DB10BB62BB6A0021184636F07DF87862AC
:1053E0007B6A002B04D1F86A35F014FE002350E0EC
:1053F00000237B6400233B6407F108037A6B796820
:1054000018462FF069FB31E007F108031846FFF753
:10541000D6FC034687F8233097F823300A2B05D1B2
:1054200000237B643B6C01333B641AE097F8233024
:10543000202B13D03B6CFA6B02FB03F27B6C134402
:10544000FB61FB69D908FB6903F00703802242FA7C
:1054500003F3DAB20123786A34F0B4F97B6C0133D8
:105460007B6407F1080318462FF048FC07F1080396
:105470001846FFF7BAFC0346002BC5D107F1080315
:105480001846FFF7D4FC7A6A0749F86A33F07AFBCA
:10549000FB6A18464837BD4680BD00BFD87F040868
:1054A000EC7F040888800408EC7D040880B590B087
:1054B00000AF78600B46FB7007F108037968184667
:1054C00018F06CFA034683F00103DBB2002B01D025
:1054D00000231EE0B7F80D309BB203F00803002B49
:1054E0000DD0FB78002B14BF01230023DBB283F027
:1054F0000103DBB2FB70FB7803F00103FB70FB7868
:10550000002B03D0B7F811309BB202E0B7F80F3090
:105510009BB218464037BD4680BD80B590B000AF05
:10552000786007F108037968184618F037FA0346DF
:1055300083F00103DBB2002B0AD107F10803184600
:1055400018F0CCFC07F10803184618F089FA00E0BF
:1055500000BF4037BD4680BD90B595B002AFF86042
:10556000B9607A603B6007F11003F968184618F0DB
:1055700015FA034683F00103DBB2002B13D1BB689D
:1055800019B27B681AB23B681CB2BB6D1BB207F143
:1055900010000093234618F072FC07F11003184620
:1055A00018F05EFA00E000BF4C37BD4690BD90B5E4
:1055B00095B002AFF860B9607A603B6007F1100304
:1055C000F968184618F0EAF9034683F00103DBB2E4
:1055D000002B13D1BB6819B27B681AB23B681CB2AE
:1055E000BB6D1BB207F110000093234618F09DFC21
:1055F00007F11003184618F033FA00E000BF4C37EB
:10560000BD4690BD80B592B000AFF860B9607A60D9
:105610003B6007F11003F968184618F0BFF903461C
:1056200083F00103DBB2002B0FD1BB6819B27B689A
:105630001AB23B681BB207F1100018F08CFD07F19D
:105640001003184618F00CFA00E000BF4837BD46BA
:1056500080BD80B592B000AFF860B9607A603B6001
:1056600007F11003F968184618F098F9034683F01B
:105670000103DBB2002B0FD1BB6819B27B681AB2F1
:105680003B681BB207F1100018F0AEFC07F11003E5
:10569000184618F0E5F900E000BF4837BD4680BD68
:1056A00080B592B000AFF860B9607A6007F110037E
:1056B000F968184618F072F9034683F00103DBB26B
:1056C000002B01D0002309E0BB6819B27B681AB235
:1056D00007F11003184618F0B7FB03461846483781
:1056E000BD4680BD80B594B000AFF860B9607A6007
:1056F0003B6007F11403F968184618F04FF90346A8
:1057000083F00103DBB2002B26D13B6AFB643868CF
:1057100037F0F3FE034683F00103DBB2002B04D025
:10572000386834F011FA0346FB64BB6819B27B6831
:105730001AB207F11400FB6C18F068FBBB681BB2CF
:10574000A7F82B307B681BB2A7F82D3007F11403A4
:10575000184618F085F900E000BF5037BD4680BDFF
:1057600090B5A1B000AFF860B9607A603B6007F116
:105770001003F968184618F011F9034683F0010385
:10578000DBB2002B40F0F7800023FB67B86834F0F1
:1057900051FBC7E91A01786834F04CFBC7E91801DE
:1057A000386834F047FBC7E91601786837F0A5FE82
:1057B000034683F00103DBB2002B00F0C880386899
:1057C00037F09BFE034683F00103DBB2002B00F0B1
:1057D000BE804FF000026A4BD7E91A01FAF798FE33
:1057E00003460C4618462146FBF742F90346BB67C1
:1057F0004FF00002624BD7E91801FAF789FE034621
:105800000C4618462146FBF733F903467B674FF0F9
:1058100000025B4BD7E91601FAF77AFE03460C4605
:1058200018462146FBF724F903463B67BB6FFF2B65
:1058300001DDFF23BB677B6FFF2B01DDFF237B6750
:105840003B6FFF2B01DDFF233B67BB6F002B01DAB2
:105850000023BB677B6F002B01DA00237B673B6F64
:10586000002B01DA00233B67B7F815309BB203F435
:10587000E0737B657B6D002B32D0BB6F3B657B6F2C
:10588000FB643B6FBB647B6DC02B19D0C02B04DC69
:10589000402B09D0802B0ED022E0B3F5807F16D0AC
:1058A000B3F5A07F18D01BE0BB6CBB673B6D7B677B
:1058B000FB6C3B6714E0BB6CBB673B6D3B670FE069
:1058C000FB6CBB67BB6C7B673B6D3B6708E0FB6CAD
:1058D000BB673B6D7B6703E0BB6C7B67FB6C3B6727
:1058E000FB7E102B0BD13B6FDA107B6F9B105B01A3
:1058F0001A43BB6FDB10DB021343FB672CE0FB7E1C
:10590000202B0AD17B6F1A023B6F1A43BB6F1B041B
:10591000134343F07F43FB671EE0FB7E182B08D147
:105920007B6F1A023B6F1A43BB6F1B041343FB6769
:1059300012E0BA6F7B6F1A443B6F1344B3F5C07F1C
:1059400002DB4FF0FF3300E00023FB6704E0B868A0
:1059500034F0FAF80346FB6797F89030002B02D03A
:10596000FB6FFB6101E0FB6F3B6207F11003184620
:1059700018F076F800E000BF8437BD4690BD00BF48
:105980000000704080B590B000AF78600B46FB70AF
:1059900007F108037968184618F000F8034683F009
:1059A0000103DBB2002B01D000230BE0FB78002BBE
:1059B00001D07B6900E0BB69FA7C114601228A4074
:1059C000013A134018464037BD4680BD80B592B0BD
:1059D00000AFF860B9601346FB7107F11003F96876
:1059E000184617F0DBFF034683F00103DBB2002B00
:1059F0002CD1FB79002B0BD0BB68002B01DC0123E1
:105A0000BB60BB68B3F5806F02DB40F2FF33BB6065
:105A1000B7F9243013F1020F0FD10E49F86833F0B3
:105A2000C3F80D49F86833F0BFF80C49F86833F053
:105A3000BBF80B49F86833F0B7F8BB681BB2BB84FE
:105A400007F11003184618F00BF800E000BF4837C4
:105A5000BD4680BDF47F0408FC7F04080480040870
:105A60000C80040880B592B000AFF860B9607A602D
:105A70003B6007F11003F968184617F08FFF0346E3
:105A800083F00103DBB2002B5ED1B86837F081FBF5
:105A9000034683F00103DBB2002B04D02C49012024
:105AA0002CF0CCFC50E07B68002B02DB7B68FF2BEA
:105AB00004DD284901202CF0C1FC45E0386837F0AE
:105AC00068FB034683F00103DBB2002B0DD038687E
:105AD00037F0EEFA034683F00103DBB2002B04D06B
:105AE0001D4901202CF0AAFC2EE03B6D002B02DDAD
:105AF0003B6DFF2B04DD194901202CF09FFC23E0B6
:105B0000BA681749F86832F0C5FF3A681549F8686D
:105B100032F0C0FF386D35F051FD03461A46124988
:105B2000F86833F02FF8786835F048FD03461A46D8
:105B30000E49F86833F026F84FF6FE73BB8407F180
:105B40001003184617F08CFF4837BD4680BD00BFD4
:105B500014800408348004085480040880800408F9
:105B6000F47F0408FC7F0408048004080C80040807
:105B700080B592B000AFF860B9607A603B6007F121
:105B80001003F968184617F009FF034683F0010374
:105B9000DBB2002B48D1BB68B3F1FF3F02DA4FF014
:105BA000FF33BB60BB68012B01DD0123BB607B6859
:105BB000B3F1FF3F02DA4FF0FF337B607B68012BCC
:105BC00001DD01237B603B68002B01DA00233B6091
:105BD0003B68032B01DD03233B60BB68DBB203F0B2
:105BE0000303DAB297F8263062F3010387F8263010
:105BF0007B68DBB203F00303DAB297F8263062F376
:105C0000830387F826303B68DBB203F00303DAB284
:105C100097F8263062F3051387F8263007F1100352
:105C2000184617F01DFF00E000BF4837BD4680BD95
:105C300090B5B5B002AFF860B9607A603B6007F12B
:105C40004C03F968184617F0A9FE034683F00103D8
:105C5000DBB2002B40F0B2820023C7F8C43000232F
:105C6000C7F8C0300023C7F8BC300023C7F8B830ED
:105C7000B7F96030002B04DDB7F96030C7F8BC30ED
:105C800031E0B7F96030B3F1FF3F03D10623C7F825
:105C9000BC3028E0B7F9603013F1020F23D10022A5
:105CA000C149F86832F07EFEC7F8C4000022BF493F
:105CB000F86832F077FEC7F8C0000022BC49F868E7
:105CC00032F070FE0346184634F0EAF9C7F8BC001B
:105CD0000022B849F86832F065FE0346184634F0F1
:105CE000DFF9C7F8B8003B6DC3F30F23A7F8A63060
:105CF00097F8623003F03003DBB2102B16D1B7F8FF
:105D000051309BB283F018039BB2A7F85130B7F81B
:105D100053309BB21A467B680133D31AC7F8A030C0
:105D20003B687B60D7F8A0303B603CE097F862307E
:105D300003F03003DBB2202B18D1B7F851309BB2FF
:105D400083F030039BB2A7F85130B7F853309BB2C1
:105D50001A467B680133D31A7B60B7F855309BB283
:105D60001A463B680133D31A3B601CE097F8623057
:105D700003F03003DBB2302B15D1B7F851309BB2B2
:105D800083F028039BB2A7F85130B7F855309BB287
:105D90001A463B680133D31AC7F89C307B683B60D6
:105DA000D7F89C307B6097F86230C3F30103DBB215
:105DB000012B13DCB968F86800F004FA024697F882
:105DC0006230C3F30103DBB2013303FB02F3DA0FEA
:105DD00013445B101A467B689B1A7B6097F862300D
:105DE000C3F38103DBB2012B11DC97F86230C3F3FC
:105DF0000103DBB20133D7F8BC2002FB03F3DA0F57
:105E000013445B105B421A463B6813443B60B7F88F
:105E100051309BB203F00803002B03D0B7F8553084
:105E20009BB202E0B7F853309BB2C7F89830B7F88E
:105E300051309BB203F00803002B03D0B7F8533066
:105E40009BB202E0B7F855309BB2C7F894307B683C
:105E5000C7F89030B86836F04FFAC7F88C0007F1F1
:105E600038030022D7F88C1018462EF035FE85E155
:105E700007F138031846FEF7A2FF034687F88B3078
:105E800097F88B300A2B0DD1D7F890307B603A68A9
:105E9000D7F8BC3013443B6007F1380318462EF0A6
:105EA0002DFF6BE1B7F96030002B35DDB7F96010DD
:105EB00097F88B2007F14C03184618F0F3FD0346C2
:105EC000C7F88430D7F884305A427B689A421DDA8A
:105ED0007A68D7F898309A4218DAB7F960305A429F
:105EE0003B689A4212DA3A68D7F894309A420DDA4F
:105EF0007B6819B23B681AB2B7F9604007F14C00F1
:105F000097F88B300093234618F0FEFC7A68D7F898
:105F1000843013447B6027E1B7F96030B3F1FF3F71
:105F20001FD17B6813F1030F17DB7A68D7F898301D
:105F30009A4212DA3B6813F1050F0EDB3A68D7F884
:105F400094309A4209DA7B6819B23B681AB297F822
:105F50008B3007F14C0017F081FB7B6804337B60CA
:105F600002E1B7F9603013F1020F40F0FD80002329
:105F7000C7F8B4300023C7F8B030D7F8C00037F006
:105F800008F90346002B4CD097F88B20D7F8B8308F
:105F90009A4257DB07F110030022D7F8C0101846C9
:105FA0002EF09AFD19E000BFF47F0408FC7F04087E
:105FB000048004080C80040807F110031846FEF75B
:105FC000FEFE03461A46D7F8B0301344C7F8B03087
:105FD00007F1100318462EF091FE07F11003184642
:105FE000FEF703FF0346002B0DD007F11003184600
:105FF000FEF70EFF0346194697F88B20D7F8B83006
:10600000D31A9942D8DB07F110031846FEF7D7FEE2
:106010000346C7F8B43007F110031846FEF707FF30
:1060200010E0D7F8C00033F08FFDC7F8B40097F840
:106030008B20D7F8B830D31AD7F8B42002FB03F37B
:10604000C7F8B03097F88B20D7F8B8309A42C0F232
:106050008680D7F8B4305A427B689A427FDA7A68F1
:10606000D7F898309A427ADAD7F8BC305A423B686F
:106070009A4274DA3A68D7F894309A426FDAD7F8CD
:10608000B030D7F8BC2002FB03F3C7F8B030D7F824
:10609000B030DA0807F12403D7F8C41018462EF000
:1060A0001BFDD7F8B03003F00703C7F8B03000236A
:1060B000C7F8AC3048E00023C7F8A83039E007F152
:1060C00024031846FEF77BFE03461A46D7F8B03085
:1060D00002FA03F303F08003002B14D0D7F8AC309E
:1060E0009AB27B689BB213449BB219B2D7F8A8301E
:1060F0009AB23B689BB213449BB21AB2BB6D07F1D4
:106100004C0017F083FED7F8B0300133C7F8B03039
:10611000D7F8B030082B07D10023C7F8B03007F10B
:10612000240318462EF0EAFDD7F8A8300133C7F84B
:10613000A830D7F8A820D7F8BC309A42BFDBD7F8F0
:10614000AC300133C7F8AC30D7F8AC20D7F8B43056
:106150009A42B0DB07F124031846FEF768FE7A681E
:10616000D7F8B43013447B602DF08EFC0346002B2F
:106170000DD107F1380318462EF0C0FD07F13803A2
:106180001846FEF732FE0346002B7FF471AE07F18E
:1061900038031846FEF74BFED7F8C020D7F8C410D6
:1061A000D7F88C0034F070FFB7F8A630A7F851305C
:1061B00007F14C03184617F053FC00E000BFCC3742
:1061C000BD4690BD80B59CB000AF7860396007F1E6
:1061D00020037968184617F0E1FB034683F00103BA
:1061E000DBB2002B01D000239AE00023FB660023E2
:1061F000BB66B7F9343013F1020F0FD100224A49C0
:10620000786832F0CFFBF86600224849786832F0AF
:10621000C9FB0346184633F043FFB866386836F0CA
:106220006BF8F86507F10C030022F96D18462EF0A3
:1062300053FC00237B6600233B665BE007F10C0305
:106240001846FEF7BCFD034687F85B3097F85B30D5
:106250000A2B07D17A6E3B6E9A4201DD7B6E3B665C
:1062600000237B66B7F93430002B0EDDB7F934100C
:1062700097F85B2007F12003184618F013FC03463B
:106280001A467B6E13447B662FE0B7F93430B3F1C6
:10629000FF3F03D17B6E04337B6626E0B7F93430D1
:1062A00013F1020F21D1F86E36F073FF0346002B75
:1062B00012D097F85B20BB6E9A4215DB97F85B20F3
:1062C000BB6ED31A1946F86E33F054FA03461A46D9
:1062D0007B6E13447B6608E0F86E33F035FC0246B3
:1062E0007B6E13447B6600E000BF07F10C03184689
:1062F0002EF004FD07F10C031846FEF776FD034669
:10630000002B9BD107F10C031846FEF790FDF96EA8
:10631000F86D34F0ABFE3A6E7B6E9342B8BF134615
:1063200018467037BD4680BDFC7F04080C80040809
:1063300090B595B002AFF860B9607A603B6007F144
:106340001003F968184617F029FB034683F0010390
:10635000DBB2002B13D1BB6819B27B681AB23B6861
:106360001CB2BB6D1BB207F110000093234617F05F
:106370009CFF07F11003184617F072FB00E000BF06
:106380004C37BD4690BD90B595B002AFF860B9608E
:106390007A6007F11003F968184617F0FFFA034610
:1063A00083F00103DBB2002B1DD1B7F9273019B2FE
:1063B000B7F929301AB2BB681CB27B681BB207F16F
:1063C00010000093234617F070FFBB681BB2A7F8BC
:1063D00027307B681BB2A7F8293007F11003184655
:1063E00017F03EFB00E000BF4C37BD4690BD80B5C6
:1063F00092B000AFF860B9607A6007F11003F968F5
:10640000184617F0CBFA034683F00103DBB2002BEA
:106410000DD1BB681BB2A7F827307B681BB2A7F869
:10642000293007F11003184617F01AFB00E000BFEF
:106430004837BD4680BD90B5A7B002AFF860B960DF
:106440001346FB7107F14003F968184617F0A6FAE6
:10645000034683F00103DBB2002B7CD1B86837F030
:10646000B4F9034683F00103DBB2002B73D10023A0
:10647000C7F8803007F114030122B96818462FF0DD
:1064800037FA41E007F1140318462FF04BFBF86789
:10649000D7F8803003F00103002B28D0FB6FBB67D7
:1064A000D7F88030012B07D1D7F88C30C7F8883067
:1064B000BB6FC7F8843010E0B7F9573019B2B7F99D
:1064C00059301AB2D7F88C301CB2BB6F1BB207F12F
:1064D00040000093234617F0E8FED7F88C301BB23B
:1064E000A7F85730BB6F1BB2A7F8593002E0FB6F1B
:1064F000C7F88C30D7F880300133C7F8803007F107
:10650000140318462BF050FB07F1140318462BF028
:1065100005FB0346002BB5D107F1140318462BF0F9
:1065200095FBFB79002B11D0B7F9573019B2B7F9A9
:1065300059301AB2D7F888301CB2D7F884301BB261
:1065400007F140000093234617F0AFFE07F1400328
:10655000184617F085FA9437BD4690BD2DE9F043F3
:10656000A1B000AF786039606B461E4607F1380372
:106570007968184617F012FA034683F00103DBB27C
:10658000002B77D1386837F020F9034683F00103F8
:10659000DBB2002B6ED18023BB67BB6F013B7B67F7
:1065A000BB6F1A464FF000034FEA031949EA12790C
:1065B0004FEA0218BB6F1A464FF000031D0145EA6F
:1065C00012751401BB6F5B0001330733DB08DB007E
:1065D000ADEB030D6B4601335B085B003B670023AB
:1065E000FB6707F10C030122396818462FF080F988
:1065F00011E0FC6F631CFB6707F10C0318462FF0DA
:1066000091FA03461AB23B6F23F8142007F10C03EA
:1066100018462BF0C9FA07F10C0318462BF07EFA46
:106620000346002B03D0FA6FBB6F9A42E1DB07F100
:106630000C0318462BF00AFBFA6FBB6F9A4207D186
:10664000BB6FDA0F13445B1019460D482BF0D4FED4
:10665000FB6FDA0F13445B1019463A6F07F13803EA
:10666000184617F0B9FF07F13803184617F0F8F984
:10667000B54600E0B5468437BD46BDE8F08300BFAF
:106680009080040880B592B000AFF860B9601346FE
:10669000FB7107F11003F968184617F07FF90346FC
:1066A00083F00103DBB2002B51D1B7F815309BB258
:1066B00023F038039BB2A7F81530BB68032B25D80D
:1066C00001A252F823F000BF0D670008D966000848
:1066D000EB660008FD660008B7F815309BB243F082
:1066E00018039BB2A7F8153010E0B7F815309BB22D
:1066F00043F030039BB2A7F8153007E0B7F8153028
:106700009BB243F028039BB2A7F81530FB79002B0E
:1067100017D0B7F815309BB203F00803002B08D050
:10672000B7F815309BB283F020039BB2A7F8153061
:1067300007E0B7F815309BB283F010039BB2A7F8BF
:10674000153007F11003184617F08AF900E000BF72
:106750004837BD4680BD00BF90B5A7B000AFF86018
:10676000B9607A603B6007F12803F968184617F0B2
:1067700015F9034683F00103DBB2002B40F02581BD
:10678000B86836F017FE034683F00103DBB2002B36
:1067900004D08F4901202BF051FE16E100228D49D3
:1067A000B86832F0FFF80346184633F079FCF86712
:1067B00000228949B86832F0F5F80346184633F0EC
:1067C0006FFCB86700228549B86832F0EBF80346E1
:1067D000184633F065FCC7F89400D7F89430002BC6
:1067E00002DC0123C7F894300122D7F8943002FA72
:1067F00003F3013B7B6700227949B86832F0D2F895
:1068000038673B6F002B14BF0123002387F86F30DC
:10681000386F33F099F90346BB66386F34F0FAFBF2
:1068200000227049B86832F0BDF87866786E36F0AC
:10683000FCFD034683F00103DBB2002B08D0786E29
:1068400036F0A7FC034683F00103DBB2002B09D12D
:10685000FB6F002B06DDBB6F002B03DDD7F89430F8
:10686000202B07DD604901202BF0E8FD786E34F025
:10687000D1FBAAE0786E33F003FE3866786E34F010
:10688000C9FB0023C7F890300023C7F88C300023E1
:10689000C7F888300023C7F8843007F114030022BA
:1068A000396E18462EF018F96FE0D7F884301C02C4
:1068B00007F114031846FEF782FA03462343C7F88C
:1068C000843007F1140318462EF018FAD7F88830F0
:1068D0000833C7F88830D7F88820D7F894309A4220
:1068E000E3DBD7F88820D7F89430D31AD7F8842080
:1068F000DA407B6F1340C7F88030D7F88820D7F88C
:106900009430D31AC7F8883097F86F3083F00103BA
:10691000DBB2002B04D1BA6ED7F880309A4222D075
:10692000D7F89430012B08D1D7F88030002B01D054
:106930007B6B00E0BB6BC7F88030D7F890309AB221
:106940007B689BB213449BB219B2D7F88C309AB2D1
:106950003B689BB213449BB21AB207F12800D7F8E8
:10696000803017F053FAD7F890300133C7F89030E1
:10697000D7F89020FB6F9A4207DB0023C7F89030CE
:10698000D7F88C300133C7F88C30D7F88820D7F887
:1069900094309A4207DA07F114031846FEF725FAF5
:1069A0000346002B04D0D7F88C20BB6F9A4292DBB1
:1069B00007F114031846FEF73AFA386E34F02AFB52
:1069C00007F12803184617F04BF89C37BD4690BDD9
:1069D000C4800408EC7F040888800408F080040860
:1069E000F4800408EC7D04080081040890B5A1B08F
:1069F00000AF786007F120037968184616F0CEFFE3
:106A0000034683F00103DBB2002B01D00023A3E097
:106A100034F060FEF866FB6E002B01D100239BE092
:106A200000217868FEF742FDB86601217868FEF71C
:106A30003DFD786697F82B303B66B86E34F0BEFDAE
:106A400003461A464649F86E32F09CF8786E34F0E8
:106A5000B5FD03461A464349F86E32F093F83B6E93
:106A6000012B08D0386E34F0A9FD03461A463E4982
:106A7000F86E32F087F8BB6E7A6E02FB03F33A6E63
:106A800002FB03F30733DB10FB65FB6D00211846A7
:106A900034F022FDB865BB6D002B04D1F86E34F0E4
:106AA000B9FA002358E00023FB670023BB670023EB
:106AB0007B6700233B6707F10C030022B96D184682
:106AC0002EF00AF835E07A6F3B6E02FA03F4FB6FA2
:106AD00019B2BB6F1AB207F12003184617F0B4F9C8
:106AE000034623437B673B6E3A6F13443B67FB6F60
:106AF0000133FB67FA6FBB6E9A4217DB0023FB671B
:106B0000BB6F0133BB6711E03B6F083B7A6F22FA22
:106B100003F3DAB207F10C03114618462EF0D5F84C
:106B20007B6F1B0A7B673B6F083B3B673B6F072B09
:106B3000EAD807F10C031846FEF757F90346002B75
:106B4000C1D107F10C031846FEF771F9BA6D074978
:106B5000F86E32F017F8FB6E18468437BD4690BDCC
:106B6000EC7F040888800408F0800408EC7D0408A9
:106B700080B592B000AF78600B46FB7007F10C0354
:106B80007968184616F00AFF034683F00103DBB26A
:106B9000002B01D000236AE000237B64B7F9273083
:106BA0001AB2B7F92B301BB29A4235DC34F092FDA1
:106BB00078647B6C002B2FD0B7F927301BB21846B6
:106BC00034F0FCFC03461A462B49786C31F0DAFFAE
:106BD000B7F929301BB2184634F0F0FC03461A46C8
:106BE0002649786C31F0CEFFB7F92B301BB218462E
:106BF00034F0E4FC03461A462149786C31F0C2FFB8
:106C0000B7F92D301BB2184634F0D8FC03461A46AB
:106C10001C49786C31F0B6FFFB78002B26D000239E
:106C200087F82B30002363F07F0387F82C30002394
:106C300087F82D30002363F07F0387F82E304FF064
:106C4000FF3387F82730002343F07F0387F828308D
:106C50004FF0FF3387F82930002343F07F0387F894
:106C60002A3007F10C03184616F0FAFE7B6C184622
:106C70004837BD4680BD00BF2C8104083081040820
:106C8000348104083881040880B592B000AFF86000
:106C9000B9607A6007F11003F968184616F07EFEB5
:106CA000034683F00103DBB2002B0CD107F1100384
:106CB0007A68B968184617F029FF07F110031846DB
:106CC00016F0CEFE00E000BF4837BD4680BD000094
:106CD00090B59FB000AF786007F108037968184657
:106CE00016F05CFE034683F00103DBB2002B01D0FB
:106CF000002323E1FB7C012B08D0FB7C182B05D063
:106D0000904901202BF09AFB002317E1B7F80F30D0
:106D10009BB2FA7C02FB03F31F335B119B003B66C3
:106D2000FB7C012B0CBF0123002387F85F3097F811
:106D30005F30002B01D0202300E01A23BB65B7F899
:106D400011309BB21A463B6E03FB02F2BB6D13443B
:106D50007B657B6D184634F09DFA38653B6D002BE2
:106D600001D10023EAE0386D35F0F6FCF864FB6CE5
:106D700042221A70FB6C01334D221A70FB6C0233F5
:106D80007A6DD2B21A70FB6C03337A6D1212D2B2E2
:106D90001A70FB6C0A33BA6DD2B21A70FB6C0E33E8
:106DA0000C221A70FB6C1233B7F80F2092B2D2B2D9
:106DB0001A70FB6C1333B7F80F2092B2120A92B21A
:106DC000D2B21A70FB6C1433B7F8112092B2D2B25F
:106DD0001A70FB6C1533B7F8112092B2120A92B2F6
:106DE000D2B21A70FB6C163301221A70FB6C183386
:106DF000FA7C1A7097F85F30002B0BD0FB6C1A33BB
:106E0000FF221A70FB6C1B33FF221A70FB6C1C33C1
:106E1000FF221A7000237B6787E0B7F811309BB21E
:106E20001A467B6F0133D31ABB64FB7C012B36D12E
:106E300000233B672BE00023FB660023BB6614E0C6
:106E4000FB6E5C003B6F5A1C3A6719B27B6F1AB23B
:106E500007F10803184616F0F7FF034603F0010395
:106E60002343FB66BB6E0133BB66BB6E072BE7DDBE
:106E7000BB6C3A6E02FB03F2BB6D1A443B6FDB1036
:106E80001344013BFA6C1344FA6ED2B21A70B7F88D
:106E90000F309BB21A463B6F9A42CCDC42E0002393
:106EA0007B6638E07B6E19B27B6F1AB207F108037C
:106EB000184616F0C9FF7864BB6C3A6E02FB03F209
:106EC000BB6D1A44FB7CDB08DBB219467B6E03FB0F
:106ED00001F313443B643B6C5A1C3A641A46FB6C46
:106EE00013447A6CD2B21A703B6C5A1C3A641A463C
:106EF000FB6C13447A6C120AD2B21A703B6C5A1CA7
:106F00003A641A46FB6C13447A6C120CD2B21A70B3
:106F10007B6E01337B66B7F80F309BB21A467B6EEF
:106F20009A42BFDC7B6F01337B67B7F811309BB2AD
:106F30001A467B6F9A423FF770AF3B6D18467C371D
:106F4000BD4690BD3C81040880B586B000AF786036
:106F50007868FFF7BDFE78617B69002B01D10023C3
:106F600014E078690BF0DEFC3861786934F052F88F
:106F70003B69002B01D1002308E03969054832F054
:106F800043FBF860386934F045F8FB681846183759
:106F9000BD4680BD6C81040880B584B000AF7860C8
:106FA0007868FFF7D1FFF860FB68002B02D0F86823
:106FB00022F0EBFFF86834F02DF8034822F022FFAE
:106FC0001037BD4680BD00BF149F040880B582B055
:106FD00000AF1B2036F0D8FF78607B681846083772
:106FE000BD4680BD80B500AF022036F0CDFF034620
:106FF000184680BD80B582B000AF78600B46FB704C
:10700000FB1C01221946786832F082FA0837BD4627
:1070100080BD80B483B000AF78607B681B69002BB3
:1070200001D1002305E07B681A697B681B68134463
:107030001B7818460C37BD465DF8047B704780B45A
:1070400083B000AF78607B681A687B685B689A429F
:1070500034BF01230023DBB218460C37BD465DF870
:10706000047B704780B582B000AF78607B68DB68D6
:10707000184633F0CFFF0837BD4680BD80B584B0D9
:1070800000AF786039603968786804F0D3FDF86043
:10709000FB68002B0AD0F86836F03FFA034683F00D
:1070A0000103DBB2002B01D0012300E00023FB72BF
:1070B000FB7A03F00103FB72F86833F0ABFFFB7A55
:1070C00018461037BD4680BD80B58AB000AF7860E5
:1070D0000B46FB7000222449786831F063FC38626B
:1070E000002387F82730386A36F053F80346002B20
:1070F00030D007F10C030022396A18462DF0ECFC61
:107100001BE007F10C03184604F0C5F803461A46C5
:10711000FB7893420CBF01230023DBB21A4697F899
:1071200027301343002B14BF0123002387F8273097
:1071300007F10C0318462DF0E1FD07F10C0318468A
:1071400004F0BFF80346002BDBD107F10C0318460F
:1071500004F0D9F8386A33F05DFF97F82730184605
:107160002837BD4680BD00BF8881040880B500AFC8
:10717000052036F009FF0346184680BD80B588B06B
:1071800000AFF860B9607A60F86822F0D6FC034678
:10719000FB77786836F0B1F90346002B06D0002261
:1071A0003849F86831F0FEFB786002E0786837F023
:1071B00055F907F110037A68B96818461CF04CF8C5
:1071C0000346BB77BB7F83F00103DBB2002B03D008
:1071D000786833F01FFF51E03B69184634F0EEF950
:1071E00003461A462849F86831F0CCFC7B68002B2E
:1071F00005D07A682349F86831F0C4FC03E02149DE
:10720000F86831F0D1FCFB7F102B10D9FB7F1A2BD3
:107210000DD8FB7F142B30D9FB7F1A2B2DD807F10B
:107220001002FB7F114618460EF02CFC26E0FB7F77
:10723000002B23D17B7DFF2B09D07B7D01211846BC
:1072400012F044FB7B7D0121184621F08BFF3B7D32
:10725000FF2B0AD03B7D0521184612F037FB07F1C2
:1072600010031946F8681CF0CFF9BB7DFF2B05D041
:10727000064901202BF0E2F800E000BF2037BD46B0
:1072800080BD00BF908104089C810408A881040887
:1072900080B58AB000AF7860786822F04EFC034673
:1072A00087F8273000222F49786831F07BFB38625D
:1072B0003B6A002B04D12C4901202BF0BFF84EE093
:1072C00000222A49786831F06DFBF86107F10C0360
:1072D0003A6AF96918461BF0BFFFF969386A33F05A
:1072E000C5FE2249786831F05FFC1E49786831F0AC
:1072F0005BFC97F82730102B03D997F827301A2B0F
:1073000006D907F10C03194678681CF001FA06E06B
:1073100097F82730FF22002118461EF0D3FEBB7CD1
:10732000FF2B04D0BB7C0421184612F0CFFAFB7C63
:10733000FF2B04D0FB7C0421184612F0C7FA3B7CDB
:10734000FF2B04D03B7C0421184612F0BFFA7B7C53
:10735000FF2B04D07B7C0421184612F0B7FA2837A3
:10736000BD4680BD90810408D08104089C8104083A
:1073700080B500AF1CF012FA0346184680BD80B5F8
:107380008AB000AFF860B96011461A460B46FB712F
:107390001346BB7107F1140207F124031946F8687C
:1073A0001CF0A2F8034683F00103DBB2002B23D1CB
:1073B000FB79002B03D0B86834F09EFFB8607B6A7D
:1073C00007F114021946B8682DF002FAFB79002B78
:1073D00002D0B86833F01EFEBB79002B0DD07B6A5B
:1073E00007F1140211460D2098477B6A07F1140239
:1073F00011460A20984700E000BF2837BD4680BDEF
:1074000080B582B000AF786039600023012239680E
:107410007868FFF7B4FF0837BD4680BD80B582B0FD
:1074200000AF786039600123012239687868FFF77E
:10743000A6FF0837BD4680BD80B582B000AF78603A
:1074400039600023002239687868FFF798FF083711
:10745000BD4680BD80B584B000AF786039603B68C0
:107460001B78FB737B68DAB2FB7B114618461EF073
:10747000D2FA1037BD4680BD80B584B000AF7860C9
:107480003960786822F059FB0346FB73FB7B102BB5
:107490000AD9FB7B1A2B07D807F10F031A460449B8
:1074A00038682DF095F900E000BF1037BD4680BD6B
:1074B0005574000880B500AF37F03EF880BD90B538
:1074C00083B000AF786078683AF08AFA03460C46D9
:1074D0001846214637F05EF80C37BD4690BD90B592
:1074E00083B000AF786078683AF07AFA03460C46C9
:1074F0001846214637F08AFD034618460C37BD462C
:1075000090BD90B585B000AF786078683AF068FAC1
:1075100003460C461846214637F078FDF860FB68B4
:10752000002B01D1002303E0F86808F03BF9034683
:1075300018461437BD4690BD90B585B000AF786051
:1075400078683AF04DFA03460C461846214637F063
:107550005DFDF860FB68002B01D1002304E00021F1
:10756000F86834F021F9034618461437BD4690BD3B
:1075700080B588B002AFF860B9607A603B60B868E7
:1075800035F018FF0346002B0AD000220021B8680E
:1075900007F022FF786100237B6000233B6003E05B
:1075A000B86833F0F7FC7861F8683AF019FA3B688C
:1075B00001937B68009300237A6937F04DFD034601
:1075C000FB74786933F026FDFB7C18461837BD46FE
:1075D00080BD80B500AF37F0B1FE0346184680BDD0
:1075E00080B500AF37F0A0FA80BD80B500AF37F0AE
:1075F00059FC80BD80B500AF0121002037F0F0F8C4
:107600000346184680BD80B582B000AF1B2036F01F
:10761000BBFC78607B6818460837BD4680BD80B4E7
:1076200083B000AF78607B681B69002B01D1002319
:1076300005E07B681A697B681B6813441B78184651
:107640000C37BD465DF8047B704780B483B000AF53
:1076500078607B681A687B685B689A4234BF012354
:107660000023DBB218460C37BD465DF8047B70473B
:1076700080B582B000AF78607B68DB68184633F075
:10768000C9FC0837BD4680BD80B500AF34F022F894
:107690000346184680BD000080B586B000AF786014
:1076A0003960786822F049FA0346FB7507F10C034C
:1076B000396818461CF030FB034683F00103DBB247
:1076C000002B39D1FB7D202B0AD9FB7D242B07D839
:1076D00007F10C02FB7D114618460EF02FFB1AE055
:1076E000FB7D002B28D17B7CFF2B04D07B7C0121F0
:1076F000184612F0EBF8BB7CFF2B04D0BB7C0421B6
:10770000184612F0E3F8FB7CFF2B04D0FB7C012130
:10771000184612F0DBF83B68002B09D0084A39689C
:10772000786830F032FD0346184633F073FC03E00E
:107730000349786831F038FA1837BD4680BD00BF7C
:107740009081040880B584B000AF786039603B68F0
:107750001B683A680432114678689847F8607B687D
:10776000002B04DB3B685B695A1C3B685A61FB6871
:10777000002B11DB3B681833FA68D2B21146184669
:107780002EF000F83B68183318462EF071F83B686D
:107790001B695A1C3B681A611037BD4680BD00004A
:1077A00080B5A2B000AFF860B9601346FB71F8680D
:1077B00022F0C3F9034687F8733007F128031A1D36
:1077C00007F128031946F8681CF046FB034683F0CE
:1077D0000103DBB2002B01D0002304E10023C7F832
:1077E000843097F87330202B09D997F87330242B05
:1077F00005D897F87330012118460EF0F1FCFB799B
:10780000FF2B04D0FB790021184621F0ABFCB868AF
:1078100035F056FD0346002B26D0B86832F094F9B7
:10782000C7F88000D7F88030002B02DA0023C7F8B1
:107830008030BB6A07F1280204321146D7F8800075
:107840009847F867FB6F002B08DABB6A07F128023C
:10785000043211464FF0FF309847F867F86F33F065
:10786000ADFEC7F88400B4E0B86835F092FC03467A
:10787000002B72D0FFF7C7FEC7F8840007F114038E
:107880000022B96818462DF027F90023BB670023B2
:107890007B6729E007F114031846FFF7C0FE034693
:1078A00087F87230BB6F0133BB67BB6A97F8720011
:1078B00007F12802043211469847F866FB6E002B48
:1078C0000DDB7B6F01337B67FB6EDBB2BB7407F1B3
:1078D000120301221946D7F8840031F019FE07F18E
:1078E000140318462DF00AFA07F114031846FFF79F
:1078F000ACFE0346002B07D02CF0C6F8034683F0FD
:107900000103DBB2002BC5D107F114031846FFF7C2
:10791000AFFE15E07B6F01337B67BB6A07F128027E
:10792000043211464FF0FF3098470346DBB2FB7438
:1079300007F1130301221946D7F8840031F0E8FD5E
:107940007A6FBB6F9A4244DA2CF09EF8034683F0BC
:107950000103DBB2002BDDD13BE0B8682DF06EF8FF
:10796000B866B96E01202CF0EDFDC7F88400D7F899
:107970008430002B2DD00023FB63FB6BBB6307F12E
:10798000280318330022D7F8841018462DF07AFB0C
:1079900007F128031A461649B8682CF019FF06E0CB
:1079A00007F1280319464FF0FF30FFF7CBFEBA6B03
:1079B000FB6B9A4207DA2CF067F8034683F0010369
:1079C000DBB2002BECD107F12803183318462DF059
:1079D00080FFFB79FF2B04D0FB790121184621F0B1
:1079E000C1FBD7F8843018468837BD4680BD00BF3C
:1079F0004577000880B58AB000AF78603960786854
:107A000022F09BF8034687F8263007F10C0207F1B5
:107A10001803194678681CF01FFA034683F0010327
:107A2000DBB2002B5DD1FF2387F82730386831F0B7
:107A300059F938623B6A002B1CDD3B6A013B194651
:107A4000386831F041FBF861F86935F0FDFA03461A
:107A5000002B0CD0F86921F0C3FA034687F82730D1
:107A600038682EF0C9F90346184633F0D3FAF8699E
:107A700033F0D0FA97F82630202B09D997F8263022
:107A8000242B05D897F82630002118460EF0A8FBC5
:107A900097F82730FF2B05D097F82730002118469C
:107AA00021F060FBBB6907F10C02194638682CF025
:107AB0008FFE97F82630202B08D997F82630242BF4
:107AC00004D897F8263018460EF0C6FB97F82730F2
:107AD000FF2B07D097F827300121184621F042FBF1
:107AE00000E000BF2837BD4680BD000080B592B0E1
:107AF00000AFF860B9607A603B60F86822F01DF86A
:107B0000034687F8473097F84730202B03D997F87A
:107B10004730242B04D9544901202AF08FFCA0E0DF
:107B200097F84730012118460EF018FB7B68002BB0
:107B300006D13B68002B03D101237B6003233B600C
:107B40007B6803F00F037B603B6803F00F033B602F
:107B500097F84730184611F07DFB034683F0010388
:107B6000DBB2002B0CD007F13C0318461CF0F9FAED
:107B700007F13C0297F84730114618460EF0DEF840
:107B800097F84730002118460EF02AFB97F850303E
:107B9000FF2B05D097F850300021184621F0E2FA6B
:107BA000B86835F08DFB0346002B0BD0B86831F078
:107BB000CBFF0346D9B297F847003B687A681CF0C0
:107BC000C1F939E0B86835F000FE0346002B2ED02D
:107BD00011F030FE07F110030122B96818462DF0AC
:107BE00087FE14E007F1100318462DF09BFF0346B3
:107BF00087F8463097F8461097F847003B687A6850
:107C00001CF0A0F907F11003184629F0CDFF07F189
:107C10001003184629F082FF0346002BE2D107F13A
:107C2000100318462AF012F811F00BFE04E0BA68AF
:107C30000E4901202AF002FC97F8473018460EF052
:107C40000BFB97F85030FF2B05D097F850300121EF
:107C5000184621F087FA97F84730002118460EF0B1
:107C60007DFA4837BD4680BDF881040820820408AB
:107C700080B592B000AFF860B9607A603B60F86898
:107C800021F05BFF034687F8473097F84730202BF9
:107C900003D997F84730242B04D9534901202AF0FF
:107CA000CDFB9EE097F84730012118460EF056FABA
:107CB0007B68002B06D13B68002B03D103237B603C
:107CC0000F233B607B68DBB27B603B68DBB23B60D1
:107CD00097F84730184611F0BDFA034683F00103C8
:107CE000DBB2002B0CD007F13C0318461CF039FA2C
:107CF00007F13C0297F84730114618460EF01EF87F
:107D000097F84730002118460EF06AFA97F850307D
:107D1000FF2B05D097F850300021184621F022FAA9
:107D2000B86835F0CDFA0346002B0BD0B86831F0B7
:107D30000BFF0346D9B297F847003B687A681CF0FE
:107D400065F939E0B86835F040FD0346002B2ED0C8
:107D500011F070FD07F110030122B96818462DF0EB
:107D6000C7FD14E007F1100318462DF0DBFE0346B3
:107D700087F8463097F8461097F847003B687A68CE
:107D80001CF044F907F11003184629F00DFF07F124
:107D90001003184629F0C2FE0346002BE2D107F17A
:107DA0001003184629F052FF11F04BFD04E0BA68A9
:107DB0000E4901202AF042FB97F8473018460EF092
:107DC0004BFA97F85030FF2B05D097F8503001212F
:107DD000184621F0C7F997F84730002118460EF0F1
:107DE000BDF94837BD4680BD54820408208204088E
:107DF00080B500AF33F06EFC0346184680BD00002E
:107E000080B584B000AF78603960786821F095FE65
:107E10000346FB7307F10803396818461AF05CFE45
:107E20000346002B3BD0FB7B242B0AD9FB7B272B63
:107E300007D807F10802FB7B114618460EF054FAEA
:107E40001CE0FB7B002B19D13B7BFF2B09D03B7B3C
:107E50000121184611F01CFF3B7B0321184611F04D
:107E600035FD7B7BFF2B09D07B7B0121184611F070
:107E70000FFF7B7B0321184611F028FD3B68002B88
:107E800009D0084A3968786830F07FF90346184607
:107E900033F0C0F803E00349786830F085FE10370E
:107EA000BD4680BD9081040880B584B000AF786085
:107EB00039603B6801221A70786835F07BFA034616
:107EC000002B1AD000221149786830F06BFDF86061
:107ED000FB68002B06D0F86832F0FCF803461A461F
:107EE0003B681A7000220A49786830F05BFD03464F
:107EF000184632F0D5F8034603E0786831F024FEE6
:107F0000034618461037BD4680BD00BF7C8204087A
:107F10008482040890B58FB002AFF860B9607A60CF
:107F2000F86821F00AFE034687F82B300123FB771F
:107F300007F11F031946B868FFF7B6FF7862002300
:107F4000BB6107F118031946786834F02DFCF8621C
:107F5000FB6A002B23D178682CF070FD0346BB61CF
:107F6000BB6903F580742BF0B5F903469C4204D934
:107F7000354901202AF062FA11E0BB690733073363
:107F8000DB08DB00ADEB030D02AB0733DB08DB00E6
:107F9000FB62BB691A46F96A78682CF083FDFB6ABC
:107FA000002B4ED0BB69002B4BD097F82B30242BE5
:107FB0000FD997F82B30272B0BD87B6AD9B2BB6926
:107FC0001A46FB7F97F82B000093FB6A0EF018FA15
:107FD00037E097F82B30002B33D100221B49F8688B
:107FE00030F0E0FC386207F11003396A18461AF0E5
:107FF00073FD0346002B15D000221549F86830F0B8
:10800000D1FC0346184632F065F80346BB757B6A1F
:10801000D9B2BB691A46FB7F07F110000093FB6AD7
:108020001AF074FFBB7D184633F0DDFA03461A469A
:108030000749F86830F02EFD0346396A184633F0D8
:1080400015F83437BD4690BD587C0408908104086B
:108050008C82040890B599B002AFF860B9607A607C
:10806000F86821F06AFD034687F85330012387F84A
:108070003F3007F13F031946B868FFF715FFF86472
:108080007B68002B01DC002398E07B6803F580749B
:108090002BF020F903469C4205D94A4901202AF0D9
:1080A000CDF900238AE07B6807330733DB08DB0068
:1080B000ADEB030D02AB0733DB08DB00BB6497F8C5
:1080C0005330242B0FD997F85330272B0BD8FB6C48
:1080D000D9B297F83F3097F853000093BB6C7A6899
:1080E0000EF042FA3CE097F85330002B36D10022D4
:1080F0003549F86830F056FC786407F13803796C3C
:1081000018461AF0E9FC0346002B16D000222F492E
:10811000F86830F047FC0346184631F0DBFF0346B1
:1081200087F83E30FB6CD9B297F83F3007F1380042
:108130000093BB6C7A681AF032FF97F83E3018460D
:1081400033F051FA03461A462049F86830F0A2FC91
:108150000346796C184632F089FF01E000232DE0D8
:10816000796801202CF0EEF938643B6C002B24D0A8
:1081700007F110030022396C18462CF083FF00230E
:108180007B6511E0BA6C7B6D13441A7807F110031C
:10819000114618462DF0F6FA07F1100318462DF097
:1081A00067FB7B6D01337B657B687A6D9A42E9D30F
:1081B00007F1100318462DF08CFB3B6C18465C371A
:1081C000BD4690BD94820408908104088C82040806
:1081D00080B582B000AF1B2035F0D6FE78607B689A
:1081E00018460837BD4680BD80B584B000AF7860C2
:1081F000786835F0DFF8034683F00103DBB2002B2B
:1082000001D0002316E000220C49786830F0CAFB48
:10821000B8600023FB60B86834F0BBFF0346002B56
:1082200004D0B86834F041FA0346FB60B86832F015
:10823000F1FEFB6818461037BD4680BDCC820408AD
:1082400080B586B000AF78603960786835F0B2F8F4
:10825000034683F00103DBB2002B01D000233DE095
:1082600000222049786830F09DFB786100233B6153
:10827000786934F08EFF0346002B28D0786934F0FB
:1082800014FAF8603B68002B03DD3A68FB689A42F9
:1082900008D37B693B6100237B611249786830F029
:1082A00083FC17E03B681A460021786931F03CFAFC
:1082B00038613B686FF000421946786931F034FA52
:1082C000B860BA680749786830F05CFC02E0FFF7F4
:1082D0007FFF3861786932F09DFE3B691846183798
:1082E000BD4680BDCC82040880B58AB000AFF8607E
:1082F000B9601346FB71F86835F05CF8034683F00B
:108300000103DBB2002B04D0474A4A2147482AF038
:1083100009F9BB68184634F03CFF034683F00103BB
:10832000DBB2002B04D0424A4B2140482AF0FAF835
:10833000012387F8273000223E49F86830F03CF8E6
:1083400038623B6A002B1FD007F108030122396A0B
:10835000F8681FF02DFE034683F00103DBB2002B0B
:108360000ED035482AF026F8344B1B78DBB243F0A8
:108370000403DAB2314B1A702E49F86830F014FC5D
:10838000386A32F047FE48E000222D49F86830F0A4
:1083900009FBF861F86934F0FCFE034683F0010341
:1083A000DBB2002B06D0BB681A462549F86830F0CE
:1083B00071FB32E0F86934F078F9B861BB681846AF
:1083C00034F073F97861BA697B691344B3F5007FBF
:1083D0000DD9FB79002B07D0184B1B78DBB243F08B
:1083E0000203DAB2154B1A70002387F8273097F88A
:1083F0002730002B02D1FB79002B0BD0BB69B3F5E2
:10840000007F07D2B968BB69C3F500730022F86921
:1084100031F02CF9F86932F0FDFD97F82730184655
:108420002837BD4680BD00BFF87B0408D48204080D
:10843000E882040800830408088304084D510120E1
:10844000CC82040880B582B000AF1B2035F09CFDC3
:1084500078607B6818460837BD4680BD80B483B01D
:1084600000AF0346FB71FB79602B06D9FB797A2BB1
:1084700003D8FB79203BDBB200E0FB7918460C37D0
:10848000BD465DF8047B704780B483B000AF0346FF
:10849000FB71FB79402B06D9FB795A2B03D8FB796A
:1084A0002033DBB200E0FB7918460C37BD465DF89F
:1084B000047B704780B483B000AF78607B681B6931
:1084C000002B01D1002305E07B681A697B681B68DB
:1084D00013441B7818460C37BD465DF8047B704783
:1084E00080B483B000AF78607B681A687B685B6893
:1084F0009A4234BF01230023DBB218460C37BD4635
:108500005DF8047B704780B483B000AF78607B680F
:108510009A687B681B68134418460C37BD465DF8A3
:10852000047B704780B582B000AF78607B68DB6801
:10853000184632F06FFD0837BD4680BD80B582B069
:1085400000AF78607B681B68002B01D1002305E039
:108550007B681B68184632F0BBF90346184608379B
:10856000BD4680BD80B483B000AF78607B681B6877
:10857000002B14BF01230023DBB218460C37BD4685
:108580005DF8047B704780B582B000AF78607B688F
:108590001B68184632F03EFD0837BD4680BD80B5E9
:1085A00082B000AF7860786830F09CFB0346002B07
:1085B00003D1FFF747FF034608E00021786830F059
:1085C00083FD0346184633F073FF03461846083709
:1085D000BD4680BD80B586B000AF7860786834F065
:1085E0000AFF034683F00103DBB2002B04D01F4ACD
:1085F0004A211F4829F096FFFFF724FF78617B6925
:10860000002B01D100232CE007F1100379681846F4
:108610002CF090FC17E007F110031846FFF78EFFCF
:108620000346184631F03CFD0346DBB2FB7307F10D
:108630000F0301221946786930F06AFF07F1100331
:1086400018462CF0CAFC07F110031846FFF78AFF02
:108650000346002BDFD107F110031846FFF793FF05
:108660007B6918461837BD4680BD00BF3C830408AF
:108670004C83040880B58AB000AF78603960FFF79A
:10868000E1FE78627B6A002B2AD0786834F081FDA5
:108690000346002B24D03B68002B21DB3A6807F10E
:1086A0001003796818462CF017FA07F110031846E2
:1086B000FFF716FF0346002B0DD007F110031846F5
:1086C000FFF7F8FE0346FB7307F10F03012219467B
:1086D000786A30F01DFF07F110031846FFF722FFFC
:1086E0007B6A18462837BD4680BD80B582B000AF92
:1086F000786039603B681946786831F03BF803468A
:1087000018460837BD4680BD80B58CB002AFF86012
:10871000B9607A60FB70F86834F03BFD034683F083
:108720000103DBB2002B01D0002380E0B86833F0F6
:10873000E3FDB860BB68002B01D1002377E0F86847
:1087400033F0B3FF0346BB61B86833F0AEFF0346B6
:108750007B617A69BB699A4205DDB86832F05AFCE0
:108760004FF0FF3363E0BA697B69D31A3B61FB7852
:1087700083F00103DBB2002B1CD001233B623B6979
:108780000133FB6100237B62786834F099FD034676
:10879000002B2DD0786831F0D7F978627B6A002BF6
:1087A00001DA00237B627A6AFB699A4220DDFB6969
:1087B0007B6233E04FF0FF333B624FF0FF33FB61EE
:1087C0003B697B62786834F07BFD0346002B25D043
:1087D000786831F0B9F978627B6A002B01DA0023FE
:1087E0007B627A6A3B699A4218DD3B697B6215E0DD
:1087F00000BF13E07A6A012300930023B968F86888
:1088000032F0AAF90346002B04D1B86832F002FC1A
:108810007B6A0CE07A6A3B6A13447B627A6AFB6982
:108820009A42E7D1B86832F0F5FB4FF0FF331846B3
:108830002837BD4680BD000080B58AB000AF7860A3
:108840003960786834F0A5FC034683F00103DBB29D
:10885000002B01D00023A8E0386834F04EFE034618
:10886000002B01D00023A0E0524938682BF02EFEE7
:108870000346002B68D0002032F0A0FE03461A46C3
:108880004D49386830F07EF97968386803F0D2F9DC
:10889000786267213868FEF717FC034683F001030E
:1088A000DBB2002B01D07B6A7FE032F01BFF386225
:1088B0003B6A002B2ED1002377E00021786A30F04C
:1088C00003FCF86100223D49786A30F06BF80346FA
:1088D000184631F0E5FBB861F86933F0E6FE03466F
:1088E0007B61BA697B6913443B61F969386A2DF091
:1088F00007FA786A32F08EFB386932F05FFE034681
:108900001A462D49386830F03DF97968386803F027
:1089100091F978627B6A002B08D0786A34F0FDFD0B
:10892000034683F00103DBB2002BC6D1786A32F034
:1089300071FB002032F042FE03461A461E49386899
:1089400030F020F93B6A30E0386833F0D5FC38600D
:108950000023002239687868FFF7D6FEF860FB68CC
:10896000002B1EDB32F0BEFEB860BB68002B04D1CA
:10897000386832F04FFB002317E03968B86830F0F0
:10898000F5FCF86832F01AFE03461A460B49B8683F
:1089900030F0F8F83A680A49B86830F0F3F8BB6884
:1089A00003E0386832F036FB002318462837BD460E
:1089B00080BD00BF608304086883040874830408D2
:1089C0007C83040890B5AFB002AFF860B9607A60FC
:1089D000F86833F091FCC7F8AC00E349B8682BF0B5
:1089E00075FD0346002B00F0C781786834F089FCE0
:1089F0000346002B05D1786834F0CBFB0346002BEF
:108A000005D0786835F02AFDC7F8A80004E078683A
:108A100033F072FCC7F8A800002032F0CFFD034607
:108A20001A46D249B86830F0ADF86721B868FEF749
:108A30004BFB034687F89B30D7F8AC10B86803F0BF
:108A4000F9F8C7F8A40060E10021D7F8A40030F0DD
:108A50003BFBC7F894000022C549D7F8A4002FF0CB
:108A6000A1FF0346184631F01BFBC7F89000D7F86A
:108A7000940033F01AFE0346C7F88C30D7F89030D4
:108A80001A460021D7F8AC0030F04EFEC7F8880037
:108A900007F15C030022D7F8881018462CF01CF868
:108AA00007F15C0318462CF033F9D7F8A80034F02E
:108AB00028FC0346002B78D00023C7F8A030D7F855
:108AC000A040631CC7F8A030D7F8940035F0C6FC6E
:108AD0000246A30007F1B0010B4443F89C2C0CE0C4
:108AE000D7F8A0305A1CC7F8A0209B0007F1B002AD
:108AF0001344D7F8842043F89C2CD7F8A0301946AB
:108B0000D7F8A40030F0E0FAC7F88400D7F8843032
:108B1000002BE5D1D7F8A040631CC7F8A030002295
:108B20009349D7F8A4002FF03DFF0246A30007F1B8
:108B3000B0010B4443F89C2CD7F8A040631CC7F845
:108B4000A03000228B49D7F8A4002FF02BFF02465B
:108B5000A30007F1B0010B4443F89C2CD7F8A030D8
:108B600007F1140201920093002300220021D7F89C
:108B7000A80027F0A9FA0346184633F099FCC7F875
:108B8000800007F114031946D7F8A00032F0A4FAC8
:108B900007F15C030022D7F8801018462CF09CF9EE
:108BA000D7F8800032F036FA70E007F1480300226F
:108BB000D7F8A81018462BF08FFF5AE007F14803AA
:108BC0001846FFF777FC034687F87F3097F87F3029
:108BD000242B41D107F1480318462CF08FF807F1F8
:108BE00048031846FFF766FC034687F87F300023EA
:108BF000C7F89C3097F87F30302B0DD997F87F302D
:108C0000392B09D897F87F30303B1946D7F8A400A4
:108C100030F05AFAC7F89C00D7F89C30002B0CD0E3
:108C200007F15C030022D7F89C1018462CF054F989
:108C3000D7F89C0032F0EEF916E007F15C0324212E
:108C400018462CF0B5F897F87F2007F15C03114621
:108C500018462CF0ADF807E097F87F2007F15C0389
:108C6000114618462CF0A4F807F1480318462CF0DA
:108C700045F807F148031846FFF732FC0346002B7E
:108C80009CD107F148031846FFF74CFC07F15C0341
:108C90001846FFF738FC03460133BB67D7F890202E
:108CA000D7F88C3013441A4607F15C03D7F8AC10A0
:108CB00018462CF011F907F15C031846FFF732FC57
:108CC000D7F89410D7F8AC0032F0D0F9D7F8883044
:108CD000C7F8AC30D7F8A40032F09CF90023C7F8ED
:108CE000A43097F89B30002B0FD0B86F32F066FCA1
:108CF00003461A461D49B8682FF044FFD7F8AC1058
:108D0000B86802F097FFC7F8A400D7F8A430002B8A
:108D100012D0D7F8A40034F000FC034683F001031E
:108D2000DBB2002B08D02AF0AFFE034683F001032C
:108D3000DBB2002B7FF488AED7F8A40032F06AF9DA
:108D4000D7F8A80032F066F997F89B30002B08D0CE
:108D5000002032F033FC03461A460449B8682FF06D
:108D600011FFD7F8AC3042E0608304086883040840
:108D7000748304087C830408786833F0BDFA786053
:108D8000B86833F0B9FAB86000230022B968F8680F
:108D9000FFF7BAFC78677B6F002B22DB7B6F1A46EC
:108DA0000021D7F8AC0030F0BFFC38676FF000430B
:108DB00000227968386F30F059FCB86833F075FCE0
:108DC00002467B6F1A446FF00043D7F8AC10386F3F
:108DD00030F04CFCD7F8AC0032F01CF93B6FC7F810
:108DE000AC307968B86832F041F9D7F8AC30184641
:108DF000B437BD4690BD00BF80B588B000AFF86005
:108E0000B9607A60786834F078FB0346002B04D1AF
:108E1000786830F099FE034601E06FF00043FB6193
:108E2000BB68002B01DA0023BB60FB69002B01DA71
:108E30000023FB61FA69BB689A4205DABB68BB6133
:108E4000FB69BB60BB69FB61FFF7FCFA78617B697A
:108E5000002B01D1002309E0B968FA69BB68D31A75
:108E60000A46F968786930F001FC7B6918462037BA
:108E7000BD4680BD80B586B000AFF860B9607A604D
:108E8000786834F03AFB0346002B04D1786830F060
:108E90005BFE034601E06FF000437B617B69002BC2
:108EA00001DA00237B61BB68002B07DAF86833F036
:108EB000FCFB03461A46BB681344BB60BB68002B2F
:108EC00001DA0023BB60FFF7BDFA38613B69002B74
:108ED00001D1002306E0BA687B69F968386930F08F
:108EE000C5FB3B6918461837BD4680BD80B586B0C6
:108EF00000AFF860B9607A60786834F0FEFA034633
:108F0000002B04D1786830F01FFE034601E06FF0BB
:108F100000437B61BB68002B07DAF86833F0C5FBC0
:108F200003461A46BB681344BB607B69002B07DA13
:108F3000F86833F0BAFB03461A467B6913447B6139
:108F4000BB68002B01DA0023BB607B69002B01DAD0
:108F500000237B61FFF776FA38613B69002B01D172
:108F600000230DE07A69BB689A4208DDB9687A6926
:108F7000BB68D31A0A46F968386930F077FB3B6959
:108F800018461837BD4680BD80B590B002AF7860F6
:108F90003960786834F0FDF8034683F00103DBB2F2
:108FA000002B01D00023E3E032F09CFB78627B6A67
:108FB000002B01D10023DBE0386834F09EFA034631
:108FC000002B05D07968786A30F0D0F97B6ACFE061
:108FD000694938682BF07AFA0346002B63D00023E6
:108FE0007B63002032F0EAFA03461A466349386888
:108FF0002FF0C8FD7968386802F01CFE386338E04D
:109000000021386B30F060F8386200225C49386B20
:109010002FF0C8FC0346184631F042F8F861386A70
:1090200033F043FB0346BB61386A31F0F3FF796BE1
:10903000FA697B6BD31A1A46786830F075FB0346E1
:109040001946786A2CF05CFEFA69BB6913447B63AD
:10905000386B31F0DFFF786B32F0B0FA03461A4616
:10906000464938682FF08EFD7968386802F0E2FDD5
:1090700038633B6B002B08D0386B34F04EFA034654
:1090800083F00103DBB2002BBAD1386B31F0C2FFA1
:10909000002032F093FA03461A46384938682FF018
:1090A00071FD7B6A64E0386833F026F9386000238C
:1090B000BB62386834F021FA0346002B04D13868CB
:1090C00033F0F3FA034600E000237B61786833F065
:1090D000ECFA03465A1C7B69D31A3B610023FB62FE
:1090E0003EE07B69002B02D1FB6A002B34D0FA6A88
:1090F0003B699A420DD07B69002B0AD0FA6A0123A2
:10910000009300233968786831F026FD0346002B70
:1091100023D1FA6A3B699A4206D13A697B691344C2
:10912000FB627B69002B1FD0B96AFA6ABB6AD31A4B
:109130001A46786830F0F8FAF860FB68002B13D014
:10914000F968786A30F012F9F86831F063FFFA6A6A
:109150007B691344BB6200E000BFFB6A0133FB6222
:10916000FA6A3B699A42BCDD386831F053FF7B6A8A
:1091700018463837BD4680BD6083040868830408FC
:109180007483040880B590B000AF78600B46FB7024
:10919000FFF758F9F863FB6B002B01D100234FE078
:1091A000786833F0A9F8B86307F120030022B96B9F
:1091B00018462BF091FC07F10C030022F96B1846BE
:1091C0002BF08AFC26E007F120031846FFF772F91E
:1091D000034687F83730FB78002B06D097F83730F6
:1091E0001846FFF73BF9034605E097F83730184675
:1091F000FFF74AF9034687F8373097F8372007F129
:109200000C03114618462BF0D3FD07F12003184636
:109210002BF074FD07F120031846FFF761F90346B0
:10922000002BD0D107F120031846FFF77BF907F197
:109230000C031846FFF776F9B86B31F0EBFEFB6BC9
:1092400018464037BD4680BD80B58EB000AF78600F
:10925000786833F051F8B862BB6A002B01D1BB6A61
:1092600056E000237B634FF0FF333B6307F10C03B1
:109270000022B96A18462BF02FFC27E007F10C03F7
:109280001846FFF717F90346184628F0E3FD034692
:1092900087F8273097F8273083F00103DBB2002BE3
:1092A0000FD03B6B002B05DA07F10C031846FFF7D4
:1092B0002AF9786307F10C031846FFF724F90346EF
:1092C0003B6307F10C0318462BF018FD07F10C0364
:1092D0001846FFF705F90346002BCFD107F10C0321
:1092E0001846FFF71FF90023FB627B6B3A6B9A422B
:1092F00004DB3A6B7B6BD31A0133FB62FA6A796B3E
:10930000B86A30F011FA3862B86A31F083FE3B6A0D
:1093100018463837BD4680BD90B589B002AFF860B9
:10932000B9607A60F86833F034FF034683F00103D4
:10933000DBB2002B01D0002326E0B86832F0DCFF5E
:1093400038610023FB757B68002B19DB386933F02B
:10935000ACF902467B68D418F86833F0A6F90346E6
:109360009C420DD87A680123009300233969F8687C
:1093700031F0F2FB0346002B0CBF01230023FB75E9
:10938000386931F047FEFB7D18461C37BD4690BD5D
:1093900090B58BB002AFF860B9607A60F86833F0CE
:1093A000F8FE034683F00103DBB2002B01D000235B
:1093B0003DE0786833F084FF0346002B04D07868E2
:1093C00030F0C2FB034603E0F86833F06EF9034661
:1093D000BB61B86832F090FF7861786933F065F965
:1093E0000246BB699B1ABB610023FB77BB69002B5C
:1093F00019DB786933F059F90246BB69D418F8686B
:1094000033F053F903469C420DD8BA690123009307
:1094100000237969F86831F09FFB0346002B0CBFED
:1094200001230023FB77786931F0F4FDFB7F1846B8
:109430002437BD4690BD80B582B000AF78607B68B0
:109440001B68002B01D1002305E07B681B681846D0
:1094500031F03EFA034618460837BD4680BD80B459
:1094600083B000AF78607B681B68002B14BF0123BA
:109470000023DBB218460C37BD465DF8047B70470D
:1094800080B582B000AF78607B681B68184631F009
:10949000C1FD0837BD4680BD80B586B000AFF8601D
:1094A000B9607A60BB68002B01D1174B00E0174B05
:1094B00000221946F8682FF075FA78617B69002B55
:1094C00001D100231CE07B68002B11D07B680022B7
:1094D0001A70786933F0A9FF0346002B08D07B6926
:1094E0009B8803F00F03022B02D17B6801221A70C4
:1094F000786930F0C5FF3861786931F08BFD3B69E0
:1095000018461837BD4680BDEC7D0408F47D04087C
:1095100080B592B000AF664B5B6800226549184683
:109520002FF040FA38643B6C002B00F0BB8007F151
:109530002C03396C18462BF0FDFCA2E007F12C033C
:109540001846FFF778FFF86300225B49F86B2FF0AD
:1095500029FA0346184630F0BDFD034687F8473028
:1095600097F84730002B76D000220021F86BFFF7E8
:1095700093FFB86307F10C031946B86B18F0B0FD00
:10958000034683F00103DBB2002B1FD000224B49BE
:10959000F86B2FF007FA03467B603A1D0123484918
:1095A000F86B1EF0F9FB7B68184631F033FD0023A1
:1095B00087F8473097F84730184632F014F80346DA
:1095C0001A463D49F86B2FF0DDFA41E0FB8B002B8A
:1095D0003ED0FA8BBB8B9A423AD0B86B34F0E0FEA7
:1095E00003461A46BB8B9A4214BF01230023DBB209
:1095F0007B6309223349F86B2FF0D4F903461846F0
:1096000030F04EFD38633A6B7B6B9A4220D0786B1A
:1096100031F0D4FF03461A462A49F86B2FF0B2FA0C
:109620007B6B002B01D1284B00E0244B0022194614
:10963000F86B2FF0B7F90346BB6007F1080201236E
:109640002249F86B1EF0A8FBBB68184631F0E2FC1B
:10965000B86B31F0DFFCF86B31F0DCFC97F8473089
:1096600083F00103DBB2002B06D007F12C03396C29
:1096700018462BF0E2FC04E007F12C0318462BF00F
:10968000ACFC07F12C031846FFF7E9FE0346002B5C
:109690007FF454AF07F12C031846FFF7F1FE386C46
:1096A00031F0B8FC002318464837BD4680BD00BFE6
:1096B00058510120387D0408887E0408EC7D040898
:1096C0008483040890830408F47D0408A0830408BC
:1096D00090B587B000AFB960C7E900230346FB73BC
:1096E000FB7B0321184610F0F1F84FF001034FF017
:1096F0000004C7E9043439E0D7E90012D7E904349B
:1097000003EA010304EA0204234314D010F092F8A0
:10971000FB7B0021184610F0BBFA0A2010F0AAF8D3
:10972000FB7B0121184610F0B3FA10F08AF83720BD
:1097300010F0A0F813E010F07DF8FB7B0021184634
:1097400010F0A6FA412010F095F8FB7B0121184695
:1097500010F09EFA10F075F8052010F08BF8D7E99C
:109760000434DB1844EB0404C7E90434BB685A1E14
:10977000BA60002BC0DC1C37BD4690BD80B584B0FC
:1097800000AF0346FB710C49002023F0BFFCF860DA
:10979000FB68002B01D100230AE0FB79184631F069
:1097A0007CFF03461A460549F8682FF0EBF9FB6881
:1097B00018461037BD4680BDAC830408207E0408DF
:1097C00080B584B000AF7860786804F0ABFA0346E7
:1097D000FB73FB7B184623F071FF034683F0010304
:1097E000DBB2002B01D0002304E0FB7B184604F021
:1097F000ADFA034618461037BD4680BDF0B58DB0B2
:1098000000AF78603960786804F08CFA034687F816
:10981000233097F82330184623F050FF034683F097
:109820000103DBB2002B7FD1386833F0B2FC034672
:1098300083F00103DBB2002B05D1386832F035FF2D
:109840000346102B05D03A683949032028F0F6FD6D
:109850006AE097F82330184604F078FA4FF00002D7
:109860004FF00003C7E90A2307F10C03002239680F
:1098700018462BF031F900237B623DE007F10C0321
:10988000184604F02DFA03463B7207F10C03184604
:109890002BF034FA07F10C03184604F021FA0346C2
:1098A0007B7207F10C0318462BF028FA0023BB72D9
:1098B00007F1080000230022102128F0D4FC024602
:1098C0000B46796AC900A1F12006C1F1200003FA14
:1098D00001F502FA06F6354322FA00F0054302FAD2
:1098E00001F4D7E90A2342EA040243EA0503C7E97F
:1098F0000A237B6A01337B627B6A072BBEDD07F19B
:109900000C03184604F002FA97F823004FF05502B2
:109910004FF000030821FFF7DBFE97F82300D7E99B
:109920000A234021FFF7D4FE3437BD46F0BD00BF07
:10993000B483040880B584B000AF7860786804F020
:10994000F1F90346FB73FB7B184623F0B7FE034691
:1099500083F00103DBB2002B07D1F87B4FF0CC0280
:109960004FF000030821FFF7B3FE1037BD4680BD5E
:1099700090B583B000AF786039603B6818787B6839
:109980004FF000041A4623460821FFF7A1FE0C37CA
:10999000BD4690BD80B586B000AFF860B960134693
:1099A000FB71F86804F0BEF90346FB75FB7D1846B1
:1099B00023F084FE034683F00103DBB2002B1FD1AA
:1099C00007F117031A461049B8682AF001FFFB791E
:1099D000002B0AD0FB7D0121184610F059F9FB7DC0
:1099E000012118460FF072FF0BE0FB7D04211846A1
:1099F0000FF06CFFFB7D0121184610F049F900E0E3
:109A000000BF1837BD4680BD7199000880B590B081
:109A100000AF78603960786804F084F9034687F80D
:109A20003B3097F83B30184623F048FE034683F05E
:109A30000103DBB2002B01D0002345E0386833F08E
:109A40003FFC0346002B34D0386830F07DF8F863D3
:109A5000F96B01202AF076FD78637B6B002B01D136
:109A6000002331E007F10C030022796B18462BF03C
:109A700009FB12E097F83B300821184604F09CF9E6
:109A80000346DAB207F10C03114618462BF07AFEB2
:109A900007F10C0318462BF0EBFEFB6B5A1EFA6322
:109AA000002BE7D107F10C0318462BF012FF7B6B5C
:109AB0000AE097F83B300821184604F07DF9034688
:109AC000184631F07BFD034618464037BD4680BD41
:109AD00090B597B000AF78603960786804F022F9EB
:109AE000034687F8373097F83730184623F0E6FDFD
:109AF000034683F00103DBB2002B01D0002339E1E0
:109B000031F0F0FD38633B6B002B01D1002331E1D4
:109B10003B68002B02DD3B68FF2B01DDF0233B603F
:109B200000237B6500233B650023FB620123FB646C
:109B30001BE10123BB6400237B6400233B640123FE
:109B400087F83F300023FB643B6D002B40F0BD8065
:109B500097F83730184604F0F9F8034683F001030C
:109B6000DBB2002B07D000237B6500233B6500237D
:109B7000FB623B6BFEE03B684FEAE37497F837000B
:109B80001A4623460821FFF7A3FD97F83730012135
:109B9000184604F011F9034687F82B3097F8373050
:109BA0000121184604F008F9034687F82A3097F88F
:109BB0002B30012B03D197F82A30012B79D097F85D
:109BC0002B2097F82A309A4204D097F82B3087F848
:109BD0003E3028E0BA6C7B6D9A4210DA07F1200221
:109BE0003B6C13441A7897F83F301340DBB2002BDC
:109BF00014BF01230023DBB287F83E3008E0BA6CC3
:109C00007B6D9A420CBF01230023DBB287F83E3004
:109C100097F83E30002B06D1BB6C7B647B6C082B25
:109C200001DC7B6CFB6297F83E30012B0FD107F112
:109C300020023B6C13441A7897F83F301343D9B293
:109C400007F120023B6C13440A461A7010E007F13A
:109C500020023B6C13441A7897F83F30DB43DBB2A9
:109C60001340D9B207F120023B6C13440A461A7024
:109C700097F83E304FF0000497F837001A46234615
:109C80000121FFF725FDBB6C0133BB6497F83F3022
:109C90005B0087F83F3097F83F30002B05D13B6CD5
:109CA00001333B64012387F83F303B6C072B7FF780
:109CB0006CAFBB6C402B08DD7B6C7B657B6D002B38
:109CC00001D101233B650123FB64FB6C002B03D016
:109CD00097F82030002B07D100237B6500233B65DC
:109CE0000023FB620023FB64FB6C002B3DD00023B0
:109CF000BB632BE0BB6B5C0007F12002BB6B134422
:109D00001B781B09DBB203F00F03184628F0A8FDEF
:109D100003461A4607F15803234403F84C2CBB6B47
:109D20005B005C1C07F12002BB6B13441B7803F043
:109D30000F03184628F094FD03461A4607F158030E
:109D4000234403F84C2CBB6B0133BB63BB6B072B69
:109D5000D0DD00233B7707F10C03184631F062FB9E
:109D600003461946386B2BF0CBFFFB6C002B7FF4BE
:109D7000E0AE3B6B18465C37BD4690BD80B582B007
:109D800000AF78607B681B68002B01D1002305E0E1
:109D90007B681B68184634F061FB03461846083799
:109DA000BD4680BD80B582B000AF78607B681B681F
:109DB000002B01D1002305E07B681B68184630F0BA
:109DC00087FD034618460837BD4680BD80B483B082
:109DD00000AF78607B681B68002B14BF0123002351
:109DE000DBB218460C37BD465DF8047B704780B582
:109DF00082B000AF78607B681B68184631F00AF9C2
:109E00000837BD4680BD000080B582B000AF034674
:109E1000FB71084B5868FB79002B01D0032300E04D
:109E200000231A4604492EF0BDFD034618460837A4
:109E3000BD4680BD58510120D883040890B58FB02D
:109E400000AFF860B9607A6078683A1D01236F4905
:109E50001DF0A2FF7B6800226D4918462EF0A2FD7E
:109E600078637B6800226B4918462EF09BFD3863AF
:109E70007B6B002B4DD03B6B002B4AD000226649F8
:109E8000786B2EF08FFD03467B617B69002B3CD005
:109E90007B69184632F009FC0346002B35D05E4939
:109EA000786B2EF081FE00225C49386B27F07AF83F
:109EB000F862F86A33F025FA0346002B0AD007F15E
:109EC00014030122396BF86A23F0E0FA03461846BE
:109ED00031F0A0F8F86A31F09DF87B680022504913
:109EE00018462EF05FFDB862B86A2FF02DFE0446CA
:109EF0007B69184632F0D9FB034623441946B86AF9
:109F00002FF018FFB86A31F085F87B69184631F0F8
:109F100081F87B680022434918462EF043FD034632
:109F2000184630F0D7F80346002B5CD03B6B002B73
:109F300039D03D49386B03F009FC3C49386B03F0DC
:109F400005FC00223749386B27F02CF87862786AD4
:109F500033F0D7F90346002B09D000230022396BD8
:109F6000786A23F093FA0346184631F053F8786A7A
:109F700031F050F800222D49386B27F013F8386281
:109F8000386A33F0BEF90346002B09D000230022C3
:109F9000396B386A23F07AFA0346184631F03AF8FA
:109FA000386A31F037F87B6B002B1CD01F49786B77
:109FB00003F0CCFB00221D49786B26F0F3FFF8611B
:109FC000F86933F09EF90346002B09D000230022E4
:109FD000796BF86923F05AFA0346184631F01AF8FB
:109FE000F86931F017F8396B786B31F03FF8B868E1
:109FF000FFF7C4FEB861B969F8682EF069FBB8696B
:10A0000031F008F83C37BD4690BD00BFE08304083E
:10A01000EC830408F4830408CC8204080084040858
:10A0200008840408148404084C8F04081884040865
:10A0300080B58EB000AFF860B9607A6000226B49DD
:10A0400078682EF0AFFC0346184630F043F803461C
:10A0500087F8363097F83630002B01D00023C0E067
:10A060000022634978682EF09DFC38630022614924
:10A0700078682EF097FC03467B6100225E49786881
:10A080002EF090FCF86200225C4978682EF08AFC81
:10A09000B862002387F83730FB6A002B00F08A8013
:10A0A000BB6A002B00F086807B69002B00F0828069
:10A0B0003B6B002B7ED000225149F86A26F072FFDC
:10A0C000786200224F49B86A26F06CFF3862786ADD
:10A0D00033F017F90346002B4ED0386A33F011F9EC
:10A0E0000346002B48D007F114030122F96A786A6D
:10A0F00023F0CCF903463B613B69002B56D03B690A
:10A1000018462EF035FEF861FB69002B2CDD07F1B7
:10A1100010030122B96A386A23F0B8F9B861B86946
:10A1200033F016F80346002B11D0B8692FF020FE4B
:10A13000034683F00103DBB2002B08D0012031F08D
:10A1400052FA03461A46294978682EF01BFDB86971
:10A1500030F060FF386B2FF0F7FC0246FB691344C8
:10A160001946386B2FF0E6FD3B69184630F052FF78
:10A17000012387F8373019E0786A33F0C2F80346D4
:10A1800083F00103DBB2002B03D01F49012028F02C
:10A1900055F9386A33F0B5F8034683F00103DBB2B2
:10A1A000002B03D01949012028F048F9396A786A50
:10A1B00030F05CFF97F8373083F00103DBB2002BFF
:10A1C00004D07A68B968F868FFF738FE7B691A46E8
:10A1D000B96AF86A30F058FF386B30F01BFF97F817
:10A1E000373018463837BD4680BD00BF208404088C
:10A1F000088404082C840408EC830408F48304080D
:10A200003884040800840408408404088484040812
:10A2100080B584B000AF0023FB730020FFF7F4FD8E
:10A22000B860BB68002B2FD03B46B96818462AF0AF
:10A2300081FE1BE03B461846FFF7B4FD78603B46C5
:10A240007A681946B868FFF7F3FE03461A46FB7BA7
:10A250001343DBB2002B14BF01230023FB73786888
:10A2600030F0D8FE3B4618462AF0B7FE3B4618466B
:10A27000FFF7ACFD0346002BDCD13B461846FFF749
:10A28000B6FDB86830F0C6FEFB7B18461037BD46F9
:10A2900080BD80B582B000AF0020FFF7B5FD7860CB
:10A2A0007B68002B05D078682EF0F4FA786830F0DF
:10A2B000B1FE0837BD4680BD80B586B000AF78607E
:10A2C000786833F077F8034683F00103DBB2002BA4
:10A2D0003FD10020FFF798FD78617B69002B38D0D3
:10A2E00007F10803796918462AF024FE21E007F1F6
:10A2F00008031846FFF756FD3861002216493869F1
:10A300002EF050FBF860FA687B689A4208D1002072
:10A3100031F069F903461A46104938692EF032FCCB
:10A320003969F86830F0A2FE07F1080318462AF0F0
:10A3300054FE07F108031846FFF748FD0346002BBB
:10A34000D5D107F108031846FFF751FD786930F0C1
:10A3500061FE1837BD4680BDF483040820840408DC
:10A3600080B586B000AF78603960786833F022F845
:10A37000034683F00103DBB2002B3DD10020FFF741
:10A3800043FD78617B69002B36D007F108037969BA
:10A3900018462AF0CFFD1FE007F108031846FFF723
:10A3A00001FD38610022396838692EF0FBFAF86047
:10A3B000FA687B689A4206D107F108033A691946A0
:10A3C0007869FFF73BFD3969F86830F04FFE07F117
:10A3D000080318462AF001FE07F108031846FFF7A4
:10A3E000F5FC0346002BD7D107F108031846FFF709
:10A3F000FEFC786930F00EFE1837BD4680BD0000C7
:10A4000080B582B000AF786003497868FFF7A8FF95
:10A410000837BD4680BD00BFEC83040880B582B01C
:10A4200000AF786003497868FFF79AFF0837BD46A8
:10A4300080BD00BFF4830408B0B58CB000AFF860F5
:10A44000B9607A60FB68002B00F0E980BB68002BE4
:10A4500000F0E5807349002022F058FE7862012068
:10A46000FFF7D2FC3862002031F0A8F8F8617B6A6F
:10A47000002B00F0CF803B6A002B00F0CB80FB6903
:10A48000002B00F0C78000226749F86826F08AFD9B
:10A49000B86100226549B86826F084FD7861B86922
:10A4A00032F02FFF0346002B00F0AC80786932F0C9
:10A4B00028FF0346002B00F0A0804023FB6201230D
:10A4C00087F82B30786832F075FF0346002B41D0B7
:10A4D0000022574978682EF065FA38613B69002BF5
:10A4E00007D03A695349786A2EF0D4FA386930F0C7
:10A4F00091FD0022504978682EF054FA38613B698A
:10A50000002B05D038692FF0E5FD034687F82B3086
:10A5100000224A4978682EF045FA38613B69002BE1
:10A5200026D0386932F0CCFE0346002B0AD03869B9
:10A530002FF00AFB0346002B04DD38692FF004FBE3
:10A54000F86203E03E49032027F078FF386930F0D5
:10A5500061FD0EE0786832F0D0FF034683F001031E
:10A56000DBB2002B05D03749032027F067FF00E05E
:10A5700000BF4FF40043344A3449F86802F086FEC5
:10A580000823334A3349B86802F080FE4FF4004391
:10A59000314A2E49B86802F079FEF86A31F00EF8B7
:10A5A00003461A462549786A2EF0ECFA97F82B30C4
:10A5B000184631F018F803461A461F49786A2EF0FB
:10A5C000E1FA264AF969786A2DF0C2FD0446244A68
:10A5D000F968786A2DF0BCFD0546224AB968786AA8
:10A5E0002DF0B6FD03461A462946204630F04CFDB4
:10A5F000796A386A2EF0BAFE08E01B49012027F07C
:10A600001DFF03E01949012027F018FF7969B86997
:10A6100030F02CFDFA69796A386A30F035FD303750
:10A62000BD46B0BDD0840408388404080084040802
:10A63000D8840408E0830408148404082C840408E3
:10A64000E48404080885040801A4000818840408A8
:10A65000B9A200084C8F04081DA40008088404084F
:10A66000EC830408F4830408348504089085040806
:10A6700080B582B000AF31F02DF87860304830F00E
:10A68000D1FE03461A462F4978682EF07BFA2E48F1
:10A6900030F0C8FE03461A462C4978682EF072FA4C
:10A6A0002B4830F0BFFE03461A462A4978682EF040
:10A6B00069FA4FF4002030F081FF03461A4626491C
:10A6C00078682EF05FFA4FF4C03030F077FF034621
:10A6D0001A46224978682EF055FA08F06FFE0346B4
:10A6E0001A461F4978682EF04DFA1FF06DFB03469D
:10A6F00018461BF059FB0346184630F093FE0346FC
:10A700001A46184978682EF03DFA16F041FE0346C5
:10A71000184630F087FE03461A46134978682EF033
:10A7200031FA124B184630F049FF03461A461049D9
:10A7300078682EF027FA7B6818460837BD4680BD3A
:10A74000E8850408F0850408E89F0408F8850408F3
:10A7500004860408148604081C8604082486040859
:10A76000288604083086040838860408D0000020B3
:10A770004086040890B58DB000AF0FF00DFDC7E91D
:10A7800008012DF047F8F8610FF006FDC7E9040154
:10A7900030F0A0FFF860FB68002B00F098800023E9
:10A7A000FB624D4B5B6800224C4918462EF0FAF8CC
:10A7B000B860BB68002B06D0B8682EF0D6FBF862F4
:10A7C000B86830F027FC33F0ADF90246FB6AD31AC3
:10A7D0007B6033F0E1F938603A687B68D31A184639
:10A7E00030F0ECFE03461A463D49F8682EF0CAF9EF
:10A7F0007B68184630F0E2FE03461A463949F8688D
:10A800002EF0C0F93B68184630F0D8FE03461A46D1
:10A810003549F8682EF0B6F9FB6A184630F0CEFEDE
:10A8200003461A462D49F8682EF0ACF9F86930F065
:10A83000C5FE03461A462D49F8682EF0A3F9D7E95C
:10A840000412D7E90834CB1A62EB040418462146F7
:10A850000FF078FC03460C461846214630F0DAFE2D
:10A8600003461A462249F8682EF08CF9214B184607
:10A8700030F0A4FE03461A461F49F8682EF082F90C
:10A880004FF0006030F09AFE03461A461B49F86804
:10A890002EF078F91A4B184630F090FE03461A460F
:10A8A0001849F8682EF06EF9174830F087FE034615
:10A8B0001A461649F8682EF065F94FF4002030F07A
:10A8C0007DFE03461A461249F8682EF05BF9FB68D4
:10A8D00018463437BD4690BD5851012048860408BB
:10A8E00050860408588604086086040868860408B0
:10A8F0006C860408D05701207486040884860408F6
:10A9000090DB04089086040800000608A48604086A
:10A91000B886040880B582B000AF78607B681B6899
:10A92000002B01D1002305E07B681B6818462FF03F
:10A93000CFFF034618460837BD4680BD80B483B0BC
:10A9400000AF78607B681B68002B14BF01230023D5
:10A95000DBB218460C37BD465DF8047B704780B506
:10A9600082B000AF78607B681B68184630F052FBFD
:10A970000837BD4680BD000080B584B000AF786068
:10A98000786822F049FCF860FB68002B06D0FB6871
:10A990001B68094A934201D1012300E00023FB72A6
:10A9A000FB7A03F00103FB72F86830F033FBFB7AAB
:10A9B00018461037BD4680BD0DAE000880B58EB07C
:10A9C00000AFF860B9607A6000237B63786832F08A
:10A9D00012FD0346002B3AD007F11403796818469C
:10A9E0002AF0A8FA012387F8333022E007F1140394
:10A9F0001846FFF78FFFF86207F108030122F96894
:10AA0000F86A22F043FDB86297F83330002B05D086
:10AA1000002387F83330BB6A7B6302E0B86A30F00A
:10AA2000F9FAF86A30F0F6FA07F1140318462AF03A
:10AA3000D4FA07F114031846FFF780FF0346002BF2
:10AA4000D4D107F114031846FFF789FF0AE07B68A9
:10AA5000002B07D007F108030122F968786822F07B
:10AA600015FD78633049F8682EF09EF82F49F86894
:10AA70002EF09AF800222E49F8682DF093FF7862A4
:10AA80002B49F8682EF090F825F012F838623B6AEE
:10AA9000002B09D0396A786A00F016F97A6A796B66
:10AAA000386A30F0F1FA3BE07B6A002B34D0786BE7
:10AAB000FFF762FF0346002B2AD048F208011D4829
:10AAC00030F03DFEF86148F208011B4830F037FED7
:10AAD000B861FB69002B16D0BB69002B13D07A6AD2
:10AAE0001649F8692DF0D6FF7A6A1449B8692DF035
:10AAF000D1FF0122F969786B00F0F2FA0022B969FE
:10AB0000786B00F0EDFAB969F86930F0AFFA03E05C
:10AB1000796B786A00F0A6F8796A786B30F0A6FA5B
:10AB20003837BD4680BD00BFC8860408D0860408FB
:10AB3000D886040865AC0008C9AC0008E0860408A3
:10AB400080B58AB000AFF860B9601346FB71FB793D
:10AB5000002B01D0364B00E0364BFB61002236491A
:10AB6000F8682DF01FFFB861BB69002B03D0B869EE
:10AB700030F050FA58E0012030F035FD03461A4617
:10AB80002D49F8682DF0FEFF0022F969F8682DF0D4
:10AB900009FF78627B6A002B27D100222749F868D9
:10ABA0002DF000FF38621DE00022F969386A2DF0AF
:10ABB000F9FE78627B6A002B09D07A6AB968386A34
:10ABC000FFF7FCFE396A786A30F050FA2CE0002278
:10ABD0001A49386A2DF0E6FE7861386A30F01AFAC0
:10ABE0007B693B623B6A002BDED1FB79002B04D0F2
:10ABF000BA681349F8682DF04DFF7B6A002B08D026
:10AC00007A6AB968F868FFF7D9FE786A30F002FA14
:10AC10000AE0FB7983F00103DBB2002B04D0BA68B1
:10AC20000849012027F00AFC2837BD4680BD00BF37
:10AC3000C8860408D0860408E8860408D886040874
:10AC4000F0860408FC86040880B582B000AF786006
:10AC50003960012239687868FFF772FF0837BD460E
:10AC600080BD000080B584B000AF7860396048F2E4
:10AC700008010C4830F063FDF860FB68002B0DD034
:10AC80007A680949F8682DF005FF3A460123F9680A
:10AC900078681DF02BF8F86830F0BCF91037BD4625
:10ACA00080BD00BF49AC0008E086040880B582B0D2
:10ACB00000AF78603960002239687868FFF740FF9C
:10ACC0000837BD4680BD000080B584B000AF786015
:10ACD000396048F208010C4830F031FDF860FB683B
:10ACE000002B0DD07A680949F8682DF0D3FE3A465A
:10ACF0000123F96878681CF0F9FFF86830F08AF9E8
:10AD00001037BD4680BD00BFADAC0008E08604082A
:10AD100080B586B000AFF860B9607A60002218494B
:10AD2000F8682DF03FFE034618462FF0B9F9786118
:10AD300000221449F8682DF035FE38613B69002B7C
:10AD40001AD07A68B96838692EF0D0F97B69013B6E
:10AD50007B61786930F032FC03461A460849F8688E
:10AD60002DF010FF7B69002B03D13969F868FFF7DC
:10AD700079FF386930F04EF91837BD4680BD00BF05
:10AD80001C8704082487040880B584B000AF78606D
:10AD9000396000220A4978682DF004FEF860FB68EB
:10ADA000002B0AD0F86830F035F9054978682DF0A5
:10ADB000FBFE39687868FFF787FF1037BD4680BD16
:10ADC0002487040880B500AF0349002022F09EF9D3
:10ADD0000346184680BD00BF2C87040880B582B0AA
:10ADE00000AF7860396039687868FFF73BFF083753
:10ADF000BD4680BD80B582B000AF786039603968EB
:10AE00007868FFF761FF0837BD4680BD80B58AB01E
:10AE100002AF7860FFF7D6FFF861FB69002B4AD0DC
:10AE200048F20801264830F08AFC0346FB6048F2ED
:10AE30000801244830F083FC03463B61FB68002B8B
:10AE400005D0FB68FA69204918462DF023FE3B69BE
:10AE5000002B05D03B69FA691B4918462DF01AFEF4
:10AE60001A4B1B8E7B837B68002B0ED007F10C03E3
:10AE70000193022300930023FA690021786825F0EA
:10AE800023F90346184630F0C5F8104A7B8B138629
:10AE900007F10C031946022030F01EF924F008FED9
:10AEA00078617B69002B06D07969F869FFF70CFFA0
:10AEB000786930F0AFF8FB6918462037BD4680BD91
:10AEC00065AC0008C9AC0008E086040858510120B0
:10AED00080B58CB000AF7860786832F076FC0346BD
:10AEE00083F00103DBB2002B06D07A6849490320C6
:10AEF00027F0A4FA002388E04749002022F006F951
:10AF000078627B6A002B01D100237EE048F20801C1
:10AF1000424830F014FC38623B6A002B71D07A6AE8
:10AF20003F49386A2DF0B6FD30F0DCFBF8610023B4
:10AF3000FB620023BB6207F10C037968184629F015
:10AF4000F9FF40E007F10C031846FFF7E3FCB86196
:10AF5000B869FFF711FD0346002B21D048F26001CC
:10AF6000304830F0ECFB7861F86A30F027FB38614C
:10AF70003A690021786930F0FBFD386930F04AF811
:10AF80007A6A274978692DF085FD3A6A7969B86946
:10AF900000F03EF903467969184630F067F807E09B
:10AFA000BA69F96AF8692EF0A1F8BB6A0133BB628D
:10AFB000B86930F02FF8FB6A0133FB6207F10C032C
:10AFC00018462AF00AF807F10C031846FFF7B6FCFA
:10AFD0000346002BB6D107F10C031846FFF7BFFC60
:10AFE000FA6ABB6AD31A184630F0E8FA03461A46E2
:10AFF0000D49786A2DF0C6FDFA690C49786A2DF082
:10B00000C1FD386A30F006F87B6A18463037BD4615
:10B0100080BD00BF348704082C87040889AD000870
:10B02000E086040811AD00081C8704082487040882
:10B0300080B584B000AF78600023FB607868FFF7CC
:10B040009BFC0346002B04D0786833F007FA0346D4
:10B050002AE0786832F0AEF90346002B17D00022C0
:10B06000134978682DF09EFCB860B86832F049F951
:10B070000346002B03D0B868FFF7C8FEF860B86835
:10B080002FF0C8FFFB68002B01D0FB680CE0FFF736
:10B0900099FEF860FB68002B01D1002304E0796879
:10B0A000F868FFF79BFEFB6818461037BD4680BD69
:10B0B0005C87040880B584B000AF7860FFF782FE3B
:10B0C000F860FB68002B01D1002304E07968F86880
:10B0D000FFF790FEFB6818461037BD4680BD0000A4
:10B0E00080B58AB000AFF860B9601346FB71B868EC
:10B0F00032F007F9034683F00103DBB2002B05D0E1
:10B10000BA682F49032027F099F955E0FB79002B05
:10B110001BD000222B49F8682DF04EF903463B6105
:10B120003B69002B11D03B6918462FF02DFC0346DC
:10B130003B6107F110020123B96800201CF0D6FD25
:10B140003B6918462FF066FF36E0FB79002B01D0F3
:10B150001D4B00E01D4B7B620022796AF8682DF0E0
:10B1600021FC38623B6A002B05D1BA68796AF8681D
:10B170002DF090FC20E0386A32F03DF90346002BB8
:10B1800004D0B968386A2EF0F1F812E03B6A7B61AE
:10B19000BB68BB6107F114030221184630F0AAFA1C
:10B1A000F861FA69796AF8682DF074FCF8692FF093
:10B1B00031FF386A2FF02EFF2837BD4680BD00BF13
:10B1C00064870408F0860408C8860408D08604084A
:10B1D00080B584B000AF786000220B4978682DF00C
:10B1E000E1FBF860FB68002B09D10849002021F041
:10B1F0008DFFF860FA68044978682DF04BFCFB6815
:10B2000018461037BD4680BDD88604082C87040830
:10B2100080B584B000AFF860B9607A600122B96887
:10B22000F868FFF75DFF7B68002B04D00022796887
:10B23000F868FFF755FFF868FFF7CAFF034618469E
:10B240001037BD4680BD80B582B000AF78603960F0
:10B25000002239687868FFF743FF7868FFF7B8FF86
:10B26000034618460837BD4680BD80B483B000AFA2
:10B270000346FB71FB79402B06D9FB795A2B03D887
:10B28000FB792033DBB200E0FB7918460C37BD4672
:10B290005DF8047B704780B483B000AF78607B6852
:10B2A0001B69002B01D1002305E07B681A697B68CC
:10B2B0001B6813441B7818460C37BD465DF8047BA9
:10B2C000704780B483B000AF78607B681A687B6891
:10B2D0005B689A4234BF01230023DBB218460C3767
:10B2E000BD465DF8047B704780B483B000AF7860E2
:10B2F0007B689A687B681B68134418460C37BD4608
:10B300005DF8047B704780B582B000AF78607B68E1
:10B31000DB6818462FF07EFE0837BD4680BD000072
:10B3200084B080B586B000AF786007F1240080E873
:10B330000E0030F0D7F938617868FFF7D5FFF86074
:10B34000786AB96ABB6AFA68D31A1A462EF0ECF921
:10B35000B860BA68002138692DF0C8FEB8682FF0CF
:10B3600059FE00237B6127E0786A7B6904339B00E8
:10B3700007F12002134459687B690C339B0007F1E5
:10B38000200213449A687B6904339B0007F1200E66
:10B3900073445B68D31A1A462EF0C6F9B8607B690D
:10B3A0000133BA68194638692DF0A0FEB8682FF04D
:10B3B00031FE7B6901337B613A6B7B699A42D3DC56
:10B3C000BB6A184630F0FAF803461A46084938694D
:10B3D0002DF0D8FB7B6A1A46064938692DF05AFBD6
:10B3E0003B6918461837BD46BDE8804004B0704739
:10B3F000748304087C830408B0B5BAB014AFF86055
:10B40000B9607A60FB70BB68FB637B683B64FB7868
:10B4100087F84430002387F845304FF48073A7F84D
:10B4200046300023BB6407F128037A68B9681846E0
:10B4300029F052FBFB681B785E2B1BD1FB685C1C60
:10B4400007F12805684607F144035022194638F0F1
:10B45000F6FC07F13C030CCB2946204600F016FA17
:10B46000C7F8940007F128031846FFF74CFFD7F8F8
:10B47000943051E007F12804684607F14403502254
:10B48000194638F0DCFC07F13C030CCB2146F86888
:10B4900000F0FCF9C7F8940007F12803184629F0DA
:10B4A0002DFC26E03B6C01333B6407F1140307F1EC
:10B4B00028021146184629F0B5FB07F11404684626
:10B4C00007F144035022194638F0B9FC07F13C0358
:10B4D0000CCB2146F86800F0D9F9C7F8940007F1C1
:10B4E00014031846FFF70FFF07F12803184629F049
:10B4F00005FCD7F89430002B07D107F12803184634
:10B50000FFF7DFFE0346002BCCD107F128031846D6
:10B51000FFF7F9FED7F8943018469837BD46B0BD0E
:10B5200090B589B000AFF860B9607A603B607B6825
:10B5300001221A60B868FFF7AEFE0346FB77FB688E
:10B540001B782E2B01D1012399E1FB681B785B2B23
:10B550005ED13B6801225A72FB6801331B785E2B77
:10B560000CBF01230023FB76FB7E002B04D07B68FD
:10B570001B685A1C7B681A600023BB771AE07B6843
:10B580001B681A46FB68981807F110023B68B968F7
:10B59000FFF7C6FF03461A46BB7F1343DBB2002BFF
:10B5A00014BF01230023BB777B681A683B691A44E8
:10B5B0007B681A607B681B681A46FB6813441B781B
:10B5C000002B07D07B681B681A46FB6813441B7866
:10B5D0005D2BD4D17B681B681A46FB6813441B782B
:10B5E0005D2B0FD17B681B685A1C7B681A603B6817
:10B5F00000225A72BA7FFB7E9A4214BF01230023B5
:10B60000DBB23CE1A049012026F018FF002336E11F
:10B61000FB681B787B777B7F5C2B40F0C4807B686A
:10B6200002221A60FB685B787B777B7F642B05D1F5
:10B63000FB7F184626F031FC034620E17B7F442B3C
:10B6400010D1FB7F184626F028FC0346002B14BFC0
:10B6500001230023DBB283F00103DBB203F001031B
:10B66000DBB20CE17B7F662B02D10C237B779AE067
:10B670007B7F6E2B02D10A237B7794E07B7F722B3A
:10B6800002D10D237B778EE07B7F732B05D1FB7F6F
:10B69000184626F0DFFB0346F1E07B7F532B10D1E9
:10B6A000FB7F184626F0D6FB0346002B14BF012370
:10B6B0000023DBB283F00103DBB203F00103DBB252
:10B6C000DDE07B7F742B02D109237B776BE07B7FEE
:10B6D000762B02D10B237B7765E07B7F772B17D10D
:10B6E000FB7F184626F0D9FB0346002B09D1FB7FD0
:10B6F000184626F00CFC0346002B02D1FB7F5F2B83
:10B7000001D1012300E0002303F00103DBB2B6E026
:10B710007B7F572B1DD1FB7F184626F0BEFB0346CF
:10B7200083F00103DBB2002B0ED0FB7F184626F01E
:10B73000EEFB034683F00103DBB2002B04D0FB7F5A
:10B740005F2B01D0012300E0002303F00103DBB2F3
:10B7500095E07B7F302B02D100237B7723E07B7F3A
:10B76000782B20D1FB6802331B78002B1BD0FB68A1
:10B7700003331B78002B16D07B6804221A60FB6809
:10B7800002331B78184626F046FD03461B015CB2C7
:10B79000FB6803331B78184626F03DFD03465BB279
:10B7A00023435BB27B773B685B7A002B25D07B68B9
:10B7B0001B681A46FB6813441B782D2B1DD17B7F19
:10B7C0001AB23B685A817B681B685A1C7B681A60F6
:10B7D0007B681B681A46FB68981807F114023B68DF
:10B7E000B968FFF79DFE0346BB767B681A687B69E4
:10B7F0001A447B681A60BB7E41E03B681B7A002BD1
:10B800000BD0FB7F1846FFF730FD0346FB777B7FAD
:10B810001846FFF72AFD03467B773B68B3F90A30E9
:10B82000B3F5807F24D03B68B3F90A303B773B689F
:10B830001B7A002B05D03B7F1846FFF716FD034609
:10B840003B773B684FF480725A81FA7F3B7F9A4284
:10B8500009D3FA7F7B7F9A4205D83A7F7B7F9A4251
:10B8600001D2012300E0002303F00103DBB206E074
:10B870007A7FFB7F9A420CBF01230023DBB218467C
:10B880002437BD4690BD00BF8887040882B0B0B59C
:10B89000A8B014AFF861B96107F1600181E80C004C
:10B8A00028F0F2F80346002B01D0002367E1FB6982
:10B8B0001B78002B0ED1684607F16C034C22194609
:10B8C00038F0BDFA07F160030ECBB869FFF728FD29
:10B8D000034654E1FB691B78282B38D1FC6EB8690C
:10B8E000FFF702FD0246231D07F1600141F8232006
:10B8F000FB6EFA6E043207F1600151F822200C331E
:10B900009B0007F160010B445A60FB6E082B02DCC0
:10B91000FB6E0133FB6628F01DFB034683F0010339
:10B92000DBB2002B01D0002329E1FB695C1C6846D7
:10B9300007F168035022194638F081FA07F16003D5
:10B940000CCBB9692046FFF7A1FF034617E1FB695D
:10B950001B78292B2BD1FB6E002B0CDDFB6E5C1EA4
:10B96000B869FFF7C1FC024604F10C039B0007F124
:10B9700060010B445A6028F0EDFA034683F001039E
:10B98000DBB2002B01D00023F9E0FB695C1C6846A8
:10B9900007F168035022194638F051FA07F16003A5
:10B9A0000CCBB9692046FFF771FF0346E7E007F1CA
:10B9B000380207F16003B969F869FFF7B1FD034682
:10B9C00087F84F30BB6B1A46FB6913441B782A2B50
:10B9D00006D0BB6B1A46FB6913441B782B2B7FD117
:10B9E000BB6B1A46FB6913441B7887F8473097F8FE
:10B9F0004F3083F00103DBB2002B05D097F84730BE
:10BA00002B2B01D10023BAE0BB6B0133FA6913443D
:10BA10003B643B46B969184629F004F907F1240450
:10BA20003D460FCD0FC42B68236007F12404684600
:10BA300007F168035022194638F001FA07F1600354
:10BA40000CCB2146386CFFF721FFB86407F12403C3
:10BA50001846FFF758FC37E0B86929F04FF907F1AD
:10BA6000380207F16003B969F869FFF759FD034629
:10BA700087F84F303B46B969184629F0D3F807F1EB
:10BA800024043D460FCD0FC42B68236007F1240426
:10BA9000684607F168035022194638F0D0F907F1DB
:10BAA00060030CCB2146386CFFF7F0FEF86307F11A
:10BAB00024031846FFF727FCFB6B002B04D0B86C5F
:10BAC0002FF0A8FAFB6BBB64B869FFF7FAFB0346DB
:10BAD000002B03D097F84F30002BBDD1BB6C4EE04C
:10BAE000FB691B78242B1ED1FB6901331B78002BCB
:10BAF00019D1B869FFF7E5FB034683F00103DBB218
:10BB0000002B0ED0684607F16C034C22194638F022
:10BB100096F907F160030ECBB869FFF701FC034605
:10BB20002DE000232BE0B869FFF7CBFB0346002B89
:10BB300024D097F84F30002B20D0B86929F0DEF8D8
:10BB400028F008FA034683F00103DBB2002B01D092
:10BB5000002314E0BB6B1A46FB699C18684607F18A
:10BB600068035022194638F06AF907F160030CCBDC
:10BB7000B9692046FFF78AFE034600E00023184615
:10BB80005037BD46BDE8B04002B0704780B584B0C4
:10BB900000AF78603960786831F0FBFA034683F0D3
:10BBA0000103DBB2002B06D07A681D49032026F082
:10BBB00045FC002330E01B49002021F0A7FAF86083
:10BBC0007A681949F8682CF065FF386831F095FCFF
:10BBD000034683F00103DBB2002B13D0386831F049
:10BBE000D8FA034683F00103DBB2002B05D07A6854
:10BBF0000B49032026F022FC04E03A680B49F86860
:10BC00002CF048FF00202FF0D9FC03461A460849C3
:10BC1000F8682CF0B7FFFB6818461037BD4680BDAA
:10BC2000AC87040860830408EC8304088881040856
:10BC30006883040890B58BB000AF786039603868CD
:10BC400030F05AFBF8610022454978682CF0AAFED2
:10BC5000034618462EF024FA78620022414978689B
:10BC60002CF0A0FEB861B86931F093FA034683F076
:10BC70000103DBB2002B05D0B969F8692FF0F6F9A2
:10BC8000002368E0B86930F010FD78617B6901330A
:10BC900007330733DB08DB00ADEB030D6B460733DF
:10BCA000DB08DB003B613B69002B05D1B969F86912
:10BCB0002FF0DCF900234EE07B6901331A46396925
:10BCC000B86930F0B1F9B8692FF0A4F97C6A69213C
:10BCD0007868FBF7F9F903462246F9693869FFF7F6
:10BCE0008BFB3862F8692FF095F93B6A002B06D17F
:10BCF000022032F049F9386200237B6221E067219B
:10BD00007868FBF7E1F90346002B18D00021386A68
:10BD10002DF0DAF9F86000221349386A2CF042FE5F
:10BD2000034618462EF0BCF90446F86830F0BDFC16
:10BD3000034623447B62F8682FF06CF901E000238E
:10BD40007B62786A2FF03AFC03461A460449786809
:10BD50002CF018FF3B6A18462C37BD4690BD00BF3B
:10BD600068830408EC8304087483040880B58CB0ED
:10BD700002AFF860B9603B601346FB80B86831F0F1
:10BD800008FA034683F00103DBB2002B05D0114A09
:10BD90004FF4F771104826F0C5FB07F11403002299
:10BDA000B968184628F098FE07F11403184628F0E1
:10BDB000AFFFF98807F114030093084B3A68F8685D
:10BDC00003F0C0FF07F11403184603F0B4FA283754
:10BDD000BD4680BDD8870408EC8704088D9503080C
:10BDE00080B584B000AFF860B9601346FB80FA8874
:10BDF0000023B968F868FFF7B9FF1037BD4680BD6A
:10BE000080B584B002AF78600B467B8079880023D0
:10BE10000093044B0022786803F094FF0837BD4676
:10BE200080BD00BF059E020880B582B000AF78607B
:10BE30007B681B68002B01D1002305E07B681B6831
:10BE4000184632F00BFB034618460837BD4680BD46
:10BE500080B483B000AF78607B681B68002B14BF90
:10BE600001230023DBB218460C37BD465DF8047B86
:10BE7000704780B582B000AF78607B681B68184659
:10BE80002FF0C8F80837BD4680BD000080B500AF70
:10BE9000044B5B680522044918462CF083FD0346D9
:10BEA000184680BD585101200088040880B5A8B00C
:10BEB00000AF7860786831F06CF9034683F00103D5
:10BEC000DBB2002B06D07A684D49032026F0B6FA83
:10BED000002391E007F1080380221946786830F0CA
:10BEE000A3F803467F2B05D94649032026F0A6FA7E
:10BEF000002381E0FFF7CAFFC7F89800D7F8983011
:10BF0000002B01D1002377E007F108030022194636
:10BF1000D7F898002CF050FA034618462EF034FD5E
:10BF2000C7F89C00D7F898002FF074F8D7F89C3029
:10BF3000002B02D0D7F89C305EE007F108031846CA
:10BF400015F016F8C7F89400D7F89430002B07D0F6
:10BF5000D7F89430002118462FF0F1FBC7F89C0069
:10BF6000D7F89C30002B24D107F10803184615F0B0
:10BF700004FAC7F89000D7F89030002B19D0D7F802
:10BF80009000F4F7DBFF03461946D7F890002FF036
:10BF9000F0FBC7F88C00D7F88C30002B09D0D7F80D
:10BFA0008C0021F0CDFAC7F89C00D7F88C002FF058
:10BFB00031F8D7F89C30002B15D0FFF767FFC7F892
:10BFC0008800D7F88830002B08D007F10803D7F88D
:10BFD0009C201946D7F888002CF05CFDD7F8880023
:10BFE0002FF018F806E007F108031A460649012069
:10BFF00026F024FAD7F89C301846A037BD4680BDFD
:10C0000008880408388804086088040880B586B069
:10C0100000AF2FF067FB78617B69002B01D1002313
:10C0200032E0FFF733FF38613B69002B01D17B69B8
:10C030002AE03B1D3969184628F07CFF15E03B1DBE
:10C040001846FFF7F1FEF86000220021F8682EF094
:10C050006FFEB860B968786929F052FEF8682EF072
:10C06000D9FF3B1D184628F0B8FF3B1D1846FFF7C7
:10C07000EFFE0346002BE2D13B1D1846FFF7F9FE09
:10C0800038692EF0C7FF7B6918461837BD4680BD5A
:10C0900080B584B000AF7860786831F07AF80346F4
:10C0A00083F00103DBB2002B04D01349012026F0FA
:10C0B000C5F91EE0FFF7EAFEF860FB68002B18D018
:10C0C00000227968F8682CF0C7FAB860BB68002BCA
:10C0D00005D17A680949012026F0B0F906E0B9686F
:10C0E000F8682CF0F5FAB8682EF094FFF8682EF096
:10C0F00091FF1037BD4680BD74880408A4880408E9
:10C1000080B582B000AFFFF7C1FE78607B68002B7E
:10C1100005D078682CF0BEFB78682EF07BFF0837DE
:10C12000BD4680BD80B584B000AF78603960786866
:10C1300031F02FF8034683F00103DBB2002B11D15D
:10C14000386831F026F8034683F00103DBB2002B98
:10C150000DD0386831F0D5F8034683F00103DBB227
:10C16000002B04D01249012026F068F91DE0FFF7EA
:10C170008DFEF860FB68002B17D0386821F0E0F9DD
:10C18000B860BB68002B05D17A680A49012026F007
:10C1900055F907E0BA687968F8682CF0B7FCB86818
:10C1A0002EF038FFF8682EF035FF1037BD4680BD01
:10C1B000B8880408E888040880B584B000AF7860C7
:10C1C00078681CF00DFF0346FB73FB7B184621F0DB
:10C1D00075FA034683F00103DBB2002B01D0002384
:10C1E00004E0FB7B18462FF058FA03461846103738
:10C1F000BD4680BD80B584B000AF786078681CF023
:10C20000EFFE0346FB73FB7B18461CF07BFF0346E7
:10C2100018461037BD4680BD80B584B000AF786049
:10C2200078681CF0DDFE0346FB73FB7B012118469A
:10C230001CF098FF1037BD4680BD80B584B000AFBC
:10C24000786078681CF0CCFE0346FB73FB7B002112
:10C2500018461CF087FF1037BD4680BD80B584B0FE
:10C2600000AF78600B46FB7078681CF0B9FE03469F
:10C27000FB73FA78FB7B114618461CF073FF1037EE
:10C28000BD4680BD90B58BB002AFF860C7E9002312
:10C290000B46FB72F8681CF0A3FE0346FB754FF0DB
:10C2A00000020C4BD7E90001F4F732F903460C46C3
:10C2B000184621460DF01CFFC7E90601FB7A07F17D
:10C2C000170200930123D7E9060115F021FF243757
:10C2D000BD4690BD00408F4080B582B000AF786011
:10C2E00078681CF07DFE0346184602F091FB034679
:10C2F00018460837BD4680BD80B582B000AF786073
:10C30000396078681CF06CFE0346002239681846D4
:10C3100002F0B4FA0837BD4680BD80B584B000AFE6
:10C32000786078681CF05CFE0346FB73FB7B184664
:10C3300021F0C4F9034683F00103DBB2002B01D0E6
:10C34000002312E0FB7B18460DF0A2FB034603F02E
:10C350001003002B0CBF01230023BB73BA7BFB7BB4
:10C36000114618461CF0FEFEBB7B18461037BD4632
:10C3700080BD000080B592B000AF786078681CF096
:10C380002FFE034687F83F3097F83F30184621F0DC
:10C3900095F9034683F00103DBB2002B01D00023A3
:10C3A000F7E097F83F2013469B0013445B001344CB
:10C3B0007A4A1344BB632FF08DF978637B6B002BB3
:10C3C00001D10023E5E0BB6B1B784033DBB23B7748
:10C3D00000237B7707F11C0318462FF023F8034650
:10C3E0001A466F49786B2CF0CDFBBB6B5B78184617
:10C3F0002FF0E4F803461A466A49786B2CF0C2FB2A
:10C4000097F83F30002118460AF00AFC38633B6B6E
:10C41000002B09D03B6B18462FF0D0F803461A4684
:10C420006149786B2CF0AEFB97F83F30012118463C
:10C430000AF0F6FB38633B6B002B09D03B6B1846C8
:10C440002FF0BCF803461A465849786B2CF09AFB3B
:10C45000BB6B9B78002B3AD02FF03CF9F862FB6A5B
:10C46000002B34D02FF03EF9B862BB6A002B21D0EC
:10C4700000237B6416E0BB6B9B78194620227B6C03
:10C4800002FA03F30B40002B09D07B6C01331846F2
:10C490002FF094F803461946B86A29F031FC7B6CFA
:10C4A00001337B647B6C002BE5DDBA6A4049F86A96
:10C4B0002CF068FBBB6B9B7803F01F0318462FF032
:10C4C0007DF803461A463B49786B2CF05BFB2FF056
:10C4D00001F978627B6A002B5AD000233B644FE05D
:10C4E000BA6B3B6C5B001344B3F803309BB2002B78
:10C4F00043D02FF0EFF838623B6A002B3DD0BA6B87
:10C500003B6C5B001344B3F8033098B207F10C02A4
:10C51000102308211CF0B8FF07F10C0318462EF079
:10C5200081FF03461A462449386A2CF02BFBBA6B6C
:10C530003B6C5B001344B3F803309BB203F00F0372
:10C5400018462FF03BF803461A461C49386A2CF06F
:10C5500019FBBA6B3B6C5B001344B3F8033098B221
:10C5600007F10C02102303211CF08EFF07F10C03CE
:10C570003A6A1946786A2CF005FB3B6C01333B6440
:10C580003B6C032BACDD7A6A0D49786B2CF0FAFA20
:10C590007B6B18464837BD4680BD00BFD87804087D
:10C5A000807B0408048904080889040810890408A9
:10C5B0001C890408248904082C8904083489040887
:10C5C0003889040880B586B000AF786078682CF0B0
:10C5D00089FB0346002B04D100202EF0EFFF034619
:10C5E00076E0002178682CF06FFD386100237B61D4
:10C5F000386930F000FF0346002B35D038692CF045
:10C6000071FBF860FB68002B04D100202EF0D6FFF0
:10C6100078614EE0FB68012B4BD1002138692CF08A
:10C6200053FDB860B86830F0B4FD0346002B0AD063
:10C63000B86830F01EF80346002B04D000202EF01E
:10C64000BDFF78610CE0B86830F082FD034683F0EE
:10C650000103DBB2002B03D0B8682DF09DFC78619C
:10C66000B8682EF0D7FC25E0386930F046FF034665
:10C67000002B05D1386930F09DFE0346002B02D017
:10C6800000237B6116E0386930F083FD0346002B00
:10C690000AD038692FF0EDFF0346002B04D00020AC
:10C6A0002EF08CFF786105E038692DF075FC78611B
:10C6B00000E000BF38692EF0ADFC7B69002B01D093
:10C6C0007B6905E04FF0000003492EF0A3FF03460D
:10C6D00018461837BD4680BD0000F87F80B596B07B
:10C6E00002AF786039603B68002B01DA00233B60C1
:10C6F0003B68142B01DD14233B6078682DF09AFB16
:10C7000007F108023B6801930A230093462326F0B1
:10C710000FF907F1080318462EF084FE0346184669
:10C720005037BD4680BD80B584B000AFF860B960B9
:10C730007A607B680122B968F86826F0A7F810379C
:10C74000BD4680BD80B582B000AF78607B681B6855
:10C75000002B01D1002305E07B681B68184631F0EF
:10C760007DFE034618460837BD4680BD80B582B0C1
:10C7700000AF78607B681B68002B01D1002305E0C7
:10C780007B681B6818462EF0A3F803461846083746
:10C79000BD4680BD80B483B000AF78607B681B6805
:10C7A000002B14BF01230023DBB218460C37BD4613
:10C7B0005DF8047B704780B582B000AF78607B681D
:10C7C0001B6818462EF026FC0837BD4680BD80B594
:10C7D00088B002AF78607B68184630F0EBFD034606
:10C7E000002B0DD17B68184630F005FE0346002B68
:10C7F00006D17B68184630F084FD0346002B05D037
:10C800007B68184631F02AFE034629E07B6818460B
:10C8100014F012FC78617B69002B04D0786924F055
:10C82000EDFA034600E000233B613B69002B03D196
:10C830002EF050FF034613E038692EF049F8F860F7
:10C840003B1D019301230093002300223969F868FE
:10C8500023F03AFCB860F96838692EF007FCBB6831
:10C8600018461837BD4680BD80B584B000AF7860EB
:10C87000786830F0C0FD0346002B04D078682CF0B7
:10C8800031FAF8602BE0786830F0CFFD0346002BDA
:10C8900005D078682DF0D6FD0346FB601FE0786870
:10C8A00030F077FC0346002B05D078682FF0FDFEB2
:10C8B0000346FB6013E0786830F023FD0346002B4D
:10C8C0000BD078682DF07AFEB860B8682CF00AFAC0
:10C8D000F860B8682EF09EFB01E0002303E0F868E2
:10C8E0002EF06CFE034618461037BD4680BD000092
:10C8F00080B582B000AF78607B68002B06D17A6883
:10C900000649032025F09AFD002303E0786831F002
:10C91000A5FD034618460837BD4680BD4489040876
:10C9200080B598B002AF78603960386830F0C0FBED
:10C930000346002B33D0786830F0C2FC0346002B4E
:10C940002DD038682DF000F978657B6D012B26DD40
:10C950007B6D242B23DC786830F0AAFB0346002B88
:10C9600009D078682DF0F0F87A6D07F10C031946BC
:10C97000FFF7D9FE0CE078682DF05CFA07F10C02A5
:10C980004FF0FF3301937B6D0093462325F0D0FFDA
:10C9900007F10C0318462EF045FD034603E07868C6
:10C9A0002FF0AAFC034618465837BD4680BD80B517
:10C9B00082B000AF7860012178682BF059F9034606
:10C9C00018460837BD4680BD80B588B000AFF86016
:10C9D000B9607A60FB68002B25D0FB681B7AFB7678
:10C9E0000023FB611BE0FB681A68FB69DB00134452
:10C9F0001A785B781B0213433B83FB685A683B8BB6
:10CA0000134418462EF00EFD7861BB68796978688A
:10CA1000984778692EF0FEFAFB690133FB61FA7ED4
:10CA2000FB699A42DFD82037BD4680BD80B5A0B0F3
:10CA300000AFF8607B600B46FB721346BB72F86870
:10CA400030F0C3FE0346002B4ED0F86827F0EAFB17
:10CA5000786707F110030022F968184628F048FFAC
:10CA600035E007F11003184628F0B2FF38677B6FF6
:10CA7000002B0FD07B6F386F9847034683F001037C
:10CA8000DBB2002B06D17649386F2EF03FF8034613
:10CA9000002B14D000220021386F2EF049F90346F4
:10CAA00018462FF0D6FDF866FB6E002B07D07B688A
:10CAB000F96ED7F888009847F86E2EF0ABFA386F09
:10CAC0002EF0A8FA07F11003184625F06DF807F1CB
:10CAD0001003184625F022F80346002BC1D107F1B8
:10CAE0001003184625F0B2F8FB7A002B00F08F8077
:10CAF000F86820F0B1FDB866BB6E002B0DD0B86EA3
:10CB000013F018FF7866B86E2EF084FAD7F88820F4
:10CB10007968786EFFF758FF18E0F86830F04AFC43
:10CB2000034683F00103DBB2002B05D1F86830F037
:10CB300071FA0346002B09D0F86813F0F7FC386649
:10CB4000D7F888207968386EFFF73EFFBB7A002B54
:10CB500045D0F86830F02EFC0346002B05D1F8686C
:10CB600030F0CFFB0346002B21D000223D49F8686E
:10CB70002BF018FFF86714E0F86F13F0DBFEF86590
:10CB8000D7F888207968F86DFFF71EFF0022354935
:10CB9000F86F2BF007FFB865F86F2EF03BFABB6D0E
:10CBA000FB67F86F30F006FC0346002BE4D1F86811
:10CBB00013F0C0FE7865D7F888207968786DFFF7A4
:10CBC00003FF002013F0B6FE38653A6D7B6D9A4284
:10CBD00005D0D7F888207968386DFFF7F5FEF8683A
:10CBE00030F009FC0346002B05D1F86830F0D1FA8B
:10CBF0000346002B0BD01C482EF014FCF8647B6815
:10CC0000F96CD7F888009847F86C2EF003FAF868AA
:10CC100030F000FA0346002B1ED00023BB6718E05B
:10CC2000BB6FDAB207F13C031146184620F0F4FD61
:10CC300007F13C0318462EF0F5FBB8647B68B96C2D
:10CC4000D7F888009847B86C2EF0E4F9BB6F013331
:10CC5000BB67BB6F312BE3DD8037BD4680BD00BFB6
:10CC6000608904086C8904087889040880B586B056
:10CC700002AF78600B46FB701346BB702EF032FD9E
:10CC8000F860FB68002B01D1002308E0BA78F9783E
:10CC9000FB680093044B7868FFF7C8FEFB681846F2
:10CCA0001037BD4680BD00BF9D5F030880B584B0CE
:10CCB00000AF78603960786830F07CFB034683F021
:10CCC0000103DBB2002B0FD0786830F026FC03465E
:10CCD00083F00103DBB2002B06D07A6813490320EE
:10CCE00025F0ACFB00231DE0386830F063FB034601
:10CCF000002B03D00E49012025F0A0FB2EF0EAFC0A
:10CD0000F860FB68002B01D100230BE0786830F05D
:10CD100051FB0346002B04D07A680649F8682BF0D3
:10CD2000B9FEFB6818461037BD4680BD80890408EF
:10CD3000B48904086C89040880B588B000AF7860B5
:10CD400039603968786800F0B5F8034683F001036C
:10CD5000DBB2002B01D0002398E038682FF016FCDE
:10CD6000F8610122F969786824F066F9B861F86918
:10CD70002EF050F9BB69002B05D1464A4FF4AF7134
:10CD8000454825F0CFFBBB69002B01D100237DE096
:10CD90002EF0A0FC78617B69002B04D1B8692EF0DD
:10CDA00039F9002372E0B86930F06FFC0346FB7478
:10CDB000786827F037FAF86001202EF014FC03465B
:10CDC0001A46364978692BF0DDFEFB68002B08D047
:10CDD000FB68B8699847034683F00103DBB2002B78
:10CDE00001D0012300E0002303F00103DBB2184669
:10CDF0002EF0F9FB03461A46294978692BF0C2FE4A
:10CE0000FB7C002B14BF01230023DBB283F0010362
:10CE1000DBB203F00103DBB218462EF0E4FB03465D
:10CE20001A46204978692BF0ADFEB8692DF02AFC2E
:10CE3000B860B86830F04EFC0346002B16D00022D4
:10CE40001949B8682BF0AEFD03461A4616497869B1
:10CE50002BF098FE00221549B8682BF0A3FD03467D
:10CE60001A46124978692BF08DFE08E0B8692DF05A
:10CE70002FFD03461A460E4978692BF083FEB868E9
:10CE80002EF0C8F8B8692EF0C5F87B69184620372F
:10CE9000BD4680BDDC890408E4890408F8890408DB
:10CEA000048A0408108A0408208A0408248A0408D2
:10CEB000288A040880B590B000AF7860396038687F
:10CEC0002FF064FBB863002387F83F30786830F0B8
:10CED000CBFE0346002B0ED00022B96B78682BF0F6
:10CEE000BBFB78637B6B002B05D0012387F83F30B9
:10CEF000786B2EF08FF897F83F3083F00103DBB2A8
:10CF0000002B27D0786830F055FA034683F00103F0
:10CF1000DBB2002B1ED0786813F008FB38633B6B44
:10CF2000002B17D007F10C0320221946B86B2FF005
:10CF30007BF807F10C031A467968386B12F0E2FFB0
:10CF4000F862FB6A002B02D0012387F83F30F86AB1
:10CF50002EF060F8B86B2EF05DF897F83F30184669
:10CF60004037BD4680BD000080B588B000AFF86096
:10CF7000B9607A60F86830F01DFA034683F0010367
:10CF8000DBB2002B06D0FA683149012025F056FAB1
:10CF9000002358E0786830F00DFA034683F001036F
:10CFA000DBB2002B06D07A682A49012025F046FA28
:10CFB000002348E0B8682FF0E9FAB8610023FB616C
:10CFC0000022254978682BF0EDFC78610022234986
:10CFD00078682BF0E7FC38617B69002B02D13B6954
:10CFE000002B1AD0062030F0CFFFF861FB69002B30
:10CFF0000FD07B69002B04D07A691749F8692BF0B0
:10D0000049FD3B69002B04D03A691449F8692BF0BB
:10D0100041FD396978692EF029F8FB69002B05D1AB
:10D0200000220F4978682BF0BDFCF861FA69B969F4
:10D03000F8682BF06BFDF969B8692EF017F8F868FD
:10D0400031F00CFA034618462037BD4680BD00BFBC
:10D05000308A04085C8A0408208A0408248A0408A8
:10D06000288A040880B586B000AF78603960786897
:10D0700030F0A0F9034683F00103DBB2002B06D0A9
:10D080007A682749012025F0D9F9002343E0386860
:10D0900030F090F9034683F00103DBB2002B06D099
:10D0A0003A682049012025F0C9F9002333E007F14F
:10D0B0000C033968184627F03DFF1BE007F10C030D
:10D0C0001846FFF73FFB786107F10C031846FFF79E
:10D0D0004DFB38613A6979697868FFF745FF034687
:10D0E0003A69796918462DF0CFFF07F10C0318460D
:10D0F00027F073FF07F10C031846FFF74BFB0346BD
:10D10000002BDBD107F10C031846FFF754FB7868BE
:10D1100031F0A4F9034618461837BD4680BD00BF5C
:10D120008C8A0408B88A040880B582B000AF7860A1
:10D1300000220449786823F035FF03461846083773
:10D14000BD4680BD6C89040880B584B000AF7860AE
:10D150003960786830F02EF90346002B06D00122A2
:10D160001249786823F01EFF034600E00023FB60AD
:10D17000F86830F006FA034683F00103DBB2002BB7
:10D1800005D0FA680A49032025F058F903E0396808
:10D19000F8682BF015F8F8682DF03CFF78682DF052
:10D1A000F9FE034618461037BD4680BD6C89040859
:10D1B000E48A040880B586B000AF786000237B6104
:10D1C00007F108037968184627F0B4FE0023FB74C2
:10D1D00036E007F108031846FFF7C8FAF860F86868
:10D1E00030F08BF90346002B22D1F86830F095F926
:10D1F0000346002B1CD1F86830F0DCF8034683F0BE
:10D200000103DBB2002B07D0FA681949032025F08F
:10D2100015F90123FB740BE07B69002B04D1F8683E
:10D2200031F01CF9786103E0F96878692BF0D4FCDF
:10D23000F8682DF0EFFE07F10803184627F0CDFE41
:10D24000FB7C83F00103DBB2002B07D007F108035E
:10D250001846FFF79FFA0346002BBAD107F10803DF
:10D260001846FFF7A8FA7B6918461837BD4680BDF7
:10D27000F88A040880B582B000AF786078682CF036
:10D2800077FD034618460837BD4680BD80B586B099
:10D2900000AFF860B9607A607B80B8682EF0C2F8A1
:10D2A00078617B88194678682EF049FA38613A69C6
:10D2B0007969F86800F008F8796938692DF0D6FEC8
:10D2C0001837BD4680BD000080B58AB000AFF86059
:10D2D000B9607A60F86830F0C7FC034683F0010358
:10D2E000DBB2002B04D04949032025F0A7F889E0E0
:10D2F000B8682FF04EFF034683F00103DBB2002B2A
:10D3000004D04349032025F099F87BE078682FF09A
:10D31000F8FF034683F00103DBB2002B0DD07868E1
:10D320002FF037FF034683F00103DBB2002B04D05C
:10D330003849032025F082F864E0B96836482CF0BB
:10D3400063F978627B6A002B5CD00122796AF86805
:10D350002BF082F93862786A2DF05CFE386A2DF085
:10D36000B7FAF861F86930F0C8F80346002B04D02A
:10D370007968386A2AF024FF1CE0F86930F03BF83D
:10D380000346002B04D07968F8692BF0EFFF11E019
:10D390002EF0A8F9B861F969B8692BF0E7FF796850
:10D3A000B8692BF0E3FFB969386A2AF009FFB86958
:10D3B0002DF030FE396AF8692DF058FE1749B8682B
:10D3C0002DF0A4FB0346002B1CD000221449F86862
:10D3D0002BF0E8FA03467B617B6918462FF0D9FEF3
:10D3E0000346002B0AD007F1140201230D49F86807
:10D3F0001AF0D2FC0A49F8682BF0D6FB7B69184674
:10D400002DF008FE2837BD4680BD00BF148B0408F0
:10D410004C8B0408848B0408DC8B0408BC7804085B
:10D42000CC820408008304082DE9F0438DB000AFDE
:10D43000F860B9607A606B461E46F86830F014FCFC
:10D44000034683F00103DBB2002B04D04A490320DA
:10D4500024F0F4FF8AE0B8682FF09BFE034683F0C7
:10D460000103DBB2002B04D04449032024F0E6FF83
:10D470007CE0B96842482CF0C7F8B862BB6A002B60
:10D4800074D004237B627B6A013B3B627B6A1A4651
:10D490004FF000034FEA431949EAD2694FEA4218B4
:10D4A0007B6A1A464FF000035D0145EAD2655401DC
:10D4B0007B6A9B0003330733DB08DB00ADEB030D16
:10D4C0006B4603339B089B00FB610023FB6207F163
:10D4D00014037968184627F02DFD1AE0FA6A7B6A72
:10D4E0009A4205D37A6A2749032024F0A7FF18E05F
:10D4F000FC6A631CFB6207F114031846FFF736F958
:10D500000246FB6943F8242007F11403184627F06C
:10D5100064FD07F114031846FFF73CF90346002B9E
:10D52000DCD107F114031846FFF745F90022B96A68
:10D53000F8682BF091F8034618462DF025FAB861EB
:10D54000B86A2DF067FDBB69002B05D0FA69FB6A4C
:10D55000B969F8681AF0CAFBB8692DF05BFDFB6980
:10D560001946F86A2DF0B8FDB54600E0B5463437E7
:10D57000BD46BDE8F08300BF148B0408E48B0408AB
:10D58000DC8B0408208C040880B588B000AFF860FC
:10D59000B9607A60F86830F067FB034683F00103F6
:10D5A000DBB2002B04D02849032024F047FF47E0DA
:10D5B000B8682FF0EEFD0346002B3DD0B968234834
:10D5C0002CF022F8F861FB69002B39D00122F969AF
:10D5D000F8682BF041F8B861F8692DF01BFDB869C7
:10D5E0002DF076F978617B69002B21D07A697B6810
:10D5F0009A4204D1B969F8682BF06AF815E07869A5
:10D600002FF0F9FE0346002B0FD0012279687869CC
:10D610002BF049FE38613B69002B06D039697869E7
:10D620002BF056F838692DF0F5FC78692DF0F2FCF6
:10D63000B8692DF0EFFC03E00549032024F0FEFE5D
:10D640002037BD4680BD00BF148B0408DC8B040866
:10D650003C8C040880B586B000AF7860396078688B
:10D6600030F002FB034683F00103DBB2002B04D051
:10D670003249032024F0E2FE5CE038682FF089FD97
:10D680000346002B1BD039682D482BF0BDFF786175
:10D690007B69002B4ED00122796978682AF0DCFF83
:10D6A000386178692DF0B6FC3B69002B41D03969AF
:10D6B00078682BF00DF838692DF0ACFC3AE038684A
:10D6C0002FF01BFF0346002B2ED007F108037968CB
:10D6D000184627F02FFC19E007F108031846FFF75A
:10D6E00031F8F86007F10803184627F076FC0122AC
:10D6F0001449F8682DF0F6F90346002B03D0F968B9
:10D7000078682AF0E5FFF8682DF084FC07F108033B
:10D710001846FFF73FF80346002BDDD107F1080359
:10D720001846FFF748F805E00749032024F086FE75
:10D7300000E000BF1837BD4680BD00BF148B040851
:10D74000DC8B0408808C0408848C040880B584B0C9
:10D7500000AF7860396038682DF064FEF860FB68CF
:10D76000002B06D0F9687868FFF774FFF8682DF091
:10D7700051FC1037BD4680BD90B589B000AF7860D0
:10D78000396038682FF0BDFD034683F00103DBB23A
:10D79000002B04D05E49032024F050FEB5E07868E9
:10D7A0002FF091FE03461C4638682FF08CFE03468E
:10D7B0009C4216D038682FF086FE0346002B08D016
:10D7C0007B68DB899BB243F040039AB27B68DA81C5
:10D7D00007E07B68DB899BB223F040039AB27B6849
:10D7E000DA8178682FF0AEFD03461C4638682FF0CA
:10D7F000A9FD03469C4220D038682FF0A3FD0346C4
:10D80000002B0DD07B68DB899BB21BB223F03F035A
:10D810001BB243F008031BB29AB27B68DA810CE0BA
:10D820007B68DB899BB21BB223F03F031BB243F042
:10D8300007031BB29AB27B68DA8100223549786807
:10D840002AF0BAFDF8610022334978682AF0B4FD65
:10D85000B86178682BF01EF8FB69002B03D0F969DA
:10D8600078682AF097FBF8692DF0D4FB07F10C03D8
:10D870003968184627F05EFB30E007F10C031846C4
:10D88000FEF760FF786107F10C03184627F0A5FB4F
:10D89000204978692DF03AF9034683F00103DBB2A1
:10D8A000002B18D01C4978692DF030F9034683F01D
:10D8B0000103DBB2002B0ED0012178692AF0D8F9E0
:10D8C00038613B69002B06D0396978682AF062FB21
:10D8D00038692DF09FFB78692DF09CFB07F10C0354
:10D8E0001846FEF757FF0346002BC6D107F10C037D
:10D8F0001846FEF760FFBB69002B03D0B969786852
:10D900002AF048FBB8692DF085FB2437BD4690BD51
:10D91000DC8C04081C8D0408248D040890B597B095
:10D9200002AFF860B9607A600023BB6400237B64B7
:10D9300078682FF04AFF0346002B6FD078682BF0F1
:10D9400017FA03467B647B6C402B06D97A6C4549F9
:10D95000012024F073FD002380E07B6C9B000733E3
:10D960000733DB08DB00ADEB030D02AB0733DB084D
:10D97000DB00BB640023FB6408E0FB6C9B00BA6C1B
:10D98000134400221A60FB6C0133FB64FA6C7B6C5D
:10D990009A42F2D307F1100301227968184627F062
:10D9A000A7FF2DE007F11003184628F011F80346F1
:10D9B00018462CF075FB38643B6C002B1BDB7B6C32
:10D9C0003A6C9A4217DA3B6C9B00BA6C13441B68A2
:10D9D000002B05D0244A40F2C931244824F0A2FD8E
:10D9E0003B6C9B00BA6CD41807F11003184628F062
:10D9F0003DF80346236007F11003184624F0D4F8DD
:10DA000007F11003184624F089F80346002BC9D10A
:10DA100007F11003184624F019F90FE078682FF089
:10DA20006CFD034683F00103DBB2002B06D07A685D
:10DA30000F49012024F002FD00230FE07B6CBA6C3B
:10DA4000019200930023BA680021F86822F03CFBA1
:10DA5000F863B96C786C2DF03FFBFB6B18465437BC
:10DA6000BD4690BD308D0408788D0408E489040813
:10DA7000848D040880B592B000AFF860B9607A6018
:10DA8000F8682FF03EFC034683F00103DBB2002B65
:10DA900006D0FA689049032024F0D0FC002317E157
:10DAA000F8682FF010FD0346002B09D0FB681A68B8
:10DAB000FB689B88194610462DF041FE78640CE007
:10DAC000F8682FF03FFC0346002B01D0082300E04C
:10DAD0000723184630F058FA78647B6C002B01D18C
:10DAE0000023F5E007F11803F968184627F022FA39
:10DAF00042E007F118031846FEF724FEF86307F129
:10DB000018031846FEF732FEB863F86B2FF034FCAA
:10DB10000346002B04D0BB6B002B01D0012300E097
:10DB2000002387F8373097F8373003F0010387F880
:10DB3000373097F83730002B0ED00121F86B2AF0E0
:10DB400097F838633B6B002B06D0396B786C2AF062
:10DB500021FA386B2DF05EFAB96BF86B2DF086FA6E
:10DB600097F8373083F00103DBB2002B0CD107F1BB
:10DB70001803184627F031FA07F118031846FEF784
:10DB800009FE0346002BB4D17B68002B00F08D808A
:10DB900007F114037968184627F0CCF959E007F12A
:10DBA00014031846FEF7E2FDF862002387F84330BD
:10DBB0002CE007F118031846FEF7C4FDB862B86AF6
:10DBC0002FF0DAFB034683F00103DBB2002B03D016
:10DBD000B86A2DF01FFA28E001220021B86A2DF062
:10DBE000A7F87862F96A786A2AF0EAFA796A786CB2
:10DBF0002AF0D0F9012387F84330796AB86A2DF00A
:10DC000035FA07F11803184627F0E7F997F843307B
:10DC100083F00103DBB2002B07D007F1180318468D
:10DC2000FEF7B8FD0346002BC3D197F8433083F0CD
:10DC30000103DBB2002B04D0FA6A0021786C2DF0CE
:10DC400097FFF86A2DF0E6F907F11403184627F05C
:10DC5000C4F907F114031846FEF79CFD0346002B98
:10DC60009DD107F114031846FEF7A5FD1DE007F14D
:10DC700018031846FEF766FD386201220121386A52
:10DC80002DF056F8F861FB69002B06D0F969786C25
:10DC90002AF080F9F8692DF0BDF9386A2DF0BAF94B
:10DCA00007F11803184627F098F907F118031846EA
:10DCB000FEF770FD0346002BD9D107F11803184673
:10DCC000FEF779FDBA680549786C2AF0E3FE7B6CB3
:10DCD00018464837BD4680BDC08D0408E08604085C
:10DCE00080B483B000AF78607B681B69002B01D1E2
:10DCF000002305E07B681A697B681B6813441B7866
:10DD000018460C37BD465DF8047B704780B582B07D
:10DD100000AF78607B68DB6818462DF07BF9083728
:10DD2000BD4680BD80B582B000AF78600022064954
:10DD300078682AF037FE034618461BF076F903464A
:10DD400018460837BD4680BD207E040880B584B0E3
:10DD500000AF0346FB71FB79032118460BF0B6FDBB
:10DD6000FB79002118460BF093FF4FF4FA700BF08B
:10DD700081FDFB79012118460BF08AFF50200BF042
:10DD800079FDFB7918460BF0AEFF0346002B14BF5C
:10DD900001230023DBB283F00103DBB2FB73FB7BC7
:10DDA00003F00103FB734FF4D2700BF063FDFB7BB8
:10DDB00018461037BD4680BD80B584B000AF03461D
:10DDC0003960FB71FB79032118460BF07FFD0023BE
:10DDD000FB600123BB6024E00BF02CFDFB790021EC
:10DDE00018460BF055FF03200BF044FDFB79012191
:10DDF00018460BF04DFF0A200BF03CFDFB7918464E
:10DE00000BF071FF0346002B03D0FA68BB68134385
:10DE1000FB600BF016FD35200BF02CFDBB685B00A2
:10DE2000BB603B685A1E3A60002BD5DCFB68184685
:10DE30001037BD4680BD000090B58BB000AFF860D4
:10DE4000C7E90023F8682FF05CFA034683F001036A
:10DE5000DBB2002B0ED0F8682FF09BF9034683F05D
:10DE60000103DBB2002B05D04549012024F0E6FA7E
:10DE7000002378E0D7E90023D7E90001F2F7E2FDBB
:10DE80000346002B09D13AA3D3E90023D7E90001C7
:10DE9000F2F7B0FD0346002B04D035A4D4E90034DA
:10DEA000C7E9003434A3D3E90023D7E90001F2F72E
:10DEB000BFFD0346002B05D03249012024F0BEFAF5
:10DEC000002350E02DF006FC7862D7E900010CF049
:10DED0000FF9C7E906010CF05FF90A4601462A4B23
:10DEE000D3E90034C91A62EB0402D7E906345B189F
:10DEF00044EB0204184621462DF0A4FB03461A46C3
:10DF00002249786A2AF03EFE97F83C3083F00103FC
:10DF1000DBB2002B09D0D7E906012DF093FB0346B5
:10DF20001A461B49786A2AF02DFEFA681949786A60
:10DF30002AF0B0FDB86B2AF0D5FE0346002B04D0C2
:10DF4000BA6B1549786A2AF0A5FD786A16F0DEFEEC
:10DF5000034618462DF032FB7861786A2DF05AF8A6
:10DF600016F0F0FE7B6918462C37BD4690BD00BF09
:10DF70009A9999999999B93F00E8E3138CAEBC42FC
:10DF8000F88D04081C8E0408A0510120447E04086A
:10DF9000408E04084C8E0408588E040880B586B064
:10DFA00002AFF860C7E9002300230193BB69009327
:10DFB000D7E90023F868FFF73FFF034618461037FC
:10DFC000BD4680BD80B586B002AFF860C7E90023CA
:10DFD00001230193BB690093D7E90023F868FFF799
:10DFE0002BFF034618461037BD4680BD80B588B06C
:10DFF00000AF78600B46FB703A4B1B88184630F038
:10E00000E7F9F86178682FF078FA0346002B33D0EF
:10E0100007F10803F969184626F08CFF1EE007F1A6
:10E020000803184604F0BDFFB86100222E49B86904
:10E030002AF0B8FC78617B69002B06D107F1080350
:10E04000F969184626F0F9FF04E007F108031846BD
:10E0500026F0C3FFB96978692DF008F807F10803C5
:10E06000184604F0B2FF0346002BD8D107F108038D
:10E07000184604F0BBFF2CE078682FF068FA0346DE
:10E08000002B06D000227968F8692AF0E5FA0346E9
:10E0900000E000233B613B69002B0ED0114B1B8835
:10E0A000184630F095F9F8603969F8682AF010FBE5
:10E0B000F96838692CF0DAFF0BE0FB78002B04D00C
:10E0C0000A49012024F0BAF903E00949012024F0AB
:10E0D000B5F9F8692CF09EFF16F034FE2037BD46E6
:10E0E00080BD00BF98510120608E0408688E04082E
:10E0F000788E040880B582B000AF7860002178681F
:10E10000FFF774FF0837BD4680BD80B582B000AF11
:10E11000786001217868FFF769FF0837BD4680BD48
:10E1200090B58BB000AFF860C7E90023344B1B8873
:10E13000184630F04DF978622FA3D3E90023D7E9D0
:10E140000001F2F757FC0346002B04D02AA4D4E9BF
:10E150000034C7E90034F8682FF0F9F90346002BC2
:10E1600006D00022F968786A2AF076FA034600E0C1
:10E1700000233B623B6A002B32D0386A2CF004FC4F
:10E18000F861D7E900010BF0B3FFC7E90401D7E953
:10E1900004012DF057FA03461A461A49F8692AF085
:10E1A000F1FC0BF0F9FF0A460146174BD3E90034A6
:10E1B000C91A62EB0402D7E904345B1844EB020489
:10E1C000184621462DF03EFA03461A460F49F869D3
:10E1D0002AF0D8FCF8692CF01DFF16F0B3FD03E01F
:10E1E0000B49012024F02AF9786A2CF013FF2C3710
:10E1F000BD4690BDAFF300809A9999999999B93F1E
:10E2000098510120408E0408A0510120447E04084A
:10E21000788E040880B483B000AF78607B689B89F7
:10E2200018460C37BD465DF8047B704780B483B058
:10E2300000AF78607B68DB8818460C37BD465DF818
:10E24000047B704780B582B000AF78607B681B6844
:10E25000002B01D1002305E07B681B6818462CF0D9
:10E2600037FB034618460837BD4680BD80B483B0EF
:10E2700000AF78607B681B68002B14BF012300236C
:10E28000DBB218460C37BD465DF8047B704780B59D
:10E2900082B000AF78607B681B6818462CF0BAFE2D
:10E2A0000837BD4680BD80B483B000AF7860396068
:10E2B0003B68012B02D17B681B7812E03B68022B84
:10E2C00008D17B681B781A467B6801331B781B02D8
:10E2D000134306E03B68042B02D17B681B6800E017
:10E2E000002318460C37BD465DF8047B704790B597
:10E2F00093B000AFF860B9607A60FB68184608F028
:10E3000041FE7864BB68012B0CDC7968786CFFF700
:10E31000CAFF03464FF00004184621462DF092F93B
:10E32000034648E07B68012B02D10123A7F8423065
:10E330007B68022B02D10223A7F842307B68042BB2
:10E3400002D10423A7F84230B7F84230B968184622
:10E3500026F0F8F8F863FB6B002B01D100232AE0CC
:10E3600007F114030022F96B184626F08BFE14E027
:10E370007968786CFFF797FF03461A4607F1140394
:10E380001146184627F010F97B687A6C13447B64B9
:10E3900007F11403184627F06BFA07F11403184627
:10E3A00027F041FA0346002BE2D107F11403184687
:10E3B00027F08FFAFB6B18464C37BD4690BD80B4F2
:10E3C00085B000AFF860B9607A607B68012B04D13A
:10E3D000FB68BA68D2B21A700DE07B68022B04D1D8
:10E3E000FB68BA6892B21A8005E07B68042B02D100
:10E3F000FB68BA681A601437BD465DF8047B704745
:10E4000080B590B000AFF860B9607A60B8682EF05F
:10E4100057FF0346002B09D0B8682BF095FB034645
:10E420007A681946F868FFF7CAFF2EE0B8682FF03F
:10E43000CCF90346002B28D007F114030122B96858
:10E44000184627F055FA13E007F11403184627F091
:10E4500069FB03467A681946F868FFF7B0FFFA6867
:10E460007B681344FB6007F11403184623F09CFB00
:10E4700007F11403184623F051FB0346002BE3D1A8
:10E4800007F11403184623F0E1FB4037BD4680BD79
:10E4900090B58DB004AF0146C7E900230B46FB736E
:10E4A0004FF000034FF00004C7E906340023FB756A
:10E4B000386B2EF07FFF0346002B2BD000221D4926
:10E4C000386B2AF06FFA034618462BF0F5FDC7E9C2
:10E4D000060100221849386B2AF064FA03461846F0
:10E4E0002BF0F8FD0346002B04D0FB7D43F0020324
:10E4F000FB750FE000221149386B2AF053FA0346EE
:10E5000018462BF0E7FD0346002B03D0FB7D43F0BC
:10E510000103FB75F97BFB7D0293D7E90634CDE956
:10E520000034D7E9002308460CF082F82437BD46B2
:10E5300090BD00BF707E04088C8E0408988E04087D
:10E5400080B592B000AF03463A60FB710B46BB71D9
:10E5500038682EF0B5FE0346002B24D038682BF027
:10E5600069FCC7E910014FF000024FF00003D7E942
:10E570001001F2F73FFA0346002B08D1D7E9102328
:10E58000D7E91001F2F75EFA0346002B04D03249B6
:10E59000012023F053FF5BE0B979F879D7E9102324
:10E5A00008F0C6F954E038682FF00FF90346002B45
:10E5B00049D007F10C0301223968184627F098F971
:10E5C00033E007F10C03184627F030FBC7E90E01D2
:10E5D0004FF000024FF00003D7E90E01F2F71EFAE8
:10E5E0000346002B0ED0D7E90E23D7E90E01F2F730
:10E5F00029FA0346002B05D1B979F879D7E90E231A
:10E6000008F096F9BB79002B14BF01230023DBB27D
:10E6100083F00103DBB2BB71BB7903F00103BB7173
:10E6200007F10C03184623F0BFFA07F10C03184654
:10E6300023F074FA0346002BC3D107F10C031846EC
:10E6400023F004FB04E03A680449012023F0F6FEBD
:10E650004837BD4680BD00BFA08E0408E48E040884
:10E6600080B58AB002AF7860396078682EF0C3FE5A
:10E670000346002B31D07868FFF7CCFD0346FB83BF
:10E6800027E0FB8B18462FF0A3FEB861B8692CF089
:10E690001FF9786178691AF0A3FC03461A463B68B3
:10E6A00003F00103002B14BF01230023DBB2194642
:10E6B00010461AF057FD78692CF0ACFCB869FFF7EA
:10E6C000B5FD0346FB83B8692CF0A4FC3B685B10E6
:10E6D0003B60FB8B002BD4D142E078682EF06AFEC1
:10E6E0000346002B2CD000221F49786822F05AFCE8
:10E6F000386138692EF005FE0346002B18D03868C3
:10E700002CF05CFF0346BB6007F108030193012373
:10E71000009300237A680021386921F0D5FC034674
:10E7200018462CF077FCBB6818462CF073FC03E00D
:10E730000E49012023F082FE38692CF06BFC0FE0BB
:10E7400078681AF04DFC0346FB733B68002B14BF3E
:10E7500001230023DAB2FB7B114618461AF002FDB2
:10E760002037BD4680BD00BF00840408088F040820
:10E7700090B58DB002AF786078682EF03CFE03460D
:10E78000002B3BD000237B6200233B6207F10C038C
:10E790007968184626F0CEFB1CE007F10C031846FA
:10E7A000FFF750FDB8613B6A5C00B8691AF018FCCD
:10E7B000034618461AF0A6FC034623433B62B86999
:10E7C0002CF028FC07F10C03184626F006FC7B6AA7
:10E7D00001337B6207F10C031846FFF747FD034640
:10E7E000002BDAD107F10C031846FFF750FD7B6AC6
:10E7F000002B01D1002338E03B6A36E078682EF028
:10E80000D9FD0346002B26D00023FB6100221949C5
:10E81000786822F0C7FB786178692EF072FD0346B4
:10E82000002B0FD0002301930023009300237A686C
:10E830000021786921F048FC034618462BF030FC93
:10E84000F86103E00C49012023F0F8FD78692CF011
:10E85000E1FBFB6909E078681AF0C2FB0346FB7430
:10E86000FB7C18461AF04EFC034618462C37BD4672
:10E8700090BD00BF38840408088F040880B584B0B8
:10E8800000AF03463960FB711346BB71FB79184634
:10E890001EF014FF034683F00103DBB2002B04D00B
:10E8A0004F49012023F0CAFD97E00023FB7338682D
:10E8B0002EF06FFC0346002B58D04A4938682CF0E4
:10E8C00025F90346002B02D00723FB734EE046498F
:10E8D00038682CF01BF90346002B02D00423FB738D
:10E8E00044E0424938682CF011F90346002B02D06D
:10E8F0000523FB733AE03E4938682CF007F90346DC
:10E90000002B02D00623FB7330E03A4938682CF024
:10E91000FDF80346002B02D00123FB7326E03649A5
:10E9200038682CF0F3F80346002B02D00223FB7367
:10E930001CE0324938682CF0E9F80346002B02D07D
:10E940000323FB7312E02E4938682CF0DFF80346EE
:10E95000002B02D00823FB7308E02A4938682CF00A
:10E96000D5F80346002B01D00923FB73FB7B002B5A
:10E9700017D0BB79002B14BF01230023DBB283F037
:10E980000103DBB203F00103DAB2FB79114618464A
:10E990001AF07CFBFA7BFB79114618460AF096FFC9
:10E9A0001BE0FB79002118461AF070FB38682EF046
:10E9B000A4FD034683F00103DBB2002B0DD0124906
:10E9C00038682CF0A3F8034683F00103DBB2002B78
:10E9D00003D00E49012023F031FD1037BD4680BD24
:10E9E000187E0408188F04087C830408208F04080C
:10E9F000308F0408408F0408488F0408548F04089F
:10EA0000688F0408748F0408848F04088C8F0408AE
:10EA100080B584B000AF0346FB71FB7918461EF049
:10EA20004DFE034683F00103DBB2002B05D02849DD
:10EA3000012023F003FD002345E0FB7918460BF08D
:10EA400027F8034603F00F03FB720023FB60FB7AF9
:10EA5000013B082B2ED801A252F823F099EA0008B6
:10EA60009FEA0008A5EA000887EA00088DEA000886
:10EA700093EA000881EA0008ABEA0008B1EA00085E
:10EA8000144BFB6016E0144BFB6013E0134BFB6070
:10EA900010E0134BFB600DE0124BFB600AE0124BE1
:10EAA000FB6007E0114BFB6004E0114BFB6001E0F1
:10EAB000104BFB60FB68002B04D0F8682CF0B2FC14
:10EAC000034600E0002318461037BD4680BD00BF56
:10EAD000187E0408188F04087C830408208F04081B
:10EAE000308F0408408F0408488F0408548F0408AE
:10EAF000688F0408748F040880B487B000AF786012
:10EB000039603B68FB6000233B6135E0FB685B6B71
:10EB1000013B7B6117E0FA687B6902339B00134479
:10EB20005B68002B09D0FA687B6902339B001344B1
:10EB30005B687A6802F001021A607B685B107B6098
:10EB40007B69013B7B617B69002BE4DAFB68DB6A54
:10EB5000002B0ED0FB68DB6AFA6892F830201A604E
:10EB6000FB68DB6AFA6892F8302082F00102D2B2C8
:10EB70001A603B6901333B61FB689A6B3B699A42BF
:10EB8000C4DC1C37BD465DF8047B704790B59FB070
:10EB900000AFF860B9607A600023FB66FF2387F856
:10EBA0004030002387F8683001233B676B4B7B6163
:10EBB0000C233B8307F138030833FB61684B3B624E
:10EBC0000B23BB8407F138033033BB62654BFB6218
:10EBD00009233B8607F1380338337B6307F11403BD
:10EBE00003221946B86825F03BFB034683F0010376
:10EBF000DBB2002B40F0AE8097F8683087F86830C1
:10EC00003B6F002B01DC01233B67F8682EF0F3FB20
:10EC10000346002B36D007F11003F968184626F09A
:10EC200089F921E0FB6E072B05DD08224E49012002
:10EC300023F004FC8EE0FC6E07F110031846FFF78A
:10EC400001FB034618461AF0F0F903461A4607F18D
:10EC50007803234403F8402CFB6E0133FB6607F175
:10EC60001003184626F0B9F907F110031846FFF70C
:10EC7000FDFA0346002BD5D107F110031846FFF724
:10EC800006FB0CE0FC6E631CFB66F8681AF0A8F942
:10EC900003461A4607F17803234403F8402C002367
:10ECA0007B6736E007F138027B6F13441B78184608
:10ECB0001EF004FD0346002B16D007F138027B6FCF
:10ECC00013441B7818461AF0C1F9034683F0010378
:10ECD000DBB2002B08D007F138027B6F13441B789E
:10ECE000012118460AF0F2FD07F138027B6F134448
:10ECF0001B780121184607F093FF02467B6F023311
:10ED00009B0007F178010B4443F83C2C7B6F0133E7
:10ED10007B67FA6E7B6F9A42C4DC97F84030012122
:10ED2000184607F07DFF03467B6697F8403018468B
:10ED30001EF0C4FC0346002B05D097F8403001219B
:10ED400018460AF0C3FD07F138031A4607497868E8
:10ED500025F03EFD7C37BD4690BD00BFA08F040866
:10ED6000A48F04084C7E0408AC8F0408F9EA00085C
:10ED700090B591B000AFF8600B467A60FB72FB7AF9
:10ED800018461EF09BFC034683F00103DBB2002B08
:10ED900004D0854823F00EFB0023E7E1FB7A1846F8
:10EDA00019F0D4F9034683F00103DBB2002B0ED037
:10EDB000FB7A18460BF084FE034683F00103DBB2B6
:10EDC000002B04D0794823F017FB0023CEE1002369
:10EDD00087F83F304FF000034FF00004C7E90C34D0
:10EDE0000023FB62002387F82B30FF2387F82A30AB
:10EDF000FB7A2C2B06D10123FB624FF000036C4CF5
:10EE0000C7E90C3478682EF0D5FA0346002B00F0E1
:10EE1000AA8000226749786829F0C4FDF861FB697F
:10EE2000002B05D0F8692BF055F9034687F83F30E1
:10EE300000226149786829F0B5FDF861FB69002B73
:10EE400004D0F8692BF038F9C7E90C01D7E90C2395
:10EE5000D7E90C01F1F7F6FD0346002B0AD14FF07C
:10EE600000024FF00003D7E90C01F1F7C3FD0346A0
:10EE7000002B05D04FF000034FF00004C7E90C341D
:10EE800000224E49786829F08DFDF861F8692EF06E
:10EE900034FB0346002B3DD1F8692EF011FA0346EE
:10EEA000002B11D0F8692AF04FFEB861BB69002B26
:10EEB00007DCBB69002B02DA4FF0FF3302E00023CE
:10EEC00000E00123FB6225E03D4BFB62F8692EF078
:10EED00060F90346002B1DD03A49F8692BF016FE65
:10EEE0000346002B02D00123FB6213E03649F86988
:10EEF0002BF00CFE0346002B03D04FF0FF33FB62D8
:10EF000008E03249F8692BF001FE0346002B01D0DE
:10EF10000023FB62F8692CF07DF8FB6AB3F1FF3F38
:10EF200002DBFB6A012B05DD2949032023F086FA69
:10EF300000231BE100222749786829F033FD0346AE
:10EF400018462BF0C7F8034687F82B3000222249D9
:10EF5000786829F027FD034618461AF066F803463C
:10EF600087F82A3005E078682AF002FF034687F820
:10EF70003F304FF0FF337B62F8682EF0C2F9034652
:10EF800083F00103DBB2002B2AD0F8682EF001F9E0
:10EF9000034683F00103DBB2002B21D00F4901208F
:10EFA00023F04CFAD9E000BF187E0408C88F04088B
:10EFB000000039404C7E0408509004085C9004081E
:10EFC00018FCFFFF649004086C9004087490040817
:10EFD0007C900408C4900408BC780408F88D0408E8
:10EFE0002CF078FB78617B69002B43D0FB7A1846C4
:10EFF0002CF053FB03461A465E49786929F0C2FD9E
:10F0000097F83F30002B0AD097F83F3018462CF085
:10F01000EAFA03461A465849786929F0B3FD4FF0D9
:10F0200000024FF00003D7E90C01F1F701FD0346A0
:10F03000002B0ED0D7E90C010BF05AF803460C4612
:10F0400018462CF0BBFA03461A464C49786929F059
:10F0500099FDFB6A002B08D0F86A2CF0AFFA034642
:10F060001A464749786929F08DFDFA68454978695B
:10F0700029F010FD002387F82330FB7A184619F099
:10F0800065F8034683F00103DBB2002B07D0FB7A5F
:10F09000012118460BF03CFD034687F8233097F812
:10F0A0002330002B3DD097F823300021184617F06D
:10F0B00053F897F82A3018461EF000FB0346002B41
:10F0C00007D097F82A2097F823301146184617F0F2
:10F0D00065F897F82B30002B2CD0F8682EF0F3F958
:10F0E0000346002B0BD0F8682CF086FD03461A4629
:10F0F00097F823301146184617F02EF81AE097F8C3
:10F100002A3018461EF0DAFA0346002B04D01E49B6
:10F11000012023F093F90DE01C49012023F08EF922
:10F1200009E097F82B30002B05D01949012023F076
:10F1300085F900E000BF174B1B8818462FF048F9EF
:10F1400038610122796938692AF0C2F80346013B27
:10F150007B62796938692BF089FF7B6A002B04DBBD
:10F16000786A2CF02BFA034600E000231846443757
:10F17000BD4690BD207E0408C89004085090040845
:10F180005C9004084C8E0408D0900408F4900408A5
:10F19000289104089A51012080B58CB000AF7860A6
:10F1A00078682EF0AAF90346002B3DD0444B1B880B
:10F1B00018462FF00DF9F86207F10C03F96A1846AA
:10F1C00025F0B8FE1CE007F10C031846FFF73AF8EB
:10F1D000B86200223B49B86A29F0E4FB7862786A99
:10F1E00019F0FEFE0346002118460BF091FCB96AA7
:10F1F000786A2BF03BFF07F10C03184625F0EDFE73
:10F2000007F10C031846FFF731F80346002BDAD15B
:10F2100007F10C031846FFF73AF8F86A29F03AFBB1
:10F22000F86A2BF0F7FE47E0254B1B8818462FF0B5
:10F23000CFF8386200227968386A29F00DFAF8614F
:10F24000386A2BF0E7FEFB69002B2FD0F8692BF012
:10F250003FFBB86100221B49B86929F0A3FB0346B4
:10F26000184619F0E2FE0346FB75B8692BF0D2FE92
:10F27000134B1B8818462FF0ABF83861F9693869D1
:10F2800029F026FA3969F8692BF0F0FEFB7D184663
:10F2900018F05CFF034683F00103DBB2002B0AD0B9
:10F2A000FB7D002118460BF033FC05E006490120E8
:10F2B00023F0C4F800E000BF3037BD4680BD00BF7A
:10F2C0009A510120207E04085091040880B582B034
:10F2D00000AF1B202EF058FE78607B681846083778
:10F2E000BD4680BD80B483B000AF78607B681B6989
:10F2F000002B01D1002305E07B681A697B681B683D
:10F3000013441B7818460C37BD465DF8047B7047E4
:10F3100080B483B000AF78607B681A687B685B68F4
:10F320009A4234BF01230023DBB218460C37BD4696
:10F330005DF8047B704780B582B000AF78607B6871
:10F34000DB6818462BF066FE0837BD4680BD80B5E9
:10F3500082B000AF78607B681B68002B01D100236E
:10F3600005E07B681B6818462FF078F803461846BE
:10F370000837BD4680BD80B582B000AF78607B683D
:10F380001B68002B01D1002305E07B681B68184631
:10F390002BF09EFA034618460837BD4680BD80B460
:10F3A00083B000AF78607B681B68002B14BF01231B
:10F3B0000023DBB218460C37BD465DF8047B70476E
:10F3C00080B582B000AF78607B681B6818462BF070
:10F3D00021FE0837BD4680BD80B58AB000AFF86019
:10F3E000B9607A60D023FB84FFF770FFF861FB6996
:10F3F000002B4ED000233B6107F1140300221A605A
:10F40000C3F8032078682EF078F80346002B30D13B
:10F4100078682EF082F80346002B2AD178682DF008
:10F420004FFF0346002B1DD078682AF08DFB034662
:10F430003B623B6A0A2B01D90A233B6207F11002A7
:10F440003B6A134400221A7008E03B6A013B3B62AE
:10F4500007F110023B6A134420221A703B6A002B0A
:10F46000F3D106E007F110030B22194678682CF05F
:10F47000DBFD07F110031B78002B03D0FB8C43F05E
:10F480000603FB8407F11003FA8CF969F868FCF7AE
:10F490006DFCFB6918462837BD4680BD80B596B027
:10F4A00000AFB24B1B68B3F90230822B78D0822BAD
:10F4B0000DDC5B2B00F097805B2B02DC2D2B30D01A
:10F4C00056E17B2B00F0E080812B53D050E1B42B30
:10F4D00009D0B42B02DC832B78D049E1B52B0CD0BA
:10F4E000B62B14D044E1A14B1B68184630F09AFCAF
:10F4F00001202CF078F803464BE19C4B1B68184622
:10F5000030F090FC00202CF06EF8034641E1974B60
:10F510001B68184630F086FC02202EF035FD0346AD
:10F5200037E1924B1B68184630F07CFC8F4B1B6810
:10F53000B3F90230812B07D08C4B1B68B3F9023032
:10F54000822B01D0002324E1884B1B681846FFF76B
:10F55000A5FF386500202CF031F8F8642D22396DB4
:10F56000F86C26F0E1FEB864F96C386D2BF07EFD86
:10F57000BB6C0EE17D4B1B68184631F0E7FC03467F
:10F58000184622F005FFC7E91001784B1B681846A2
:10F5900030F048FCD7E910012CF054F80346F8E0AD
:10F5A000724B1B68184631F0D1FC0346184623F015
:10F5B00047F9C7E90E016D4B1B68184630F032FC65
:10F5C000D7E90E012CF026F80346E2E0674B1B68F2
:10F5D000184631F0DFFC7863644B1B68184630F046
:10F5E00021FC7B6BD5E02CF07DF838633B6B002B66
:10F5F00001D10023CDE05D4B1B68184630F012FCB2
:10F6000024E05A4B1B681846FFF748FFF862FB6A74
:10F61000002B0ED0554B1B68B3F902305D2B0ED07A
:10F620002C2031F043FD034683F00103DBB2002BB5
:10F6300005D0396BF86A2BF019FD0023A9E0F96AAF
:10F64000386B29F093FEF86A2BF0E4FC474B1B68FB
:10F65000B3F902305D2B07D024F06EFA034683F035
:10F660000103DBB2002BCCD15D2031F01FFD03463E
:10F6700083F00103DBB2002B04D0386B2BF0CAFC03
:10F68000002386E03B6B84E02CF024F8B862BB6A70
:10F69000002B01D100237CE0344B1B68184630F06E
:10F6A000C1FB45E0314B1B68184631F073FC034643
:10F6B00018462CF0CEFF78622C4B1B68184630F0B1
:10F6C000B1FB00237B653A2031F0F0FC034683F068
:10F6D0000103DBB2002B17D1244B1B681846FFF740
:10F6E000DDFE78657B6D002B0ED0204B1B68B3F9D7
:10F6F00002307D2B0FD02C2031F0D8FC034683F054
:10F700000103DBB2002B06D0BA6A796D786A2BF060
:10F71000BBFC00233DE0796D786A2CF081F803464C
:10F720001946B86A28F036FC796A786D2BF09EFC91
:10F730000E4B1B68B3F90230832B07D124F0FCF980
:10F74000034683F00103DBB2002BABD17D2031F007
:10F75000ADFC034683F00103DBB2002B04D0B86A92
:10F760002BF058FC002314E0BB6A12E0400100209B
:10F770000A4B1B68B3F9023018463B1D202219467C
:10F7800031F03EFA3B1D1A460549022022F056FE92
:10F79000002318465837BD4680BD00BF40010020F9
:10F7A0006091040880B5A6B000AF786078682CF04E
:10F7B000A3FDC7F8940007F10C0318462FF0FCFFD7
:10F7C000C7F89000D7F8940031F046F9D7F89400C4
:10F7D0002BF020FCFFF762FEC7F88C0031F07EF9B9
:10F7E000D7F890002FF0E8FFD7F88C3018469837FC
:10F7F000BD4680BD80B598B000AFF8607A603B60D0
:10F800000B467B81F8682DF07CFD034683F00103F5
:10F81000DBB2002B04D0824ABA21824822F082FE59
:10F820000023FB6507F14803F968184625F082FBC1
:10F83000012387F85B307C4A3968786823F0DEFC66
:10F8400044E007F148031846FFF781FD7865786DBD
:10F850002DF092FD0346002B1DD097F85B30002B56
:10F8600003D0002387F85B3004E0704A3968786879
:10F8700023F0C4FC6FF000420121786D29F054FFA1
:10F8800038653B6D6A4A3968786823F0B7FC386D93
:10F890002BF0C0FB12E0786D2DF07BFC0346002BB3
:10F8A0000CD06449786D2BF031F90346002B05D05C
:10F8B00007F148031846FFF75EFDF865786D2BF0F9
:10F8C000A9FB07F14803184625F087FB07F1480319
:10F8D0001846FFF764FD0346002BB2D107F1480339
:10F8E0001846FFF76DFD544A3968786823F086FCA6
:10F8F000F8682DF0CEFD0346002B05D04F4A39683D
:10F90000786823F07BFC84E0FB6D002B7CD07B8946
:10F9100003F00803002B07D0494B1B68494A39689C
:10F92000786823F06BFC74E00A21F86D29F083FFFE
:10F930000346DB43DB0F87F84F3097F84F30002B3F
:10F9400001D0414A00E0414A7B6839681046984737
:10F95000F8682DF0F7FC0346002B03D07B6839686C
:10F960003B489847002387F85A3007F134030022B8
:10F97000F96D184625F0B0F82DE007F1340318466C
:10F98000FFF7B0FC034687F84E3097F84E2097F803
:10F990005A301146184631F0E9FD0346002B03D0DA
:10F9A0007B6839682B48984707F1140197F84E3067
:10F9B0002022184631F008F907F114027B683968F3
:10F9C0001046984707F13403184625F097F997F841
:10F9D0004E3087F85A3007F134031846FFF798FC89
:10F9E0000346002BC9D107F134031846FFF7A3FCE7
:10F9F00097F84F30002B01D0174A00E0174A7B6878
:10FA000039681046984704E0154A3968786823F049
:10FA1000F5FBF86D2BF0FEFA6037BD4680BD00BFE8
:10FA200080910408EC870408C8A90408949104088C
:10FA30008C99040898910408A0910408A4910408E2
:10FA4000CC000020B8910408C0910408C8910408B3
:10FA5000CC910408D4780408D4910408B491040823
:10FA6000D891040880B582B000AF786078682DF036
:10FA700044FD034683F00103DBB2002B13D078680A
:10FA80002DF04BFD034683F00103DBB2002B0AD0BF
:10FA900078682DF015FC034683F00103DBB2002BE0
:10FAA00001D0012300E0002303F00103DBB218467C
:10FAB0000837BD4680BD000080B586B000AFB96094
:10FAC0007A603B600346FB810B4A3968786823F013
:10FAD00095FBFB899B0A9BB27B6104E0BA6839689D
:10FAE000786823F08BFB7B695A1E7A61002BF5D175
:10FAF0001837BD4680BD00BF149F040880B590B084
:10FB000002AFF8607A601A460B467B8113463B8150
:10FB1000002387F8373000233B63F2E0F868FFF7F3
:10FB200016FCB862B86A2AF0ADFD7862B86A24F0B3
:10FB30004FFB0346002B1BD17B8903F01003002BE6
:10FB400005D0786A2DF0DDFB0346002B10D17B89B0
:10FB500003F04003002B05D0786A2DF0CEFC03465D
:10FB6000002B05D1786A2DF0B5FD0346002B01D09E
:10FB7000012300E0002387F8233097F8233003F0B7
:10FB8000010387F8233097F8233083F00103DBB2B9
:10FB9000002B00F0AF803B6B01333B6397F848309C
:10FBA00083F00103DBB2002B0CD07B8903F004034C
:10FBB000002B01D05D4B00E05D4B1A46796C386C30
:10FBC00023F01CFB7B8903F00103002B07D0786A2C
:10FBD000FFF748FF0346002B01D0012300E000237C
:10FBE00087F82F3097F82F3003F0010387F82F3074
:10FBF0007B8903F00103002B06D004223B6B934268
:10FC000002D9012387F837307B8903F00203002BE8
:10FC100005D0012387F83730012387F82F3097F874
:10FC20003730002B03D197F82F30002B0AD03889BA
:10FC30007B6C3A6C7968FFF73FFF002387F8373019
:10FC400000233B63012387F82E307B8903F4007384
:10FC5000002B27D0B86A2DF092FD0346002B03D06D
:10FC6000002387F82E301DE0B86A2DF092FA034683
:10FC7000002B17D0B86A2CF018FD03460E2B11D8B4
:10FC800007F1100310221946B86A2CF0CDF907F1DC
:10FC90001003184622F05BF90346002B02D0002324
:10FCA00087F82E3097F82E30002B01D0214A00E043
:10FCB000214A7B8903F00403002B01D01F4B00E095
:10FCC0001F4B0093BB6A796C386C23F097FA97F856
:10FCD0004830002B02D0002387F8483039897B6CEC
:10FCE00000933B6C7A68786A00F02CF897F82F3014
:10FCF00087F83730796AB86A2BF0B8F9F86825F0D8
:10FD00006CF9F868FFF74BFB0346002B08D023F093
:10FD1000BBFE034683F00103DBB2002B7FF4FEAE93
:10FD200097F8373018463837BD4680BD84B104088F
:10FD300094910408DC910408E4910408EC9104080F
:10FD4000F091040890B5ADB004AFF8607A603B6004
:10FD50000B467B817B8903F58063A7F88C307B6839
:10FD6000002B01D1C94B7B60F8682DF0C6FB034620
:10FD7000002B07D0C64AD7F8B010386823F03EFAF7
:10FD800000F043BCFB68DB899BB203F48073002B5B
:10FD900007D0C04AD7F8B010386823F02FFA00F027
:10FDA00034BCFB68DB899BB243F480739AB2FB6876
:10FDB000DA81F8682DF01FFB0346002B00F08281EA
:10FDC000F86828F08FFFC7F888007B8903F00803E4
:10FDD000002B07D00F231A46D7F88830934201DD55
:10FDE000012300E0002387F8873097F8873003F07D
:10FDF000010387F88730002387F89F307B8903F061
:10FE00000403002B01D0A44B00E0A44B1A46D7F802
:10FE1000B010386823F0F2F94FF0FF33C7F898308C
:10FE2000012387F89730012387F8963007F13C03C8
:10FE3000F968184625F07EF8E7E007F13C0318461C
:10FE4000FFF785FAC7F8800007F13C031846FFF773
:10FE5000A6FA034683F00103DBB2002B07D1D7F8E3
:10FE600080002DF02DFA0346002B00F0C78007F12B
:10FE70003C031846FFF793FA0346002B05D0D7F84A
:10FE8000800029F061FE034602E0D7F88830013B8C
:10FE9000FB6707F13C031846FFF76DFAB8679EE071
:10FEA000D7F898300133C7F8983097F8873083F047
:10FEB0000103DBB2002B0FD105231A46D7F8983087
:10FEC000934209DB05231A46D7F888309A1AD7F8E7
:10FED00098309A4200F3838097F8963083F00103BC
:10FEE000DBB2002B0DD07B8903F00403002B01D083
:10FEF0006B4B00E06B4B1A46D7F8B010386823F014
:10FF00007DF9002387F8963097F88730002B10D0C2
:10FF100005231A46D7F888309A1AD7F898309A42AB
:10FF200007D1614B1B681A46D7F8B010386823F028
:10FF300065F97B8903F00103002B07D0B86FFFF749
:10FF400091FD0346002B01D0012300E0002387F838
:10FF5000953097F8953003F0010387F895307B8949
:10FF600003F00203002B05D0012387F89F30012303
:10FF700087F8953097F89F30002B03D197F895308C
:10FF8000002B0AD0B7F88C00D7F8B0303A687968FF
:10FF9000FFF792FD002387F89F30D7F89820FB6F7A
:10FFA0009A420AD1B7F88C10D7F8B03000933B686A
:10FFB0007A68B86FFFF7C6FE0DE07B8903F0400357
:10FFC000002B01D0394B00E0314B1A46D7F8B01066
:10FFD000386823F013F997F8953087F89F30D7F8F1
:10FFE0009820FB6F9A42FFF65BAFB86F2BF012F8C8
:10FFF00007F13C03184624F0F0FF02E0002387F8E5
:020000040801F1
:100000009730D7F880002BF005F8D7F898305A1CB5
:10001000D7F888309A420CDA97F89730002B08D03E
:1000200023F032FD034683F00103DBB2002B7FF4A3
:1000300004AF7B8903F00403002B10D0B7F88C20A9
:10004000798907F13C0097F896300293D7F8B030E1
:1000500001933B68009313467A68FFF74FFD07F161
:100060003C031846FFF7ACF997F89F30002B06D0F9
:100070007889D7F8B0303A687968FFF71DFD7B8939
:1000800003F00403002B15D0094B14E0F49104088D
:1000900034C00408D0780408F8910408FC910408DE
:1000A00084B1040894910408CC0000200092040854
:1000B00008920408BA4B1A46D7F8B010386823F0F3
:1000C0009DF89AE2F8682DF0B0F90346002B00F095
:1000D0004181012387F8943007F114030022F96865
:1000E000184624F0CFFF15E007F11403184625F059
:1000F000C8F94FF000024FF00003F0F771FC03461F
:10010000002B02D1002387F8943007F1140318461E
:1001100025F0AEFB07F11403184625F084FB0346D7
:10012000002BE1D107F11403184625F0D2FB7B899F
:1001300003F08003002B14BF0123002387F87730DE
:1001400097F89430002B17D097F8773083F001039D
:10015000DBB2002B10D0F86810F06EFF0446F86890
:100160002AF070F90346009323468E4AD7F8B01060
:10017000386823F043F840E2F86810F05DFFC7F8F4
:1001800090008949D7F89000F0F7CEFE0346002B87
:100190000CBF0123002387F8763097F87630002BC8
:1001A00002D0824BC7F8903097F87730002B01D0FF
:1001B0007F4A00E07F4AD7F89030D7F8B01038680F
:1001C00023F01CF87B8903F00203002B07D0B7F85B
:1001D0008C00D7F8B0303A687968FFF76DFCF868A2
:1001E0002AF030F938677B8903F00803002B05D02B
:1001F0000F223B6F934201D9012300E0002387F8CF
:100200006F3097F86F3003F0010387F86F3007F114
:1002100014030022F968184624F034FF58E097F8D8
:100220006F3083F00103DBB2002B09D17B6B052219
:10023000934205D37A6B05213B6F5B1A9A4242D3F6
:100240007B6B002B0DD07B8903F00403002B01D0C6
:10025000594B00E0594B1A46D7F8B010386822F0D5
:10026000CDFF7B8903F00203002B07D0B7F88C0089
:10027000D7F8B0303A687968FFF71EFC97F86F300E
:10028000002B0DD07A6B05213B6F5B1A9A4207D188
:100290004B4B1B681A46D7F8B010386822F0AEFFF7
:1002A00007F11403184625F057F8B866B7F88C1014
:1002B000D7F8B03000933B687A68B86EFFF742FD1C
:1002C000B86E2AF0A7FE07F11403184625F0D0FAFD
:1002D00007F11403184625F0A6FA0346002B07D0B1
:1002E00023F0D2FB034683F00103DBB2002B96D14F
:1002F0007B8903F00203002B06D07889D7F8B03051
:100300003A687968FFF7D8FB07F11403184625F01F
:10031000E0FA97F87730002B01D0214B00E0294B11
:100320001A46D7F8B010386822F068FF97F8763090
:10033000002B00F0628197F8773083F00103DBB285
:10034000002B00F05A81204AD7F8B010386822F00C
:1003500055FF52E1F8682DF02DF80346002B00F010
:10036000DD807B8903F02003002B04D0F86819F0AE
:10037000E4FB034600E0002387F8673097F8673016
:10038000002B25D097F86730184615F00DFD034671
:100390000E4AD7F8B010386822F030FF2DE100BFC8
:1003A0003CD804080C920408C0C30408189204083E
:1003B000FC9104082492040884B104089491040870
:1003C000CC000020309204083492040878D8040845
:1003D000012387F88F307B8903F48073002B52D080
:1003E00000228B49F86828F0DDFA3866386E2DF067
:1003F0003BFC0346002B43D000228649386E28F090
:10040000D1FAF865FB6D002B3AD0834B1B680122B3
:10041000F96D184628F047FFB865BB6D002B06D074
:10042000BB6D7E4AD7F8B010386822F0E7FEF96D50
:10043000B86D2AF01BFE00227949F86820F0B2FD61
:1004400078657B6D002B18D07B6D1B68754A9342D5
:1004500013D000230022F968786D1DF017F8386575
:100460003B6D714AD7F8B010386822F0C7FE386D7E
:100470002AF0D0FD002387F88F30786D2AF0CAFD6E
:10048000386E2AF0C7FD97F88F30002B00F0B5804A
:1004900007F14003F968184624F04CFD7B8903F00E
:1004A0000403002B01D0614B00E0614B1A46D7F8E2
:1004B000B010386822F0A2FEB7F88C20798907F1D5
:1004C000400001230293D7F8B03001933B680093BA
:1004D00013467A68FFF712FB034687F84F3007F19F
:1004E00040031846FEF76CFF97F84F30002B06D0FC
:1004F0007889D7F8B0303A687968FFF7DDFA7B89F8
:1005000003F00403002B01D04A4B00E04A4B1A468B
:10051000D7F8B010386822F071FE6EE0F8682CF061
:10052000F0FE0346002B1AD07B8903F01003002B4A
:1005300006D0424AD7F8B010386822F05FFE5CE07F
:100540003F4AD7F8B010386822F058FEB7F88C1040
:10055000D7F8B0303A68F868FFF74CF94DE0F86822
:100560002CF017FE0346002B40D0F8682DF009F858
:10057000034683F00103DBB2002B37D07B8903F005
:100580000803002B2AD0F8682CF08FF802462823A5
:100590009A4223D911231A460021F86829F0C4F899
:1005A000B864F8682CF081F802461123D31A11229E
:1005B0001946F86829F0B8F87864224B1B687A6C01
:1005C00001920093BB6C204AD7F8B010386822F033
:1005D00015FE796CB86C2AF049FD0EE0FB681B4AE9
:1005E000D7F8B010386822F009FE06E0FB680E4A22
:1005F000D7F8B010386822F001FEFB68DB899BB2A7
:1006000023F480739AB2FB68DA81A437BD4690BDAB
:100610006C89040860890408585101203C92040840
:100620004492040821C900088C99040850920408D7
:10063000C891040854920408B491040834C0040812
:1006400058920408CC0000206492040868920408C0
:1006500090B585B000AFC7E90201C7E90023D7E92B
:100660000023D7E90201F0F7C5F90346002B03D0B8
:10067000D7E90034C7E90234D7E90823D7E90201F2
:10068000F0F7D6F90346002B03D0D7E90834C7E9C1
:100690000234D7E90234184621461437BD4690BDCE
:1006A00090B591B000AF786078682CF072FD034689
:1006B00083F00103DBB2002B1AD078682CF09BFE8C
:1006C000034683F00103DBB2002B11D078682CF0D5
:1006D000ACFE034683F00103DBB2002B08D07A683E
:1006E0001F49012021F0AAFE4FF000031D4C32E00B
:1006F0004FF000034FF00004C7E90E3407F10C037C
:1007000000227968184625F0F3F815E007F10C038C
:10071000184625F08BFA03460C461A462346D7E9BD
:100720000E01EFF743FD03460C46C7E90E3407F10F
:100730000C03184621F038FA07F10C03184621F093
:10074000EDF90346002BE1D107F10C03184621F027
:100750007DFAD7E90E34184621464437BD4690BD90
:100760006C9204080000F87F90B595B000AFF86077
:10077000C7E90023F8682DF028F8034683F0010349
:10078000DBB2002B08D0FA682849012021F056FE80
:100790004FF00003264C44E04FF000034FF00004FC
:1007A000C7E9123407F114030122F968184625F04D
:1007B0009FF827E007F11403184625F037FAC7E938
:1007C0001001D7E90023D7E91001EFF7EDFC03464C
:1007D0000C46C7E91034D7E91023D7E91001EFF729
:1007E00097FE03460C461A462346D7E91201EFF757
:1007F000DDFC03460C46C7E9123407F11403184622
:1008000021F0D2F907F11403184621F087F90346C5
:10081000002BCFD107F11403184621F017FAD7E9BE
:100820001234184621465437BD4690BD9C920408A8
:100830000000F87FB0B59EB000AFF860B9607A6094
:10084000F8682CF0C2FF034683F00103DBB2002BF3
:1008500008D1B8682CF0B9FF034683F00103DBB27E
:10086000002B09D0BB68FA684949012021F0E6FD58
:100870004FF00003474C86E04FF000034FF00004B8
:10088000C7E91C3407F140030122F968184625F036
:100890002FF807F114030122B968184625F028F84B
:1008A000B86828F065FAF8667B68FA6E93FBF2F296
:1008B000F96E01FB02F29B1A7B607B68002B09DA60
:1008C0007A68FB6E13447B6004E007F1140318465A
:1008D00021F06AF97B685A1E7A60002BF5DC3EE055
:1008E00007F14003184625F0A1F904460D4607F12B
:1008F0001403184625F09AF902460B46204629466D
:10090000EFF706FE03460C461A462346D7E91C01BC
:10091000EFF74CFC03460C46C7E91C3407F14003D3
:10092000184621F041F907F11403184621F03CF96B
:1009300007F11403184621F0F1F8034683F0010390
:10094000DBB2002B0BD007F11403184621F07EF91F
:1009500007F114030122B968184624F0C9FF07F112
:100960004003184621F0DAF80346002BB8D107F10E
:100970004003184621F06AF907F11403184621F0E4
:1009800065F9D7E91C34184621467837BD46B0BD15
:10099000CC9204080000F87F90B597B000AFB96022
:1009A0007A603B600346FB8101237B6500233B6546
:1009B00005E07B6D5B007B653B6D01333B653A6D0C
:1009C000BB689A42F5DB7B6D5B10FB620023FB6426
:1009D00000233B6544E03A6DFB6C9A422BDA3B6D99
:1009E0009B007A6813441B68BB623B6D9B003A68AE
:1009F00013441B687B623B6D9B007A681344FA6C5E
:100A0000920079680A4412681A603B6D9B003A684C
:100A10001344FA6C920039680A4412681A60FB6C3D
:100A20009B007A681344BA6A1A60FB6C9B003A68B0
:100A300013447A6A1A60FB6ABB6406E0FA6CBB6C0A
:100A4000D31AFB64BB6C5B10BB64BA6CFB6C9A4240
:100A5000F4DDFA6CBB6C1344FB643B6D01333B6506
:100A60007B6D5A1E3B6D9A42B5DCA84BFB634FF081
:100A70000003BB6301233B6400237B6407E13B6C01
:100A80003B623B6C5B003B644FF07E537B634FF0FB
:100A900000033B630023FB64A3E0FB6C3B6577E052
:100AA0003A6D3B6A1344FB61FB699B007A6813440F
:100AB00093ED007AD7ED0D7A27EE277AFB699B003C
:100AC0003A681344D3ED006AD7ED0C7A66EEA77A44
:100AD00077EE677AC7ED067AFB699B003A681344A4
:100AE00093ED007AD7ED0D7A27EE277AFB699B000C
:100AF0007A681344D3ED006AD7ED0C7A66EEA77AD4
:100B000077EE277AC7ED057AFB699B007A68134474
:100B10003A6D920079680A4492ED007AD7ED067A30
:100B200077EE677AC3ED007AFB699B003A6813445D
:100B30003A6D920039680A4492ED007AD7ED057A51
:100B400077EE677AC3ED007A3B6D9B007A681344B9
:100B50003A6D920079680A4492ED007AD7ED067AF0
:100B600077EE277AC3ED007A3B6D9B003A68134419
:100B70003A6D920039680A4492ED007AD7ED057A11
:100B800077EE277AC3ED007A3A6D3B6C13443B65F0
:100B90003A6D7B6D9A4283DB97ED0D7AD7ED0F7A34
:100BA00027EE277AD7ED0C6AD7ED0E7A66EEA77A94
:100BB00077EE677AC7ED047A97ED0D7AD7ED0E7A66
:100BC00027EE277AD7ED0C6AD7ED0F7A66EEA77A73
:100BD00077EE277AC7ED0C7A3B697B63FB6C0133B8
:100BE000FB64FA6C3B6A9A42FFF657AFF86BEFF77B
:100BF0003BFC03460C461A4623464FF0000044498E
:100C0000EFF7D2FA03460C46184621464FF0000291
:100C10004FF08043EFF7A6FD03460C4618462146E9
:100C2000F3F7A8FF03460C4618462146EFF768FF86
:100C30000346BB63B7F90E30012B05D1D7ED0E7A11
:100C4000F1EE677AC7ED0E7AF86BEFF70DFC4FF017
:100C500000022F4BEFF7AAFA03460C46184621462E
:100C60004FF000024FF08043EFF77CFD03460C4647
:100C700018462146F3F77EFF03460C4618462146E8
:100C8000EFF73EFF0346FB637B6C01337B647A6CBA
:100C9000BB689A42FFF6F3AEB7F90E30012B2FD1A5
:100CA00000233B6528E03B6D9B007A6813443A6D56
:100CB000920079680A44D2ED006A7A6D07EE902AB4
:100CC000B8EEE77AC6EE877AC3ED007A3B6D9B00FB
:100CD0003A6813443A6D920039680A44D2ED006ACA
:100CE0007A6D07EE902AB8EEE77AC6EE877AC3ED02
:100CF000007A3B6D01333B653A6D7B6D9A42D2DBE6
:100D0000012318465C37BD4690BD00BF000080BF80
:100D10000000F03F90B59BB000AFF860B96013469B
:100D2000FB71F8682CF051FD034683F00103DBB240
:100D3000002B11D1B8682CF0E0FB034683F00103CF
:100D4000DBB2002B0FD0B8682CF03FFD034683F0D8
:100D50000103DBB2002B06D0BB68FA68C64901204C
:100D600021F06CFB84E1F86828F002F80346FB648C
:100D700001237B6600233B6605E07B6E5B007B66A0
:100D80003B6E01333B667A6EFB6C9A42F5D322F0E0
:100D9000A1FA02467B6E2033DB009A4204D2B749A7
:100DA000012021F04BFB63E17B6E9B00073307338F
:100DB000DB08DB00ADEB030D6B460733DB08DB0024
:100DC000BB647B6E9B0007330733DB08DB00ADEBB6
:100DD000030D6B460733DB08DB007B6407F114036C
:100DE0000122F968184624F083FD0023FB6517E013
:100DF000FB6D5A1CFA659B00BA6CD41807F11403FA
:100E0000184624F013FF02460B4610461946EFF72A
:100E100077FE0346236007F11403184620F0C4FE52
:100E200007F11403184620F079FE0346002BDFD1AA
:100E300007F11403184620F009FF08E0FB6D5A1C67
:100E4000FA659B00BA6C13444FF000021A60FA6D09
:100E50007B6E9A42F2D30023FB65B8682CF0B5FC98
:100E60000346002B3AD007F114030122B968184653
:100E700024F03EFD17E0FB6D5A1CFA659B007A6C6E
:100E8000D41807F11403184624F0D0FE02460B468E
:100E900010461946EFF734FE0346236007F11403AA
:100EA000184620F081FEFA6D7B6E9A4207D207F158
:100EB0001403184620F032FE0346002BDBD107F165
:100EC0001403184620F0C2FE08E0FB6D5A1CFA65B8
:100ED0009B007A6C13444FF000021A60FA6D7B6E2F
:100EE0009A42F2D3FB79002B02D04FF0FF3000E0A2
:100EF00001207B6CBA6C396EFFF74EFDB8682CF0A0
:100F000064FC0346002B14BF01230023DBB283F0F3
:100F10000103DBB287F8433097F8433003F0010355
:100F200087F8433007F114030122F968184624F0CA
:100F3000DFFC0023FB6551E097F84330002B2AD0FB
:100F4000FB6D9B00BA6C134493ED007AFB6D9B0024
:100F5000BA6C1344D3ED007A27EE277AFB6D9B0021
:100F60007A6C1344D3ED006AFB6D9B007A6C1344DA
:100F7000D3ED007A66EEA77A77EE277A17EE900A1D
:100F8000EFF772FA03460C4618462146F3F7F2FDD6
:100F9000C7E914010BE0FB6D9B00BA6C13441B689E
:100FA0001846EFF761FA03460C46C7E91434D7E94F
:100FB00014012AF02FFB024607F1140311461846CC
:100FC00020F044FD034618462AF024F8FB6D013357
:100FD000FB6507F11403184620F0E6FD07F1140342
:100FE000184620F09BFD0346002BA5D107F1140302
:100FF000184620F02BFEB8682CF0E7FB0346002BC8
:1010000036D007F114030122B968184624F070FCA9
:101010000023FB651FE0FB6D5A1CFA659B007A6C90
:1010200013441B681846EFF71FFA03460C46184690
:1010300021462AF0EFFA024607F11403114618463A
:1010400020F004FD0346184629F0E4FF07F11403DD
:10105000184620F0A9FD07F11403184620F05EFDA4
:101060000346002BD7D107F11403184620F0EEFDFC
:101070006C37BD4690BD00BF089304085093040828
:10108000B0B596B000AFF860C7E90023F8682CF05F
:10109000CCF9034683F00103DBB2002B04D04FF000
:1010A00000034FF0000483E0D7E90001EFF708FDEB
:1010B00003467B657B6D1846EFF7C4F903460C4683
:1010C0001A462346D7E90001EFF76EF803460C46AF
:1010D000C7E912344FF000024FF00003D7E90001D6
:1010E000EFF788FC0346002B07D000237B654FF009
:1010F00000034FF00004C7E91234F86829F0A2F9A0
:101100000346013B1846EFF78DF9D7E90023EFF7C7
:101110007BFC0346002B0BD0F86829F093F90346BB
:10112000013B7B654FF000034FF00004C7E9123428
:1011300007F110037A6DF968184623F0A3FF07F151
:101140001003184624F09DF9C7E9100107F11003B8
:10115000184624F08DFB07F11003184624F091F98E
:10116000C7E90E0107F11003184624F0B2FBD7E9D6
:1011700012234FF000001149EFF716F803460C4612
:1011800018462146D7E91023EFF7C2F903460C466B
:1011900025461C46D7E91223D7E90E01EFF7B8F927
:1011A00002460B4620462946EFF700F803460C4658
:1011B000184621465837BD46B0BD00BF0000F03F7D
:1011C000B0B5A2B000AFF860B960C7E90023F86815
:1011D0002CF02BF9034683F00103DBB2002B04D083
:1011E0004FF000034FF000040FE1D7E92601EFF7BD
:1011F0003FFC0346C7F88430D7F88400EFF722F9A4
:1012000003460C461A462346D7E92601EEF7CCFFE3
:1012100003460C46C7E91E344FF000024FF00003AE
:10122000D7E92601EFF7E6FB0346002B08D00023A1
:10123000C7F884304FF000034FF00004C7E91E34B4
:10124000D7F88430BA6802FB03F31846EFF7FAF8D0
:10125000D7E90023EEF7AAFF03460C46C7E9163488
:10126000D7E91601EFF72CFC03467B677B6F184626
:10127000EFF7E8F803460C461A462346D7E916016D
:10128000EEF792FF03460C46C7E91A344FF000020E
:101290004FF00003D7E90001EFF7ACFB0346002B4A
:1012A0000BD0D7F88430BA6802FB03F37B674FF0AA
:1012B00000034FF00004C7E91A3407F110037A6FF6
:1012C000F968184623F0DEFE07F11003184624F0F3
:1012D000D8F8C7E9140107F11003184624F0C8FA3A
:1012E00007F11003184624F0CCF8C7E91201D7E93A
:1012F0001A234FF000004749EEF756FF03460C460D
:1013000018462146D7E91423EFF702F903460C46A5
:1013100025461C46D7E91A23D7E91201EFF7F8F85A
:1013200002460B4620462946EEF740FF03460C4690
:10133000C7E9103401237B6607E007F11003184664
:1013400024F096FA7B6E01337B667A6EBB689A4214
:10135000F3DB07F11003184624F093F8C7E91401F2
:1013600007F11003184624F083FA07F1100318461A
:1013700024F087F8C7E9120107F11003184624F09A
:10138000A8FAD7E91A234FF000002249EEF70CFF24
:1013900003460C4618462146D7E91423EFF7B8F860
:1013A00003460C4625461C46D7E91A23D7E9120105
:1013B000EFF7AEF802460B4620462946EEF7F6FE5A
:1013C00003460C46C7E90E34D7E91E234FF0000050
:1013D0001049EEF7E9FE03460C4618462146D7E9C8
:1013E0001023EFF795F803460C4625461C46D7E92F
:1013F0001E23D7E90E01EFF78BF802460B46204675
:101400002946EEF7D3FE03460C4618462146883798
:10141000BD46B0BD0000F03F90B585B000AFC7E954
:1014200002017A604FF000024FF00003D7E9020199
:10143000EFF7E0FA0346002B08D1D7E90223D7E9FA
:101440000201EFF7FFFA0346002B04D04FF0000330
:10145000124CC7E9023478682CF04FF80346002B91
:1014600005D1786828F084FC0346002B07D00C4B8C
:101470001B8843F400739AB2094B1A8006E0084BAC
:101480001B8823F400739AB2054B1A80D7E9020136
:1014900005F04AFB1437BD4690BD00BF0000F03F89
:1014A0009C51012080B500AF05F0B4FB80BD000069
:1014B00080B584B000AF0346FB712AF013F9F860E1
:1014C000FB68002B01D100235BE0FB7903F00103F3
:1014D000002B07D02D4829F0A5FF03461946F868D0
:1014E00024F00EFCFB7903F00203002B07D0284800
:1014F00029F098FF03461946F86824F001FCFB79AF
:1015000003F00403002B07D0224829F08BFF034689
:101510001946F86824F0F4FBFB7903F00803002B6C
:1015200007D01D4829F07EFF03461946F86824F0CD
:10153000E7FBFB7903F01003002B07D0174829F0D5
:1015400071FF03461946F86824F0DAFBFB7903F0D3
:101550002003002B07D0124829F064FF03461946E8
:10156000F86824F0CDFBFB7903F04003002B07D093
:101570000C4829F057FF03461946F86824F0C0FBD1
:10158000FB6818461037BD4680BD00BF789304083D
:1015900084930408909304089C930408A09304087F
:1015A000A8930408B493040880B582B000AF074B39
:1015B0001B78FB71054B00221A70FB791846FFF768
:1015C00077FF034618460837BD4680BD4D510120C0
:1015D00080B582B000AF786078682BF0DAFD034602
:1015E00083F00103DBB2002B01D0002304E00021D3
:1015F00078682AF0D9F8034618460837BD4680BDFA
:1016000080B582B000AF786039607B68DBB2194684
:10161000386823F044FB386823F070FB0837BD4678
:1016200080BD000080B58CB000AF7860786827F08E
:1016300059FB0346012B39D10021786827F044FD7E
:10164000B862B86A2BF008FE0346002B01D0BB6AD3
:1016500057E0B86A2BF0E9FE0346002B23D0BB6AA3
:101660009B8803F00F03012B1DD1BB6A1B88002B45
:1016700019D1B86A28F004FF7862786A2BF0ECFD83
:101680000346002B0CD0786A2CF06AFB0246BB6A3A
:101690005B889A4204D1B86A29F0BCFC7B6A30E0CE
:1016A000786A29F0B7FCB86A29F0B4FC786823F0AE
:1016B000C5F903463B62386A29F0ECFDF862FB6A23
:1016C000002B05D126F0A6F8386A29F0E3FDF86270
:1016D000FB6A002B01D1002313E007F10C03002269
:1016E000F96A184623F0F8F907F10C031A4607497E
:1016F000786823F06DF807F10C03184604F044F8FD
:10170000FB6A18463037BD4680BD00BF0116010890
:1017100080B582B000AF786039607B68DBB2194673
:10172000386824F02FF8386824F0A2F80837BD464E
:1017300080BD000080B58EB000AF7860786823F07F
:101740007DF903461946012022F0FCFE78637B6B8D
:10175000002B01D1002313E007F10C030022796B69
:10176000184623F08FFC07F10C031A4606497868E7
:1017700023F02EF807F10C03184624F0AAF87B6B2F
:1017800018463837BD4680BD1117010880B584B0B2
:1017900000AF78604FF43073FB8103F0E9FFB8606D
:1017A000BB68002B05D0FB891A46B9687868FAF740
:1017B00017FBBB6818461037BD4680BD80B584B0A6
:1017C00000AF786039603B68002B01DA00230BE042
:1017D0007B68184605F0D6FBF860FB683A6811464E
:1017E000184629F0C6FF034618461037BD4680BD8F
:1017F00080B582B000AF78600B46FB7078682BF044
:10180000C8FC0346002B04D078682CF027FE7860D3
:1018100002E003F0ADFF7860FB78194678682BF0A2
:1018200057F9786829F0F6FB0837BD4680BD80B5CA
:1018300082B000AF7860786805F0F0FB0346184688
:101840000837BD4680BD000080B485B000AF786029
:101850007B68DBB2FB60FA6813469B0213445B00B3
:101860000B4A1A40F9680B469B020B445B01194670
:10187000084B0B401A4313461B0213441B0213442C
:101880001B0CDBB218461437BD465DF8047B70476D
:10189000102102004084080080B500AF10F0DEFF88
:1018A00080BD80B500AF22F06BFB80BD80B500AF7E
:1018B00022F0D6FB80BD000080B588B000AF786014
:1018C00039603B68002B68DD78682CF0CDF9034661
:1018D000002B62D029F006FFF861FB69002B01D1D3
:1018E000002362E007F10C037968184623F022FB1D
:1018F00044E007F10C03184603F052FFB861B869E1
:1019000028F0E6FF786129F0E5FE38613B69002B9D
:101910002BD0B8692AF0F0FC03461A4625493869ED
:1019200027F030F90021B869FFF7C6FF03461A46D1
:101930002149386927F026F93B68012B11DD7869C8
:101940002CF092F90346002B0BD03B68013B194663
:101950007869FFF7B1FF03461A461849386927F03E
:1019600011F93969F86924F0CBF9B969786929F076
:101970007DFB07F10C03184623F02FFB07F10C0346
:10198000184603F021FF0346002BB2D107F10C03E8
:10199000184603F02AFFFB6907E0786827F0E5FAAC
:1019A0000346184629F00AFE034618462037BD466E
:1019B00080BD00BF707B040808A80408C493040815
:1019C00080B584B000AF78600B46FB70FB78002BCD
:1019D00009D00023FB6007F10C03194678682AF050
:1019E000E3FE034600E07B6818461037BD4680BD25
:1019F00080B5A2B002AFF860B9607A603B60F86869
:101A00002BF013FD034683F00103DBB2002B08D15A
:101A1000B8682BF00AFD034683F00103DBB2002B0C
:101A200004D07B49012020F009FDEDE07B68002B0C
:101A30001FD078682BF0DFFC034683F00103DBB294
:101A4000002B16D078682BF0F0FC034683F00103DE
:101A5000DBB2002B0DD078682BF053FC034683F0EB
:101A60000103DBB2002B04D06A49012020F0E6FC20
:101A7000CAE078682BF045FC034687F87330FB68B2
:101A80009B8803F00F03DB00FB663B68002B03DD44
:101A90003A68FB6E9A4201DDFB6E3B600023FB67F8
:101AA00007F140030022F968184623F0EBFA07F12A
:101AB0004003184623F0B6FCB86707F1180300226C
:101AC000B968184623F0DEFA83E0FA6E3B68D31A51
:101AD000BA6F1A4101213B6801FA03F3013B13403D
:101AE000BB66BA6F3B6802FA03F3BB67FA6F3B68E9
:101AF0001344FB67FA6FFB6E9A420CDB0023FB6713
:101B000007F14003184623F0B3FE07F140031846DF
:101B100023F088FCB8677B68002B4FD000237B67DD
:101B200097F87330002B1ED0B86E29F047FD03469E
:101B30003B6107F14003184623F067FE03467B61D3
:101B400007F11003019302230093002300220021D8
:101B500078681EF0B9FA786707F110031946022079
:101B600029F0BAFA20E078682BF045FC0346002BF8
:101B700005D0B96E786827F0A7FA786714E078681E
:101B80002BF053FC034683F00103DBB2002B05D09E
:101B9000214A40F2E741214820F0C4FCBB6E1946BF
:101BA000786828F0A1FC786707F11803796F184668
:101BB00023F05EFD786F29F02DFA05E007F1180398
:101BC000B96E184623F0F0FC07F11803184623F00D
:101BD0004FFE07F14003184623F025FE0346002B75
:101BE00008D007F11803184623F01DFE0346002B0A
:101BF0007FF46BAF07F14003184623F06AFE07F14C
